:100000000C94B4050C94DF050C94DF050C94DF050B
:100010000C940E0E0C94DF050C94DF050C94DF0598
:100020000C94DF050C94DC2E0C94DF050C94DF059A
:100030000C94DF050C9453380C94DF050C94DF0509
:100040000C94DF050C94DF050C9459840C94DF05A7
:100050000C9455820C94A0820C94DF050C94DF055F
:100060000C94DF050C94DF050C948E800C94DF0556
:100070000C94700D0C94DF820C94DF050C94DF055A
:100080000C94DF050C94DF050C94DF052D33002D57
:1000900032002D31002030002B31002B32002B3369
:1000A000002B340020430020432300204400204440
:1000B0002300204500204600204623002047002042
:1000C000472300204100204123002042004D53548B
:1000D000004D494400434C4B00322F3100312F3149
:1000E00000312F3200312F34003132700032347041
:1000F000003438700053494E005452490053415760
:100100000053515500532F48004457320044573391
:100110000044573400445735004457360054573193
:100120000054573200545733005457340045585048
:1001300000485244005346540046555A0053504B11
:1001400000535450004F666600313A3200313A3362
:1001500000313A3400313A3500313A3600313A371D
:1001600000313A3800323A3300333A3400373A3803
:100170000031302500323525003530250037352552
:100180000039302500434852004D414A006D696EE8
:100190000050454E00444F5200504852004C5944C4
:1001A000004D4958004C4F4300464F52574152446E
:1001B0002020004241434B57415244200050494EB9
:1001C000472D504F4E470052414E444F4D20202066
:1001D0000053594E0042504D00545258004356525D
:1001E0005800434C4B004E430041430050545200D2
:1001F0004C454E0053434C0054524947004C464F27
:10020000005741560046525100414D500053545042
:10021000004E5445004F4354004C454E4700555442
:100220004D0050524F00525452470050554C00421E
:1002300041520043505900415554004D414E004F2A
:10024000464600204F4E0052535400504F53005327
:100250004E47004D555400524F4F00202020004281
:1002600044005344005331005332004C54004D5469
:10027000004854004350004348004F480043520098
:100280005244003576200031307600D101D5012B63
:1002900002E201330247025302E901EC01F001F4EA
:1002A00001F801FD010102050209022F02110215E8
:1002B000021902F401E601E601E6012F021E022204
:1002C0000226022F021E02220219022F02F001F45E
:1002D00001F8014F024B02EC01F001110215020D71
:1002E000021902F401570215025B02A901B301BD14
:1002F00001C701850189018D019101950199019D38
:1003000001A101A501450149014D015101550159C5
:10031000015D016101650169016D0171017501797D
:10032000017D018101F500F900FD000101050109D0
:10033000010D011101150119011D012101250129DD
:10034000012D013101350139013D014101D900DDA6
:1003500000E100E500E900ED00F100CD00D100D59D
:10036000008C008F009200950098009B009E00A1D9
:1003700000A400A700AB00AE00B200B500B800BCFE
:1003800000BF00C300C600CA005F026202650268C7
:10039000026B026E027102740277027A027D0280A1
:1003A000023B0237023F024302830287020102033B
:1003B0000405060708090A0B0C01010303050606DC
:1003C00008080A0A0C0101030304060608080909C3
:1003D0000B0101030303050508080A0A0A010103CA
:1003E0000304060608080A0A0B01010202040606B5
:1003F000080809090B0101030305070708080A0A91
:100400000C0101030305060608080A0A0B01010294
:1004100002040606070709090B00002B005500809F
:1004200000AB00D50000012B0155018001AB01D5C7
:1004300001807C797673706D6A6763605D5A57548A
:10044000514F4C494643403E3B383633312E2C2ADF
:10045000272523211F1D1B1917151312100F0D0C13
:100460000A09080706050403030201010000000051
:10047000000000000000000101020303040506075C
:1004800008090A0C0D0F1012131517191B1D1F2137
:100490002325272A2C2E313336383B3E404346490C
:1004A0004C4F5154575A5D6063676A6D707376792B
:1004B0007C808386898C8F9295989C9FA2A5A8ABFF
:1004C000AEB0B3B6B9BCBFC1C4C7C9CCCED1D3D509
:1004D000D8DADCDEE0E2E4E6E8EAECEDEFF0F2F3B5
:1004E000F5F6F7F8F9FAFBFCFCFDFEFEFFFFFFFF57
:1004F000FFFFFFFFFFFFFFFEFEFDFCFCFBFAF9F82C
:10050000F7F6F5F3F2F0EFEDECEAE8E6E4E2E0DE30
:10051000DCDAD8D5D3D1CECCC9C7C4C1BFBCB9B63B
:10052000B3B0AEABA8A5A29F9C9895928F8C8986FC
:10053000837C7A78767472706E6C6A6866646260C6
:100540005E5C5A58565452504E4C4A4846444240BB
:100550003E3C3A38363432302E2C2A2826242220AB
:100560001E1C1A18161412100E0C0A08060402019A
:100570000000020406080A0C0E10121416181A1CA9
:100580001E20222426282A2C2E30323436383A3C9B
:100590003E40424446484A4C4E50525456585A5C8B
:1005A0005E60626466686A6C6E70727476787A7C7B
:1005B0007E80828486888A8C8E90929496989A9C6B
:1005C0009EA0A2A4A6A8AAACAEB0B2B4B6B8BABC5B
:1005D000BEC0C2C4C6C8CACCCED0D2D4D6D8DADC4B
:1005E000DEE0E2E4E6E8EAECEEF0F2F4F6F8FAFC3B
:1005F000FEFEFCFAF8F6F4F2F0EEECEAE8E6E4E2ED
:10060000E0DEDCDAD8D6D4D2D0CECCCAC8C6C4C2DA
:10061000C0BEBCBAB8B6B4B2B0AEACAAA8A6A4A2CA
:10062000A09E9C9A98969492908E8C8A88868482BA
:10063000807E0102030405060708090A0B0C0D0E53
:100640000F101112131415161718191A1B1C1D1E42
:100650001F202122232425262728292A2B2C2D2E32
:100660002F303132333435363738393A3B3C3D3E22
:100670003F404142434445464748494A4B4C4D4E12
:100680004F505152535455565758595A5B5C5D5E02
:100690005F606162636465666768696A6B6C6D6EF2
:1006A0006F707172737475767778797A7B7C7D7EE2
:1006B0007F808182838485868788898A8B8C8D8ED2
:1006C0008F909192939495969798999A9B9C9D9EC2
:1006D0009FA0A1A2A3A4A5A6A7A8A9AAABACADAEB2
:1006E000AFB0B1B2B3B4B5B6B7B8B9BABBBCBDBEA2
:1006F000BFC0C1C2C3C4C5C6C7C8C9CACBCCCDCE92
:10070000CFD0D1D2D3D4D5D6D7D8D9DADBDCDDDE81
:10071000DFE0E1E2E3E4E5E6E7E8E9EAEBECEDEE71
:10072000EFF0F1F2F3F4F5F6F7F8F9FAFBFCFDFE61
:10073000FF000000000000000000000000000000BA
:1007400000000000000000000000000000000000A9
:100750000000000000000000000000000000000099
:100760000000000000000000000000000000000089
:100770000000000000000000000000000000000079
:100780000000000000000000000000000000000069
:100790000000000000000000000000000000000059
:1007A0000000000000000000000000000000000049
:1007B0000000FFFFFFFFFFFFFFFFFFFFFFFFFFFF47
:1007C000FFFFFFFFFFFFFFFFFFFFFFFFFFFFFFFF39
:1007D000FFFFFFFFFFFFFFFFFFFFFFFFFFFFFFFF29
:1007E000FFFFFFFFFFFFFFFFFFFFFFFFFFFFFFFF19
:1007F000FFFFFFFFFFFFFFFFFFFFFFFFFFFFFFFF09
:10080000FFFFFFFFFFFFFFFFFFFFFFFFFFFFFFFFF8
:10081000FFFFFFFFFFFFFFFFFFFFFFFFFFFFFFFFE8
:10082000FFFFFFFFFFFFFFFFFFFFFFFFFFFFFFFFD8
:10083000FFFF202837465564738291202020200036
:100840002E2E2E2E2E2E2E2E2E2E2E2E2E2E2E2EC8
:1008500000444143732063616C6962726174696F23
:100860006E0020696E697469616C697A6174696F80
:100870006E20002020202020454550524F4D202042
:10088000202020002B002D00546F74616C204163E8
:10089000632076616C756520005B436F70696564E9
:1008A000215D005B5341564544215D00783200785C
:1008B0003100202020202020202020202020202047
:1008C0002020002020202000202020200020202088
:1008D000200020202020001018203040608020536D
:1008E0007465702020204163632F566F6C74006E16
:1008F0007465206F637420737470206C656E67007C
:100900005074726E2000506F73200020536F6E671A
:1009100020506C6179205300736E6720706F7320D4
:10092000707472206C656E20004F6E004F6666001A
:100930004F6E004F66660020204C464F73202043C8
:10094000562F4761746520007300626172207574D0
:100950006D2070726F207274726700626172207510
:10096000746D2070726F206C656E67006C666F200E
:100970007761762066727120616D70200073636C00
:1009800020726F6F206F637420202020200073007E
:10099000626172206E7465206F6374206C656E678F
:1009A0000020202000312F0046494C4C006261722B
:1009B000206C656E2073636C2074726967007363CA
:1009C0006C20726F6F206F637420202020200062E3
:1009D0006172206C656E2073636C207472696700AD
:1009E0004558540020205061747465726E20506C1C
:1009F0006179202000202020426172202020205395
:100A0000746570202000200061630063707920729B
:100A10007374206D75740073796E2062706D207030
:100A2000756C20636C6B2000205472636B206469CA
:100A300072656374696F6E2000205074726E20645A
:100A40006972656374696F6E20002B002D00202091
:100A500053687566666C652076616C75652000006C
:100A600002040507090B0002050709000304081228
:100A70001313111F000000000000000018040209F9
:100A800019191110080601000000000004001F00E1
:100A900000000001020C10000000001010111204F0
:100AA0000810000000171417151700000010181088
:100AB000100C0000000E0A0E0A0E0000001B091B9D
:100AC0000A1B0001010101010F1F0E00000A0A0E9E
:100AD00002020000000E020E080E0076312E3035A4
:100AE000350000002100240027002A000000220019
:100AF000250028002B0000002000230026002900EC
:100B000002020202020202020404040404040404B5
:100B100003030303030303030101010101010101B5
:100B200001020408102040800102040810204080C7
:100B300001020408102040800102040810204080B7
:100B4000000000010200080900000000040307067D
:100B50000000000000000000000000000000000095
:100B6000C727267FC383C02711241FBECFEFD0E441
:100B7000DEBFCDBF11E0A0E0B1E0E0E1FCE101E0CB
:100B80000BBF02C007900D92AC3EB107D9F71BBE58
:100B90001BE3ACEEB1E001C01D92A03AB107E1F752
:100BA0001BE0C6E6DBE004C02297FE010E94C08D78
:100BB000C036D107C9F70E9413860C94FB8D0C94A4
:100BC0000000CF93DF93BC018230910510F462E006
:100BD00070E0A0919E3BB0919F3BED01E0E0F0E022
:100BE00040E050E021C0888199818617970769F419
:100BF0008A819B81309719F09383828304C09093FC
:100C00009F3B80939E3BFE0134C06817790738F400
:100C10004115510519F08417950708F4AC01FE0140
:100C20008A819B819C01E9012097E9F641155105D4
:100C3000A9F1CA01861B970B049708F4BA01E0E0FA
:100C4000F0E02AC08D919C91119784179507F9F4D3
:100C50006417750781F412968D919C9113973097C4
:100C600019F09383828304C090939F3B80939E3BB3
:100C7000FD0132964CC0CA01861B970BFD01E80F9F
:100C8000F91F6193719302978D939C9340C0FD016E
:100C9000828193819C01D9011097A1F680919C3BA0
:100CA00090919D3B892B41F48091240190912501E5
:100CB00090939D3B80939C3B40912601509127014E
:100CC0004115510541F44DB75EB7809122019091D5
:100CD0002301481B590B20919C3B30919D3BCA013D
:100CE000821B930B8617970780F0AB014E5F5F4F17
:100CF0008417950750F0420F531F50939D3B40932C
:100D00009C3BF9016193719302C0E0E0F0E0CF01F8
:100D1000DF91CF910895CF93DF93009709F450C0EE
:100D2000EC0122971B821A82A0919E3BB0919F3BBF
:100D3000109709F140E050E0AC17BD0708F1BB8304
:100D4000AA83FE0121913191E20FF31FAE17BF0775
:100D500079F48D919C911197280F391F2E5F3F4F89
:100D60003983288312968D919C9113979B838A8354
:100D70004115510571F4D0939F3BC0939E3B20C019
:100D800012968D919C911397AD01009711F0DC01A3
:100D9000D3CFFA01D383C28321913191E20FF31FA4
:100DA000CE17DF0769F488819981280F391F2E5FDC
:100DB0003F4FFA01318320838A819B819383828311
:100DC000DF91CF910895A0E0B0E0E9EEF6E00C9459
:100DD000CC8DEC01A880B980CA80DB80A114B1045D
:100DE000C104D10441F484E2A82E89EDB82E8BE52C
:100DF000C82E87E0D82EC601B5012DE133EF41E0C2
:100E000050E00E94A38D27EA31E440E050E00E94C8
:100E10002F8D7B018C01C601B5012DE133EF41E03F
:100E200050E00E94A38DCA01B9012CEE34EF4FEFC0
:100E30005FEF0E942F8D6E0D7F1D801F911F97FF0A
:100E400004C06150704080409048688379838A83F1
:100E50009B839B01AC015F77B901CA01CDB7DEB7B7
:100E6000EAE00C94E88D0E94E306089588E291E0A0
:100E70000E94E306089560932801709329018093EE
:100E80002A0190932B010895A0E0B0E0EAE4F7E096
:100E90000C94C68D6C01009729F4CB010E94E105EA
:100EA0006C01C1C08EEF882E8FEF982E8C0C9D1C8C
:100EB0008601060F171F0815190508F4B2C0F401C2
:100EC000A081B181A617B707B8F0A530B10508F425
:100ED000AAC0CD0104978617970708F4A4C01297FB
:100EE000A61BB70BF801A193B193D4016D937C932A
:100EF000CF010E948B0697C07B01EA1AFB0AEEEF36
:100F0000FFEFEE0EFF1E36016A0E7B1EC0919E3B68
:100F1000D0919F3B44245524AA24BB244AC0C61523
:100F2000D705E1F5488159814E155F05B8F1CA0131
:100F300004978E159F05B0F41296A40FB51FF40107
:100F4000B183A0832A813B814114510431F0D20145
:100F500013963C932E93129766C030939F3B209339
:100F60009E3B61C08A819B81F801938382834250BA
:100F700050404E195F09518340834114510431F0B0
:100F8000D20113961C930E93129704C010939F3BAB
:100F900000939E3BF4017183608345C088819981F1
:100FA000A816B90608F45C012E018A819B819C0178
:100FB000E901209709F0B3CF80919C3B90919D3B34
:100FC00086159705E9F4A616B706D0F420912601F8
:100FD000309127012115310541F42DB73EB780919D
:100FE000220190912301281B390B02171307C8F423
:100FF00010939D3B00939C3BD4016D937C9313C055
:10100000CB010E94E105EC01009759F0F401408109
:101010005181B6010E942008C6010E948B066E0114
:1010200002C0CC24DD24C601CDB7DEB7E0E10C94CC
:10103000E28DFB01DC0105900D920020E1F708959F
:10104000FB01DC0102C001900D9241505040D8F7E5
:101050000895FB01DC018D91019080190110D9F3F5
:10106000990B0895FB01DC0101900D920020E1F73E
:101070000895FB019F01E8944230C4F04532B4F476
:101080004A3029F497FB1EF4909581959F4F642F69
:1010900077270E945A8D805D8A330CF0895D819399
:1010A000CB010097A1F716F45DE251931082C901BC
:1010B0000C947008FB019F01423074F0453264F4D7
:1010C000642F77270E945A8D805D8A330CF0895DEA
:1010D0008193CB010097A1F71082C9010C9470088D
:1010E000DC01FC01672F71917723E1F7329704C08F
:1010F0007C916D9370836291AE17BF07C8F308951A
:10110000CF92DF92EF92FF920F931F93CF93DF93D3
:10111000382F90914F3680E020914E36022F10E00C
:10112000082B192B332321F0313009F047C047C079
:10113000C3E7D7E340E050E081E0C82ED12CE12C9A
:10114000F12CC801042E02C0969587950A94E2F707
:10115000282F2170FA01ED57F84C20838881281739
:1011600031F1213021F5CB01042E02C096958795EF
:101170000A94E2F780FF0FC0D701C601042E04C015
:10118000880F991FAA1FBB1F0A94D2F780959095CC
:10119000682379230CC0D701C601042E04C0880F30
:1011A000991FAA1FBB1F0A94D2F7682B792B29938A
:1011B0004F5F5F4F4031510521F602C002C0B801B8
:1011C000CB01DF91CF911F910F91FF90EF90DF90B6
:1011D000CF9008952F923F924F925F926F927F929D
:1011E0008F929F92AF92BF92CF92DF92EF92FF9237
:1011F0000F931F93DF93CF9300D000D0CDB7DEB70E
:101200001C018091933685FF03C081E08093623793
:101210008091B1028A83482F50E0FA01E25BF44DDD
:101220006080629430EF63222091352B30E0909102
:10123000B903998390904C027090623703E617E3EC
:1012400060E070E084EC90E0489F5001499FB00C52
:10125000589FB00C112485E29DE0289F7001299FC2
:10126000F00C389FF00C11246A01CE0CDF1CA9ECA5
:10127000B3E0CA0EDB1E2BE3422E2BE2522E440EAD
:10128000551E562D560FE52FF0E0FC83EB83EE0F35
:10129000FF1F8B819C81E80FF91FEA0DFB1DEE0DEE
:1012A000FF1DE452FC4F8081382F3170282F269586
:1012B0002170D6018C90C101062E02C096958795AB
:1012C0000A94E2F7482F4170DB01AA0FBB1FFD0112
:1012D000E959F94C90819E7F942B9083892F8695B4
:1012E0008170481711F4592D90C09695969591707C
:1012F000913009F053C0442309F061C0332309F44D
:101300005EC0222371F4882009F4B2C0F801808104
:10131000882309F0ADC0772009F0AAC0592D21E03B
:101320004FC0F8018081882309F0A4C0772009F01C
:10133000A1C0FD01E60FF71F8A81803191F0EA0D0F
:10134000FB1DEE0DFF1DDF01A452BC4F8C9183707D
:101350008C93E352FC4F84E08083D2019C9330E075
:101360008AC0EE0DFF1DDF01AB5DBF4E8C918E7FFD
:101370008C93EA5DFF4E8081877080839C911196EB
:101380008C911197887F846011968C93119791703E
:1013900098619C9330E021E0298311C0992379F46E
:1013A000413069F4F2014083332331F4D8014C9386
:1013B00020E0882009F421E031E0772401C0592D94
:1013C000EB81FC81EE0FFF1F8B819C81E80FF91FE1
:1013D000EA0DFB1DEE0DFF1DE452FC4F80818C7F5A
:1013E0002170220F832B822B8083FB01EE0FFF1FC6
:1013F000E959F94C942F990F990F80818B7F892B94
:101400008083442311F4D8011C92FB01EE0FFF1FCF
:10141000E959F94C8081982F9170990F8D7F892B14
:1014200080836F5F7F4F0F5F1F4F6031710511F039
:10143000952E27CFB981B093B90350934C02709287
:1014400062370F900F900F900F90CF91DF911F9107
:101450000F91FF90EF90DF90CF90BF90AF909F9053
:101460008F907F906F905F904F903F902F90089556
:1014700031E0A5CF31E021E0A2CF9F92AF92BF92A1
:10148000CF92DF92EF92FF920F931F93CF93DF9350
:101490005C010091B102402F50E02091352B30E0EB
:1014A000FA01E25BF44D10811295107FA091B9030F
:1014B00060E070E085E29DE0289FE001299FD00D6B
:1014C000389FD00D11249924939484EC90E0489F88
:1014D0006001499FD00C589FD00C11249BE3E92E4A
:1014E0009BE2F92EE40EF51EC501062E02C096956C
:1014F00087950A94E2F7482F4170FB01EE0FFF1F1A
:10150000E959F94C90819E7F942B9083892F869581
:101510008170481709F459C092FD4DC0413009F05F
:101520004AC0812F860F282F30E090E0F901EE0F9E
:10153000FF1FE20FF31FEC0FFD1FEB5DFF4E8081DD
:1015400080FF91E0F901EE0FFF1FE20FF31F9F01F3
:101550002C0F3D1FD901AB5DBF4E8C918E7F892B27
:101560008C93992339F5003189F0EC0DFD1DEC0FBA
:10157000FD1FDF01A452BC4F8C9183708C93E3520A
:10158000FC4F84E08083F701908214C08E7F8C939F
:10159000F901EA5DFF4E8081877080839C911196EE
:1015A0008C911197887F846011968C93119791701C
:1015B00098619C93A1E0FB01EE0FFF1FE959F94CE4
:1015C000440F80818D7F842B80836F5F7F4F6031DC
:1015D000710509F089CFA093B903DF91CF911F91D5
:1015E0000F91FF90EF90DF90CF90BF90AF909F90C2
:1015F0000895AF92BF92CF92DF92EF92FF920F9336
:101600001F93CF93DF93EC01D0908736D694D69476
:1016100081E0D822A0902C01C090392BB090F2022A
:101620004091F0335091F13320E030E0E1E0EE2ED4
:10163000F12C012D112DF901EE0FFF1FE959F94C85
:101640006081CE01022E02C0969587950A94E2F73A
:10165000782F7170667F962F972B9083892F8695B0
:101660008170781709F453C092FD51C0713009F0B0
:101670004EC069606083DD2031F1CC2081F0CA0169
:10168000022E02C0969587950A94E2F780FD24C049
:10169000AA24A394CC24BB2440E050E038C0D80155
:1016A000C701022E04C0880F991FAA1FBB1F0A94EE
:1016B000D2F7AC0140955095AA24A394CC24C394AE
:1016C000BB24B39424C0CA01022E02C0969587950C
:1016D0000A94E2F780FF0FC0D801C701022E04C0B0
:1016E000880F991FAA1FBB1F0A94D2F78095909567
:1016F000482359230CC0D801C701022E04C0880F0B
:10170000991FAA1FBB1F0A94D2F7482B592BF90126
:10171000EE0FFF1FE959F94C8081982F9170990FB6
:101720008D7F892B80832F5F3F4F2031310509F05A
:1017300082CFA0922C01C092392BB092F20250932A
:10174000F1334093F033DF91CF911F910F91FF90D0
:10175000EF90DF90CF90BF90AF90089581E060E070
:1017600070E00E948008AC019093613780936037ED
:1017700020E030E0CA01022E02C0969587950A94B7
:10178000E2F780FF02C0822F08952F5F3F4F203184
:10179000310581F78FEF089581E060E070E00E94ED
:1017A0008008AC0190935F3780935E3760E020E063
:1017B00030E0CA01022E02C0969587950A94E2F79E
:1017C00080FF05C0613011F4822F089561E02F5F22
:1017D0003F4F2031310569F780E008953F924F92E5
:1017E0005F926F927F928F929F92AF92BF92CF92B1
:1017F000DF920F93DF93CF93CDB7DEB72C970FB661
:10180000F894DEBF0FBECDBF382E462E8091352B0B
:1018100090E0552425E23DE0829FA001839F500D7A
:10182000929F500D11245C874B874F5D5F4E5A830A
:101830004983832D90E0A0E0B0E08B839C83AD834F
:10184000BE83862F90E0A0E0B0E08F839887A987C1
:10185000BA8786C090E3491689F4852D90E0FC0193
:10186000EE0FFF1FE80FF91FAB85BC85EA0FFB1FCA
:10187000EB5DFF4E00810E730E5F24C0852D90E05E
:10188000B0E64B1681F4FC01EE0FFF1FE80FF91FC5
:101890004B855C85E40FF51FEB5DFF4E0081000F6B
:1018A0000C770C5F0FC0FC01EE0FFF1FE80FF91F54
:1018B0008B859C85E80FF91FEB5DFF4E0081069537
:1018C0000F710F5F6B817C818D819E810E94168CD0
:1018D0005B016C016F81788589859A850E94168CE1
:1018E0003B014C01602F70E080E090E00E94168C7C
:1018F0009B01AC01C401B3010E947D8B9B01AC0133
:10190000C601B5010E947D8B20E030E040E05FE33E
:101910000E94158B20E030E040E85FE30E94148BCA
:101920000E94EA8B90E3391611F4669505C0A0E693
:101930003A1611F466956695852D90E0FC01EE0F40
:10194000FF1FE80FF91F4B855C85E40FF51FEB5D6A
:10195000FF4E6F71660F8081817C862B808353944C
:10196000A981BA818C91851508F074CF1092B603C5
:101970001092B5032C960FB6F894DEBF0FBECDBF04
:10198000CF91DF910F91DF90CF90BF90AF909F905C
:101990008F907F906F905F904F903F9008950F933E
:1019A0001F93CF93DF939091352B092F10E0C82F11
:1019B000D0E0FE01EE0FFF1FEC0FFD1F85E29DE062
:1019C000089FD001099FB00D189FB00D1124EA0F98
:1019D000FB1FE95DFF4E8081482F429547708F7055
:1019E000A15EBF4E2C91680FE82FF0E0CF01861B5F
:1019F000910981309105E1F430E0C901880F991F08
:101A0000820F931F880F991F880F991FE80FF91FE6
:101A1000E355FC4F20E0349102C0615021E0FC010D
:101A2000E60FF11DE355FC4FE4913E17B1F31DC0E5
:101A30008F5F9F4FC9F430E0C901880F991F820F53
:101A4000931F880F991F880F991FE80FF91FE355FF
:101A5000FC4F249101C06F5FFC01E60FF11DE355BF
:101A6000FC4FE4912E17B9F320E06F3F19F44423A3
:101A700019F412C06C3098F0473011F4222371F041
:101A80006F3F31F4442321F0415040F440E006C060
:101A90004F5F473008F047E060E001C06BE0FE01B7
:101AA000EE0FFF1FEC0FFD1F85E29DE09C01029FE2
:101AB000C001039F900D129F900D1124E80FF91F94
:101AC000E95DFF4E6F708081807847704295407F5E
:101AD000862B842B8083DF91CF911F910F910895E6
:101AE0001F920F920FB60F9211242F933F934F9393
:101AF0005F938F939F93AF93BF939091CE0080910C
:101B000048028370813009F07CC0983F08F479C0A6
:101B10009A3F31F09C3F09F1983F09F072C020C014
:101B2000809304361092213610922236109223367A
:101B3000109224368091213690912236A09123363E
:101B4000B091243680931B3690931C36A0931D369B
:101B5000B0931E3610925D3754C08093053651C045
:101B600080915D378F5F80935D37863008F449C080
:101B700010925D3780911B3690911C36A0911D36D6
:101B8000B0911E3620912136309122364091233675
:101B900050912436821B930BA40BB50B80936801E4
:101BA00090936901A0936A01B0936B0180916801E1
:101BB00090916901A0916A01B0916B01CC97A10548
:101BC000B10560F48CE390E0A0E0B0E080936801A0
:101BD00090936901A0936A01B0936B0181E08093B7
:101BE000263680911B3690911C36A0911D36B091FF
:101BF0001E368093213690932236A0932336B093DD
:101C00002436BF91AF919F918F915F914F913F91FA
:101C10002F910F900FBE0F901F9018951F920F924B
:101C20000FB60F920BB60F9211242F933F934F9341
:101C30005F938F939F93AF93BF93EF93FF9380B185
:101C4000817080932F3690912F368091303698177F
:101C5000B9F180912F36882379F581E08093313670
:101C600010924E02EAE0F6E3819326E3EB31F207AD
:101C7000D9F72C9A2C9810924902109233011092A5
:101C8000320180E090E021E0FC01E05AFD4F10823B
:101C9000FC01E752FD4F1082FC01EA54FD4F208306
:101CA000FC01EE57FD4F1082FC01ED56FD4F2083E5
:101CB00001968131910541F780912F36809330361E
:101CC000809148028370823009F0B8C080B190E002
:101CD00095958795817080932536909125368091D2
:101CE0007001981709F474C080917001882311F075
:101CF0002C9A01C02C9880912536882309F065C064
:101D000080911B3690911C36A0911D36B0911E36E5
:101D1000209121363091223640912336509124363D
:101D2000821B930BA40BB50B809368019093690100
:101D3000A0936A01B0936B01809168019091690151
:101D4000A0916A01B0916B01885E9340A040B040C1
:101D500080F48091680190916901A0916A01B0912D
:101D60006B0180936C0190936D01A0936E01B09311
:101D70006F0121E02093263680911B3690911C360E
:101D8000A0911D36B0911E36809321369093223655
:101D9000A0932336B09324368091AB028823C1F4FC
:101DA000209327362093710180916C0190916D01F1
:101DB000A0916E01B0916F018093680190936901C9
:101DC000A0936A01B0936B0103C081E08093293630
:101DD000809125368093700180916801909169010E
:101DE000A0916A01B0916B01885E9340A040B04021
:101DF00060F088EE93E0A0E0B0E0809368019093FB
:101E00006901A0936A01B0936B0180916801909180
:101E10006901A0916A01B0916B01893C9105A1050E
:101E2000B10560F488EC90E0A0E0B0E08093680138
:101E300090936901A0936A01B0936B01FF91EF91B8
:101E4000BF91AF919F918F915F914F913F912F9152
:101E50000F900BBE0F900FBE0F901F901895E82F9C
:101E6000592F4091F6353091F7352091973722233D
:101E700081F0213051F48DB3809399379DB38091D7
:101E80009837809589238DBB04C08FB7F8948093D1
:101E900099374CBD3DBD5D985EBD00000DB407FE99
:101EA000FDCF8EB5EEBD00000DB407FEFDCF8EB5A3
:101EB0007EBD00000DB407FEFDCF8EB56EBD0000E7
:101EC0000DB407FEFDCF8EB55D9A222339F08091C7
:101ED0009937213011F48DBB01C08FBF5093583614
:101EE000E093573670935636609355360895682FB1
:101EF000592F4091F6353091F735209197372223AD
:101F000081F0213051F48DB3809399379DB3809146
:101F10009837809589238DBB04C08FB7F894809340
:101F200099374CBD3DBD5C985EBD00000DB407FE09
:101F3000FDCF8EB56EBD00000DB407FEFDCF8EB592
:101F40005C9A222339F080919937213011F48DBBAE
:101F500001C08FBF5093543660935336089540911B
:101F6000F6353091F73520919737222381F02130D3
:101F700051F48DB3809399379DB3809198378095B4
:101F800089238DBB04C08FB7F894809399374CBDDB
:101F90003DBD5C981EBC00000DB407FEFDCF8EB5A4
:101FA0001EBC00000DB407FEFDCF8EB55C9A222347
:101FB00039F080919937213011F48DBB08958FBF8E
:101FC00008959C013F7030616091F6355091F7356E
:101FD00040919737442381F0413051F48DB3809381
:101FE00099379DB380919837809589238DBB04C024
:101FF0008FB7F894809399376CBD5DBD12983EBD44
:1020000000000DB407FEFDCF8EB52EBD00000DB44F
:1020100007FEFDCF8EB5129A442339F0809199378F
:10202000413011F48DBB08958FBF08958F3708F0AC
:102030008FE7282F30E0F5E0220F331FFA95E1F704
:102040003F7030696091F6355091F7354091973780
:10205000442381F0413051F48DB3809399379DB37F
:1020600080919837809589238DBB04C08FB7F894F1
:10207000809399376CBD5DBD12983EBD00000DB4D4
:1020800007FEFDCF8EB52EBD00000DB407FEFDCFBF
:102090008EB5129A442339F080919937413011F46A
:1020A0008DBB08958FBF08959C013F703061609192
:1020B000F6355091F73540919737442381F0413000
:1020C00051F48DB3809399379DB380919837809563
:1020D00089238DBB04C08FB7F894809399376CBD6A
:1020E0005DBD13983EBD00000DB407FEFDCF8EB55B
:1020F0002EBD00000DB407FEFDCF8EB5139A44230C
:1021000039F080919937413011F48DBB08958FBF1C
:1021100008959C013F7030696091F6355091F73514
:1021200040919737442381F0413051F48DB380932F
:1021300099379DB380919837809589238DBB04C0D2
:102140008FB7F894809399376CBD5DBD13983EBDF1
:1021500000000DB407FEFDCF8EB52EBD00000DB4FE
:1021600007FEFDCF8EB5139A442339F0809199373D
:10217000413011F48DBB08958FBF08954091F6351D
:102180003091F73520919737222381F0213051F497
:102190008DB3809399379DB380919837809589232B
:1021A0008DBB04C08FB7F894809399374CBD3DBD6B
:1021B0005E9A1EBC00000DB407FEFDCF8EB51EBC9E
:1021C00000000DB407FEFDCF8EB5809308361EBC0F
:1021D00000000DB407FEFDCF8EB51EBC00000DB48F
:1021E00007FEFDCF8EB51EBC00000DB407FEFDCF6F
:1021F0008EB580930636809307365E98222339F099
:1022000080919937213011F48DBB08958FBF0895C7
:102210009C0143B148704093F83593B1947090930A
:10222000F935442311F58091FA358823F1F099238B
:1022300019F0260F371F19C08091893682FF10C010
:102240008091EF01813041F0813010F0823069F4EB
:102250002A30310554F007C02031310534F003C075
:102260002115310511F0261B370B4093FA35C901B2
:102270000895482F53B152705093FE3593B1917029
:102280009093FF355523D9F4809100368823B9F017
:10229000992369F08FEF90E0841B9109262F30E09D
:1022A0008217930714F44FEF0AC0460F08C0461771
:1022B00020F4442321F0462F02C04111461B5093C5
:1022C0000036842F90E00895CF92DF92EF92FF9234
:1022D0000F931F93CF93DF93EC01F42EE22E68014E
:1022E000188110933737812F0E9439118883F8168F
:1022F00008F0F88288818E1508F0E88288818117BD
:1023000039F08093373781E0F601808380932C0188
:10231000DF91CF911F910F91FF90EF90DF90CF90C1
:1023200008950F931F93DF93CF930F92CDB7DEB72E
:1023300089838091352B90E025E23DE0829FF0017A
:10234000839FF00D929FF00D1124E05EFF4E2081DF
:10235000203311F0203609F428E12150CE010196F6
:1023600061E040E009EB13E00E9464116981609331
:10237000EB028091913683FF26C08091352B90E04F
:1023800040E050E025E23DE0829FD001839FB00D08
:10239000929FB00D1124962F9F71990FFA01EE0FA5
:1023A000FF1FE40FF51FEA0FFB1FEB5DFF4E80815F
:1023B000817C892B80834F5F5F4F4034510571F7DB
:1023C00081E08093B903862F0F90CF91DF911F9109
:1023D0000F9108951F93FC0113B112701093FE35F5
:1023E00093B191709093FF35112361F58091003680
:1023F000882341F19923D1F0CF01A0E0B0E02FEF85
:102400003FEF40E050E0281B390B4A0B5B0B862F57
:1024100090E0A0E0B0E0281739074A075B071CF4FA
:10242000EFEFFFEF0FC0E60FF11D0CC070E0E617F5
:10243000F70720F4309731F0FB0104C0309711F01A
:10244000E61BF70B10930036CF011F910895AF9252
:10245000BF92CF92DF92EF92FF920F931F93CF9391
:10246000DF93EC01F42EE52EB22EA32E6801088135
:1024700019811093343700933337C8010E94EA1151
:102480009C01998388838F2D9E2D8217930710F0CE
:10249000998388832B2D3A2D888199818217930700
:1024A00010F039832883888199818017910749F03A
:1024B000909334378093333781E0F60180838093A3
:1024C0002C01DF91CF911F910F91FF90EF90DF9042
:1024D000CF90BF90AF9008959C0143B1427040935C
:1024E000FE3593B191709093FF35442309F58091A7
:1024F00000368823E9F070E0992369F08FEF9FE7B9
:10250000821B930B861797071CF42FEF3FE710C031
:10251000260F371F0DC0261737072CF4211531055C
:1025200039F09B0105C02115310511F0261B370B31
:1025300040930036C9010895AF92BF92CF92DF92C7
:10254000EF92FF920F931F93CF93DF93EC017A01E9
:102550006901580108811981109336370093353786
:10256000C8010E946C1299838883E816F90614F05A
:10257000F982E882888199818C159D0514F0D982B1
:10258000C882888199818017910749F090933637E6
:102590008093353781E0F501808380932C01DF91B2
:1025A000CF911F910F91FF90EF90DF90CF90BF9050
:1025B000AF9008959F92AF92BF92CF92DF92EF9229
:1025C000FF920F931F937B018C0159016A0193B015
:1025D00082E098229092FE3593B191709093FF35EE
:1025E0009920D9F5809100368823B9F1992329F0F3
:1025F000C801B7010E94158B2EC08091893682FFD9
:102600001AC08091EF01813059F0813010F0823092
:1026100021F5C801B70120E030E040E251E406C0F6
:10262000C801B70120E030E040E851E40E94C88CC6
:1026300088239CF00AC0C801B70120E030E040E0E8
:1026400050E00E94798B882341F0C801B701A601B0
:1026500095010E94148B7B018C0190920036B7018A
:10266000C8011F910F91FF90EF90DF90CF90BF9026
:10267000AF909F900895BF92CF92DF92EF92FF921A
:102680000F931F93CF93DF93742F2091352B8031BD
:1026900009F04EC030E0A0E0B0E085E29DE0289F68
:1026A0007001299FF00C389FF00C1124062F10E0C8
:1026B000C42FD0E0D42ED294DD0CDD0C30ECD3222C
:1026C000469546954770562F5295550F550F507C9D
:1026D000669566956770FD01EE0FFF1FEA0FFB1F01
:1026E000EE0DFF1DEB5DFF4E2081922F929596958A
:1026F000969593703181832F8770880F880F892B6F
:1027000090E08017910734F42F73252B2083387FB6
:10271000362B08C08C179D0734F02F732D2920838A
:10272000387F342B31831196A034B105A1F65CC0FB
:10273000422F50E0A0E0B0E0282F30E084EC90E0A1
:10274000289F6001299FD00C389FD00C112485E26E
:102750009DE0489F7001499FF00C589FF00C112498
:10276000062F10E0C72FD0E0B72EB294BB0CBB0CE5
:1027700090ECB922472F469546954770562F5295B3
:10278000550F550F507C669566956770FD01EE0FED
:10279000FF1FEA0FFB1FEC0DFD1DEE0DFF1DE452A8
:1027A000FC4F2081922F929596959695937031814A
:1027B000832F8770880F880F892B90E080179107EF
:1027C00034F42F73252B2083387F362B08C08C17C9
:1027D0009D0734F02F732B292083387F342B3183CE
:1027E0001196A034B10591F6DF91CF911F910F9111
:1027F000FF90EF90DF90CF90BF9008952F923F927F
:102800004F925F926F927F928F929F92AF92BF9200
:10281000CF92DF92EF92FF920F931F93DF93CF93AC
:10282000CDB7DEB760970FB6F894DEBF0FBECDBF51
:10283000DE011196ECEAF1E080E101900D92815009
:10284000E1F78091352B482F50E085E29DE0489FCD
:10285000F001499FF00D589FF00D1124E05EFF4EEE
:10286000D0808091973683FF0DC080915E018F5F8D
:1028700080935E01883018F087E080935E0181E0EC
:1028800080932C018091953683FF0CC080915E016E
:10289000815080935E01883010F010925E0181E0DB
:1028A00080932C0185E29DE0489FF001499FF00D47
:1028B000589FF00D1124E15EFF4EE081E33018F4E3
:1028C000E13048F405C0E33049F0E93048F403C092
:1028D000FCE07F2E05C0E7E07E2E02C075E0772E7B
:1028E0008091AB02882309F44AC08091B002813004
:1028F00009F045C08091B703882309F440C0809156
:10290000810290E0FC01EE0FFF1FE80FF91F85E246
:102910009DE0489F9001499F300D589F300D112434
:10292000E20FF31FE95DFF4E909131379F70808178
:10293000807F892B80838091810290E0FC01EE0FE3
:10294000FF1FE80FF91FE20FF31FE95DFF4E9091A3
:102950005F0197709295907F80818F78892B80831B
:102960008091810290E0FC01EE0FFF1FE80FF91F3C
:10297000E20FF31FEB5DFF4E80818E7F8083C0905E
:10298000323700913137EE24FF24472C552425E2BD
:10299000822E2DE0922E91E0292E312C87E0682E98
:1029A000F701EE0FFF1FE959F94C30818091B236E3
:1029B0009091B3360E2C02C0969587950A94E2F753
:1029C000282F2170367F932F922B9083892F869505
:1029D0008170281709F404C192FDF6C0213009F076
:1029E000F3C039603083E1E0F0E0EC0FFD1FEE0D45
:1029F000FF1DE0818E2F90E0672D70E00E945A8DC0
:102A00009B0180915E01860F80935F01883010F0FA
:102A100060925F01249DC001259D900D349D900D15
:102A200011242E2F281B8091352B90E0889DF001DA
:102A3000899DF00D989DF00D1124E15EFF4E80817F
:102A4000833018F4813068F405C0833081F0893018
:102A500098F407C0E22FF0E0E355FC4FC490CA940D
:102A60000BC0E22FF0E0E15AF54FC49005C0E22F11
:102A7000F0E0EA59F54FC4904CE0849FF001112436
:102A8000EC0DF11DE355FC4F049101508091F5359B
:102A9000882349F0080F0C3030F080915F018F5F80
:102AA00080935F010C50E02FF0E0EE0FFF1FE75E18
:102AB000FB4F8591949120915F01B22EBB0CAA240B
:102AC0008A0D9B1D0E94E10F5F9A51E05093B7035E
:102AD0008091AB02882309F477C08091B0028130E5
:102AE00009F072C08091352B482F50E08091700220
:102AF00090E0FC01EE0FFF1FE80FF91F489D9001C9
:102B0000499D300D589D300D1124E20FF31FE95DF2
:102B1000FF4E902F9F708081807F892B80838091D2
:102B2000700290E0FC01EE0FFF1FE80FF91FE20FAB
:102B3000F31FE95DFF4E90915F0197709295907F32
:102B400080818F78892B808388E1D816B9F08D1524
:102B500038F09CE0D91671F0E0E1DE1691F40CC07B
:102B6000F0E3DF1659F080E6D81651F090E2D9165E
:102B700041F406C01BE005C01FE003C017E101C01F
:102B80001FE18091810290E0FC01EE0FFF1FE80F32
:102B9000F91F489DC001499D900D589D900D11242D
:102BA000E80FF91FEB5DFF4E912F9F71990F808108
:102BB000817C892B8083E0918102F0E0EE0FFF1F82
:102BC000E059FC4C31822082F701EE0FFF1FE959DA
:102BD000F94C8081982F9170990F8D7F892B80837C
:102BE0000894E11CF11CE0E1EE16F10409F0D8CEE6
:102BF000C0923237009331378091B2369091B3361C
:102C0000892B09F071C08091B703882309F46CC047
:102C10005F981092B7038091AB02882309F464C0D7
:102C20008091B002813009F05FC0F8E1DF16D9F081
:102C3000FD1538F04CE0D41671F050E1D51651F581
:102C40000EC080E3D816D1F090E6D916F9F0E0E294
:102C5000DE1601F50FC080914E026CE007C01091A6
:102C60004E021F7017C080914E0268E10E944E8D87
:102C7000192F10C010914E021F710CC080914E028E
:102C800060E30E944E8D192F169504C010914E02DC
:102C9000169516958091810290E02091352B30E0B9
:102CA000FC01EE0FFF1FE80FF91F85E29DE0AC016C
:102CB000249FC001259F900D349F900D1124E80F93
:102CC000F91FEB5DFF4E1F71110F8081817C812BFD
:102CD0008083E0918102F0E0EE0FFF1FE059FC4C91
:102CE00081E090E091838083809170028823A9F530
:102CF0002091352B30E05091B90340E085E29DE012
:102D0000289FB001299F700D389F700D11248B01F1
:102D10000F5D1F4E1CC0242F30E0D901AA0FBB1F2E
:102D2000A059BC4C8D919C911197892B79F0F90198
:102D3000EE0FFF1FE20FF31FE60FF71FEB5DFF4ED5
:102D40008081816080831D921C9251E04F5FF80169
:102D50008081481700F35093B90360960FB6F8943A
:102D6000DEBF0FBECDBFCF91DF911F910F91FF90BE
:102D7000EF90DF90CF90BF90AF909F908F907F901B
:102D80006F905F904F903F902F900895CF93DF9377
:102D9000C82FD0E060913E0270913F0280E090E049
:102DA0000E94168CCC54D94CEC89F0E0EE0FFF1F3A
:102DB000EE0FFF1FE557FE4F208131814281538185
:102DC0000E94CC8C9B01AC0160E070E080E792E453
:102DD0000E947D8B21E338E04CEA5CE30E947D8B0E
:102DE0000E94EA8BCB016F3F710510F08EEF90E0EF
:102DF00081958A83DF91CF9108953F924F925F92A0
:102E00006F927F928F929F92AF92BF92CF92DF92FA
:102E1000EF92FF920F931F93CF93DF93909087369B
:102E200096949694AA24A3949A20992D990F809110
:102E300047368C7FD0908936D694D694DA20892B69
:102E40008D29A0909F36A694A694BB24B394AB2062
:102E50002A2D220F220F837FB090A136B694B6940C
:102E6000CC24C394BC209B2D990F990F990F822BD2
:102E7000892B40918D36469546954170342F329579
:102E8000307F8F7C20919536269526952170922F44
:102E90009295990F907E832B892B909197369695DA
:102EA00096959170392F3295330F330F307C8F7B8D
:102EB000832B80934736022F10E0000F111F000F65
:102EC000111F692F70E093E0660F771F9A95E1F765
:102ED000C42FD0E085E0CC0FDD1F8A95E1F720916B
:102EE0004636922F96959270902B822F82958695DA
:102EF0008170982B962B269526952071292B2C2BAB
:102F000020933F36E0904602F090470221E0E2161F
:102F1000F10419F45091790109C0E114F10411F49C
:102F200051E005C050919136569556955170852FB8
:102F300081708295880F807E909146369F7D982B78
:102F400090934636C7010397029720F04CE0E416B1
:102F5000F10429F4C090790181E0C82207C0CC2493
:102F600092E0E916F10411F4CC24C3949C2D990F3E
:102F7000990F809146368B7F892B8093463624E0CB
:102F8000E216F10421F04CE0E416F10421F4309152
:102F90007901317007C03091A7363695369531707A
:102FA00009F031E0932F9170990F990F990F80914B
:102FB0004636877EB091A536B695B695B1702B2F63
:102FC0002295207F892B822B809346368091B002F8
:102FD000882359F0809148368160809348369091DB
:102FE00048369170EBE3FBE220C08091382B8823B8
:102FF00081F480913702882361F48091B90388239A
:1030000041F48091E336882321F48091F1358823BF
:1030100041F0909179019170809148368E7F892B93
:10302000DCCF809148368E7FD8CF8081882319F0FD
:1030300090917901917031968BE2EB34F807A9F702
:10304000809148368E7F892B8093483695E0E9162B
:10305000F10421F480914636806403C080914636A5
:103060008F7B80934636E091F033F091F133F0930B
:103070004D36E0934C3628E0E216F104D9F4809105
:10308000F101823099F48091EF018250823070F426
:1030900081E090E00090B40202C0880F991F0A946A
:1030A000E2F790933A368093393604C010923A365C
:1030B000109239364091AB02A0E0442309F4A1E01C
:1030C000809146368E7F8A2B80934636442321F0AA
:1030D00080914736806809C090917901979599272A
:1030E0009795809147368F77892B80934736602B51
:1030F000712B6C2B7D2B809146368295869586951B
:10310000817090E014E0880F991F1A95E1F7682B01
:10311000792B8B2D90E026E0880F991F2A95E1F7F7
:10312000682B792B8B2F90E09695982F8827979571
:103130008795682B792B9A2D80E0682B792B992D18
:10314000990F990F80E0682B792B9D2D990F990F7E
:10315000990F80E0682B792B20914736221F222778
:10316000221F922F9295907F80E0682B792B2091DF
:1031700048362170922F9295990F990F907C80E09C
:10318000682B792B9A2F9295990F907E80E0682B6F
:10319000792B852F90E0682B792B8C2D90E0880F70
:1031A000991F682B792B932F990F80E0682B792B2F
:1031B00070934136609340363090B102C32DD0E019
:1031C00021E030E0C901032C02C0880F991F0A9446
:1031D000E2F790934A368093493655E0E516F104BC
:1031E00009F465C266E0E616F104B4F472E0E7168D
:1031F000F10461F143E0E416F1041CF4F7FE4BC264
:1032000076C253E0E516F10409F4EAC064E0E6167C
:10321000F10409F06CC214C27CE0E716F10409F471
:103220000FC22DE0E216F1045CF447E0E416F1046D
:1032300009F4D6C059E0E516F10409F058C2D0C02F
:103240006FE0E616F1040CF052C2CAC080919136CC
:1032500082FF08C00090B20202C0220F331F0A94FE
:10326000E2F720C2442309F46CC09091312B9923DA
:1032700009F44BC08091322B482F50E04F705070B2
:1032800060E070E020E030E0E92FF0E0B1E0EB2E0C
:10329000F12C012D112D10C0C901840F951F57016C
:1032A000680104C0AA0CBB1CCC1CDD1C8A95D2F79B
:1032B0006A297B292F5F3F4FE217F3076CF7809154
:1032C0007901FE01E658FE4FE081C15BDD4F2881A8
:1032D00040E050E0882311F441E050E08091B502D5
:1032E0008F7002C0440F551F8A95E2F740955095A4
:1032F000642375238E2F90E02F7002C0880F991FD2
:103300002A95E2F7682779275AC040917901FE0192
:10331000E658FE4F8081C15BDD4F288190E02F7021
:1033200002C0880F991F2A95E2F750E02091B5025C
:103330002F7002C0440F551F2A95E2F78427952766
:10334000D2C19091312B992309F43EC08091322B48
:10335000482F50E04F70507060E070E020E030E0A7
:10336000E92FF0E0A1E0EA2EF12C012D112D10C083
:10337000C901840F951F5701680104C0AA0CBB1C2A
:10338000CC1CDD1C8A95D2F76A297B292F5F3F4F21
:10339000E217F3076CF78091790120E030E0882391
:1033A00011F421E030E08091B5028F7002C0220F4D
:1033B000331F8A95E2F7209530956223732370932B
:1033C0003A366093393693C18091790190E020912B
:1033D000B5022F7002C0880F991F2A95E2F783C1AA
:1033E000DD2009F080C1FE01E25BF44D9080892C64
:1033F000829440EF84222091352B30E040E050E071
:1034000000E010E060E070E084EC90E0C89F2001F4
:10341000C99F500CD89F500C112485E29DE0289F35
:103420003001299F700C389F700C112431E0A32EBD
:10343000B12CC12CD12C882D840F90E020E13216C4
:1034400069F4FC01EE0FFF1FE80FF91FE60DF71DF1
:10345000EB5DFF4E808180FF3FC012C0FC01EE0F8C
:10346000FF1FE80FF91FE40DF51DE60DF71DE452EF
:10347000FC4F8081982F917081FF0FC09923E1F05C
:10348000D601C501042E04C0880F991FAA1FBB1FB7
:103490000A94D2F7682B792B1FC0992369F0D601C3
:1034A000C501042E04C0880F991FAA1FBB1F0A94D0
:1034B000D2F7082B192B10C0D601C501042E04C069
:1034C000880F991FAA1FBB1F0A94D2F78095909569
:1034D00068237923082319234F5F5F4F4034510538
:1034E00009F0A9CF00933D3610933E3660933B36EA
:1034F00070933C36FE01E15AF44D30819316B1F4DD
:10350000FE01E658FE4F8081FE01E15BFD4F208108
:1035100090E02F7002C0880F991F2A95E2F7862746
:10352000972790933A368093393604C070933A3691
:103530006093393680914B36883C08F19316B9F484
:10354000FE01E658FE4F8081C15BDD4F288190E08F
:103550002F7002C0880F991F2A95E2F780279127C4
:10356000862B972B90933A368093393606C0062BDC
:10357000172B10933A360093393610924B3647E0AA
:10358000E416F10429F059E0E516F10409F0AFC0A2
:103590009920A1F480914C02803108F0A8C02091BC
:1035A000790130E002C0220F331F8A95E2F7809143
:1035B000393690913A368227932795C061E0961666
:1035C00079F420914C02203208F091C0203108F4A7
:1035D0008EC08091790190E030E02051304024C0CD
:1035E00072E0971679F420914C02203308F07FC0E6
:1035F000203208F47CC08091790190E030E02052C4
:10360000304012C083E0981609F071C020914C023E
:10361000203408F06CC0203308F469C0809179012F
:1036200090E030E02053304002C0880F991F2A9567
:10363000E2F72091393630913A362827392732C0BF
:10364000809148028370B9F081E060E070E00E94F0
:1036500080082091A8023091A9024091433650E0A1
:1036600059014A9D90014B9D300D5A9D300D1124FA
:10367000282B392B17C0009144361091453681E034
:1036800060E070E00E948008082B192B10933A36F6
:10369000009339362CC00090F53302C0220F331F3F
:1036A0000A94E2F730933A362093393620C080915D
:1036B0008F3682FF12C08091790190E02091F23321
:1036C0003091F3336C01C29EC001C39E900DD29E17
:1036D000900D11248E279F2706C08091443690912B
:1036E00045368E2B9F2B90933A36809339366091D6
:1036F0004036709141368091393690913A364091FA
:103700003F360E942F0FDF91CF911F910F91FF90B5
:10371000EF90DF90CF90BF90AF909F908F907F9071
:103720006F905F904F903F900895A7EEB6E3E7EF5C
:10373000F6E390E928E48C918823B9F08081883100
:10374000A0F08091C80085FFFCCF9093CE008091BF
:10375000C80085FFFCCF2093CE008091C80085FF74
:10376000FCCF1092CE001C921082119631969F5F72
:10377000903A09F70895EF92FF920F931F93CF931A
:10378000DF930091B10250E02091352BC62FD0E09D
:10379000003109F073C030E0DA01AA0FBB1FA40F9B
:1037A000B51F85E29DE0AC01249FC001259F900DCF
:1037B000349F900D1124A80FB91FBD016B5D7F4E82
:1037C000FE01EE0FFF1FEC0FFD1FE80FF91F8F0129
:1037D0000B5D1F4EE80198819170EB0188818E7F0F
:1037E000892B8883AD01495D5F4E9F01295D3F4E66
:1037F000E90198819F70EA018881807F892B888305
:10380000E901988190778F78892BEA018883E90113
:10381000988190788F77892BEA018883E8019881D5
:103820009E73EB018881817C892B8883AA5DBF4EC2
:10383000EA5DFF4E9081987F8C918770892B8C93E5
:10384000F801808182958695869583709181977025
:10385000990F990F982B292F2295220F220F207C48
:1038600088818F73822B8883969596958981887F2E
:10387000892B898381E08093B90375C010E030E023
:10388000E82EFF24DA01AA0FBB1FA40FB51F64ECBA
:1038900070E0069FC001079F900D169F900D1124A8
:1038A000A80FB91F85E29DE0A901489F9001499F9B
:1038B000300D589F300D1124A20FB31FAD0144529B
:1038C0005C4FFE01EE0FFF1FEC0FFD1FE69EC001D7
:1038D000E79E900DF69E900D1124E80FF91FE20F60
:1038E000F31FBF0164527C4FEB0198819170EA0194
:1038F00088818E7F892B8883EB01988192708D7FE0
:10390000892BEA018883EB0198819C73837C892B46
:10391000EA018883EB01288122952695269523705C
:1039200099819770990F990F922B292F2295220F29
:10393000220F207C8F73822BEA01888396959695BF
:103940008981887F892B8983A352BC4FE352FC4F26
:103950009081987F8C918770892B8C93055C144D96
:1039600081E0F8018083DF91CF911F910F91FF904B
:10397000EF900895DF92EF92FF920F931F93CF93F2
:10398000DF932091352B803109F471C0422F50E034
:10399000282F30E084EC90E0289FB001299F700D23
:1039A000389F700D112485E29DE0DA01A89FA001E7
:1039B000A99F500DB89F500D1124DB01A40FB51F16
:1039C000AE53BC4FA652BF4F0D91FB01E45FF14EC9
:1039D000E652FF4F01938C918083329612968C9120
:1039E00080838E918293FA01EE53FC4FE20FF31F16
:1039F0008781245F314EF901878310E07B01EA0162
:103A0000812F90E0FC01EE0FFF1FE80FF91FEE0D74
:103A1000FF1DBF016A5D714E9F012C0F3D1FD90133
:103A2000A452BC4F9C91492F4295469546954370B0
:103A300011968C918770880F880F842B482F4295A0
:103A4000440F440F407C9F73942BDB019C9386951D
:103A50008695E95DF14E23523C4FD9019C91987FA8
:103A60008770892B80831F5F011750F679C030E083
:103A700085E29DE0F901E89F9001E99F300DF89FF4
:103A8000300D1124F901EE53FC4FE15AF34FD08071
:103A9000D0926B2A829180936A2A32968191809388
:103AA0006C2A808180936D2A349780818093692A63
:103AB00000E0E901802F90E0DC01AA0FBB1FA80FF6
:103AC000B91F9D012159354DBD016C0F7D1FE5E2E8
:103AD000EE2EE0E1FE2EE60EF71EF7011081912F8B
:103AE0009170F90180818E7F892B8083AD014F58C1
:103AF000554DFB01E95DFF4E8081FA018083912FD6
:103B00009E73F9018081817C892B8083A059B54DFA
:103B10006A5D7F4EFB019081987F8C918770892B25
:103B20008C931295169516951370D70111969C914A
:103B30009770990F990F912B492F4295440F440F7D
:103B4000407CF90180818F73842B808396959695B4
:103B50008181887F892B81830F5FD01608F0AACFDF
:103B6000DF91CF911F910F91FF90EF90DF9008951B
:103B70009F92AF92BF92CF92DF92EF92FF920F93FC
:103B80001F93CF93DF932091352B803109F481C0AF
:103B9000422F50E0C82FD0E0262F30E084EC90E098
:103BA000289F7001299FF00C389FF00C1124D70139
:103BB000A45FB14EA652BF4F9D90C89FB001C99F50
:103BC000700DD89F700D112485E29DE0FA01E89FE9
:103BD000A001E99F500DF89F500D1124FB01E40F47
:103BE000F51FEE53FC4FE652FF4F91928C9180836C
:103BF000329612968C9180838E918293FA01EE53C5
:103C0000FC4FEC0FFD1F245F314ED90117968C91AC
:103C1000878300E05B016A01802F90E0FC01EE0FDA
:103C2000FF1FE80FF91F9F012A0D3B1D2C0D3D1DA5
:103C3000B90164527C4FEE0DFF1DDF01AA5DB14E4C
:103C40009C91492F429546954695437011968C91CB
:103C50008770880F880F842B482F4295440F440F9C
:103C6000407C9F73942BDB019C9386958695235211
:103C70003C4FE95DF14E9081987F8770892BF90167
:103C800080830F5F901640F6C55CD44D81E0888339
:103C90007EC030E0D0906B2A85E29DE0A901489F6C
:103CA0009001499F300D589F300D1124F901EE53BA
:103CB000FC4FE15AF34FD08280916A2A8293329668
:103CC00080916C2A819380916D2A808334978091B2
:103CD000692A808300E0E901802F90E0DC01AA0FCF
:103CE000BB1FA80FB91FBD016C0F7D1F9B012B5D72
:103CF0003F4E1FE6E12E1AE2F12EEA0EFB1EF701FF
:103D00001081912F9170F90180818E7F892B8083A2
:103D1000AB01495D5F4EFD01EF58F54D8081FA0121
:103D20008083912F9E73F9018081817C892B808310
:103D30006A5D7F4EA059B54D9C91987FDB018C91B7
:103D40008770892B8C931295169516951370F70131
:103D500091819770990F990F912B492F4295440F9C
:103D6000440F407CD9018C918F73842B8C93969552
:103D7000969511968C911197887F892B11968C932B
:103D80000F5FD01608F0A8CF81E08093B90381E0DF
:103D900080932C01DF91CF911F910F91FF90EF90B5
:103DA000DF90CF90BF90AF909F900895CF93DF9317
:103DB0002091352B30E0C82FD0E084EC90E0C89FF4
:103DC000A001C99F500DD89F500D112485E29DE0A0
:103DD000B901689F9001699F300D789F300D1124C3
:103DE000FA01E20FF31FEE53FC4FE652FF4F8FE054
:103DF000819388E18083329681E08083129260E033
:103E000070E0FB01EE0FFF1FE60FF71FE40FF51F39
:103E1000E20FF31FDF01A452BC4F82E08C93E35208
:103E2000FC4F84E080836F5F7F4F6034710549F7FA
:103E3000C55CD44D81E0888380932C01DF91CF91C4
:103E40000895CF93DF938091352B90E025E23DE0FC
:103E5000A901849F9001859F300D949F300D1124FE
:103E6000F901EE53FC4FE15AF34F8FE0808388E174
:103E70008293329681E0819310823497108240E0E1
:103E800050E0B901FA01EE0FFF1FE40FF51FE60F36
:103E9000F71FDF01AB5DBF4E8C918E7F8C93CF01FE
:103EA000895D9F4E20E3EC0128838C91817C8861A1
:103EB0008C93EA5DFF4E8081877080838C918F7335
:103EC0008C9311968C911197887F846011968C93B6
:103ED0004F5F5F4F40345105A9F681E08093B903ED
:103EE00080932C01DF91CF9108951F9310E0812FD3
:103EF0000E94BA1C1F5F1131D1F78091B4368093B4
:103F0000CB368091B6368093CD368091B83690917D
:103F1000B936A091BA36B091BB368093CF36909324
:103F2000D036A093D136B093D2368091C6368093E6
:103F3000DD368091C8368093DF368091B536809328
:103F4000CC368091B7368093CE368091BC36909136
:103F5000BD36A091BE36B091BF368093D3369093D4
:103F6000D436A093D536B093D6368091C736809399
:103F7000DE368091C9368093E0361F9108951F93F5
:103F800010E0812F612F0E94B81D1F5F1131C9F70A
:103F90008091CB368093B4368091CD368093B636FF
:103FA0008091CF369091D036A091D136B091D23653
:103FB0008093B8369093B936A093BA36B093BB3697
:103FC0008091DD368093C6368091DF368093C83687
:103FD0008091CC368093B5368091CE368093B736BB
:103FE0008091D3369091D436A091D536B091D63603
:103FF0008093BC369093BD36A093BE36B093BF3647
:104000008091DE368093C7368091E0368093C93642
:1040100081E08093E3361F9108951F9310E0812F74
:104020000E94D61E1F5F1031D1F70E94211F1F91E1
:1040300008958F929F92BF92CF92DF92EF92FF925C
:104040000F931F93CF93DF93382FB42E2091352BEE
:10405000803161F430E0F62E85E29DE0289F60011A
:10406000299FD00C389FD00C1124E5C0822F90E0FE
:10407000062F832E992424EC30E0829E6001839EDB
:10408000D00C929ED00C112425E23DE0829F70015D
:10409000839FF00C929FF00C112458C0202F30E029
:1040A000802F8F7090E0D901AA0FBB1FA20FB31F02
:1040B000AC0DBD1DAE0DBF1DAD0144525C4FFC01EA
:1040C000EE0FFF1FE80FF91FEC0DFD1DEE0DFF1D9C
:1040D000BF0164527C4FEB0198819170EA018881A5
:1040E0008E7F892B8883EB01988192708D7F892B3D
:1040F000EA018883EB0198819C73837C892BEA0118
:104100008883EB0128812295269526952370998135
:104110009770990F990F922B292F2295220F220F1A
:10412000207C8F73822BEA018883969596958981EE
:10413000887F892B8983A352BC4FE352FC4F908127
:10414000987F8C918770892B8C930F5FB01608F045
:10415000A5CFEBE3FBE28E0E9F1E81E0E401888396
:1041600070C02F2D30E08F2D8F7090E0D901AA0FF5
:10417000BB1FA20FB31FAC0DBD1DBD016B5D7F4EFC
:10418000FC01EE0FFF1FE80FF91FEC0DFD1D8F0165
:104190000B5D1F4EE80198819170EB0188818E7F45
:1041A000892B8883AD01495D5F4E9F01295D3F4E9C
:1041B000E90198819F70EA018881807F892B88833B
:1041C000E901988190778F78892BEA018883E9014A
:1041D000988190788F77892BEA018883E80198810C
:1041E0009E73EB018881817C892B8883AA5DBF4EF9
:1041F000EA5DFF4E9081987F8C918770892B8C931C
:10420000F80180818295869586958370918197705B
:10421000990F990F982B292F2295220F220F207C7E
:1042200088818F73822B8883969596958981887F64
:10423000892B8983F394BF1408F093CF81E0809396
:10424000B90381E080932C01DF91CF911F910F91F1
:10425000FF90EF90DF90CF90BF909F908F90089548
:104260002F923F925F926F927F928F929F92AF9226
:10427000BF92CF92DF92EF92FF920F931F93CF9353
:10428000DF932091352B803109F0EFC0822E9924E5
:1042900085E29DE0889E9001899E300D989E300DAC
:1042A0001124F901EF5DFF4E7080D901AB5DBF4E67
:1042B0009C91662463946922F901E95DFF4E808137
:1042C000EFE05E2E5822E82EE2947FE0E72247E0FE
:1042D000E422A82EAA1CAA24AA1CD92ED6948FE1C7
:1042E000D822F901EA5DFF4EB080B694B694B69438
:1042F00092959695969593701196FC90F422FF0CEA
:10430000FF0CF92ACC24C394190166C02C2D30E08F
:10431000C9010197AC01440F551F480F591F420DA9
:10432000531DBA016B5D7F4ED901AA0FBB1FA20FAF
:10433000B31FA20DB31D8D010B5D1F4EE8019881C7
:104340009170FB0180818E7F892B80839A01295D8A
:104350003F4EFD01E95DFF4E90819F70E90188812C
:10436000807F892B8883908190778F78892B8883B1
:10437000908190788F77892B8883F801808182954E
:1043800086958695837091819770990F990F982BD8
:10439000292F2295220F220F207CEB0188818F7319
:1043A000822B8883969596958981887F892B89832E
:1043B0004A5D5F4EAA5DBF4E9C91987FFA01808155
:1043C0008770892B8083E80198819E73FB0180812F
:1043D000817C892B8083C3947C1408F097CF872D30
:1043E00090E0FC01EE0FFF1FE80FF91F85E29DE052
:1043F0009C01829EC001839E900D929E900D11247F
:10440000E80FF91FDF01AB5DBF4E8C918E7F8629CF
:104410008C93CF01895D9F4E37E0E322E29410EF49
:10442000E122A794AA24A794E528EA28EC01E882CF
:104430009F2D9295990F990F907C8C918F73892B5A
:104440008C93EA5DFF4EBB0CBB0CBB0CF694F69450
:10445000FB28F082EFE1DE22DD0C8C91817C8D293E
:104460008C9381E08093B903DCC0622E7724282EE0
:10447000332484EC90E0289EA001299E500D389EA4
:10448000500D112485E29DE0689E9001699E300DDB
:10449000789E300D1124DA01A20FB31FFD01E456FE
:1044A000FB4FC080FD01E452FC4F808155245394A2
:1044B0005822082F06950170F82EF694F6949FE086
:1044C000F922829586958695837011811770110F58
:1044D000110F182BA352BC4FDC90D694D694D694CF
:1044E000EE24E3944A01590157C02E2D30E0C90152
:1044F0000197DC01AA0FBB1FA80FB91FA80DB91D9A
:10450000AA0DBB1DAD0144525C4FF901EE0FFF1F18
:10451000E20FF31FE80DF91DEA0DFB1DBF01645208
:104520007C4FEB0198819170EA0188818E7F892B05
:104530008883EB01988192708D7F892BEA018883B3
:10454000EB0198819C73837C892BEA018883EB01C2
:104550002881229526952695237099819770990F29
:10456000990F922B292F2295220F220F207C8F73D7
:10457000822BEA018883969596958981887F892B7D
:104580008983A352BC4FE352FC4F9081987F8C915A
:104590008770892B8C93E394CE1408F0A6CF8C2DD2
:1045A00090E0FC01EE0FFF1FE80FF91F84EC90E094
:1045B0009C01229EC001239E900D329E900D1124DD
:1045C000E80FF91F85E29DE0EC016C9EC0016D9E35
:1045D000900D7C9E900D1124E80FF91FDF01A4526D
:1045E000BC4F0170000F02702FE0F222FF0CFF0C95
:1045F0000529812F8295880F880F807C0F29082B31
:104600000C93E352FC4FDD0CDD0CDD0C169516957A
:104610001D2910838BE39BE2280E391E81E0E10106
:10462000888380914602909147028930910511F06C
:10463000079719F481E080932C01DF91CF911F91AE
:104640000F91FF90EF90DF90CF90BF90AF909F9031
:104650008F907F906F905F903F902F9008952F9252
:104660003F924F925F926F927F928F929F92AF9202
:10467000BF92CF92DF92EF92FF920F931F93DF933F
:10468000CF93CDB7DEB728970FB6F894DEBF0FBE35
:10469000CDBF4091352B803109F009C1442E5524FE
:1046A00085E29DE0489EA001499E500D589E500D08
:1046B0001124FA01EF5DFF4E208130E0F901EE0F89
:1046C000FF1FE20FF31FE40FF51FBF016B5D7F4E6D
:1046D000DB019C91662463946922DF01A95DBF4ED2
:1046E0008C91B82FBF70BA83782E771C7724771CF3
:1046F000E82EE294AFE0EA2217E0E122B92EB69468
:104700008FE1B822EA5DFF4EA080A694A694A694FD
:104710009295969596959370DB011196FC90F122F7
:10472000FF0CFF0CF92A1C821B82690116010894F8
:10473000210831084A0174C0C601EB81FC818E1B3F
:104740009F0B9C01220F331F280F391F280D391D85
:10475000B9016B5D7F4EDA01AA0FBB1FA40FB51F15
:10476000A80DB91D8D010B5D1F4EF8019081917050
:10477000FB0180818E7F892B8083A901495D5F4E7B
:10478000CD01895D9F4E9E838D83FC0190819F703A
:10479000FA018081807F892B8083ED81FE81908169
:1047A00090778F78892BFA018083ED81FE8190814B
:1047B00090788F77892BFA018083F8018081829528
:1047C00086958695837091819770990F990F982B94
:1047D000492F4295440F440F407CFB0180818F7329
:1047E000842B8083969596958181887F892B818300
:1047F0002A5D3F4EAA5DBF4E9C91987FD9018C9156
:104800008770892B8C93F80190819E73DB018C91CA
:10481000817C892B8C93EB81FC813196FC83EB832B
:10482000A1012B813C81421B530B2C153D0509F046
:1048300083CF85E29DE0489EA001499E500D589E81
:10484000500D1124DA01AB5DBF4E8C918E7F86290D
:104850008C93CA01895D9F4E37E0E322E29420EFFA
:10486000E222779477247794EA81EE2AE728FC0104
:10487000E0829F2D9295990F990F907C8C918F7368
:10488000892B8C934A5D5F4EAA0CAA0CAA0CF69455
:10489000F694FA28FA01F082FFE1BF22BB0C8C915A
:1048A000817C8B298C9381E08093B903FBC0242EFB
:1048B0003324A82EBB2484EC90E0A89EB001A99ECE
:1048C000700DB89E700D112485E29DE0289EA00118
:1048D000299E500D389E500D1124FB01E40FF51F49
:1048E000E456FB4F208130E0F901EE0FFF1FE20F8D
:1048F000F31FE60FF71FE40FF51F1CEDC12E13E0A9
:10490000D12ECE0EDF1ED6018C91B82FB170B98397
:10491000082F06950170F82EF694F6941FE0F12208
:104920008295869586958370D60111961C91177095
:10493000110F110F182BE352FC4FE080E694E69420
:10494000E6941C821B8269012601089441085108E3
:104950003B014A0164C0C601EB81FC818E1B9F0BA9
:104960009C01220F331F280F391F260D371D280DDC
:10497000391D38872F83A90144525C4FFB01EE0F8C
:10498000FF1FE60FF71FE60DF71DE80DF91DBF012C
:1049900064527C4FDB019C919170DA018C918E7F87
:1049A000892B8C93DB019C9192708D7F892BDA018E
:1049B0008C93DB019C919C73837C892BDA018C9313
:1049C000DB012C91229526952695237011969C91BA
:1049D0009770990F990F922B292F2295220F220F52
:1049E000207C8F73822BDA018C9396959695119685
:1049F0008C911197887F892B11968C93AF81B88504
:104A0000A352BC4FE352FC4F9081987F8C918770EA
:104A1000892B8C93EB81FC813196FC83EB83B20173
:104A20002B813C81621B730B2C153D0509F093CF44
:104A300084EC90E0A89EF001A99EF00DB89EF00DC8
:104A4000112485E29DE0DC012A9EC0012B9E900D81
:104A50003A9E900D1124E80FF91F9F0124523C4FFC
:104A60000170000F0270BFE0FB22FF0CFF0C898178
:104A7000082B812F8295880F880F807C0F29082BA7
:104A8000D9010C93E352FC4FEE0CEE0CEE0C169594
:104A900016951E291083EBE3FBE2AE0EBF1E81E0EC
:104AA000D5018C93809146029091470289309105FF
:104AB00011F0079719F481E080932C0128960FB626
:104AC000F894DEBF0FBECDBFCF91DF911F910F9144
:104AD000FF90EF90DF90CF90BF90AF909F908F901E
:104AE0007F906F905F904F903F902F900895CF935D
:104AF000DF936F5F2091352B8031B9F530E085E28F
:104B00009DE0289FA001299F500D389F500D112432
:104B100029C0862F90E0FC01EE0FFF1FE80FF91F60
:104B2000E40FF51FDF01AB5DBF4E8C918E7F8C9340
:104B3000CF01895D9F4E20E3EC0128838C91817C1D
:104B400088618C93EA5DFF4E8081877080838C91B1
:104B50008F738C9311968C911197887F8460119636
:104B60008C936F5F6034A8F22EC0422F50E0282F44
:104B700030E084EC90E0289FE001299FD00D389F21
:104B8000D00D112485E29DE0489F9001499F300D92
:104B9000589F300D112415C0862F90E0FC01EE0FB8
:104BA000FF1FE80FF91FEC0FFD1FE20FF31FDF01DE
:104BB000A452BC4F82E08C93E352FC4F84E080838C
:104BC0006F5F603448F3DF91CF910895CF93DF9307
:104BD0008091352BC82FD0E085E29DE09C01C29FDB
:104BE000C001C39F900DD29F900D1124FC01EE5384
:104BF000FC4F108270914D2BDC01A456BB4F20E07E
:104C000030E060E09C918081891708F490831196D0
:104C10009C9111978C91989FA0011124241735071E
:104C200010F0A90101C0762F6F5FAC53BF4F603108
:104C300011F09A01E7CF70934D2B85E29DE0C89F5C
:104C4000F001C99FF00DD89FF00D1124EE53FC4FD9
:104C5000E15AF34F9081EF55FC408081891708F4A9
:104C6000908385E29DE0C89FF001C99FF00DD89F19
:104C7000F00D1124EE53FC4FDF01A15AB34FE25A5D
:104C8000F34F80812C91829FC0011124481759074E
:104C900018F480E180934D2BDF91CF910895DF923E
:104CA000EF92FF920F931F93CF93DF938091352B59
:104CB00090E025E23DE0829FF001839FF00D929FFE
:104CC000F00D1124EE53FC4F1182C0E0D0E0E4EC73
:104CD000EE2EF12C05E21DE0DD24D3944C2F8091C3
:104CE000352B282F30E0CE9DF001CF9DF00DDE9DBD
:104CF000F00D1124209FC001219F900D309F900D39
:104D00001124E80FF91FE356FB4FE081DC01AE539D
:104D1000BC4F11968C9111978E1710F41196EC934D
:104D2000FE01EA54FD4FD082CE9DF001CF9DF00DE3
:104D3000DE9DF00D1124209FC001219F900D309F1A
:104D4000900D1124E80FF91FE456FB4F842F60816A
:104D50000E9477252196C031D10509F0BFCF8091FF
:104D6000352B282F30E085E29DE0289FF001299F18
:104D7000F00D389FF00D1124EE53FC4FE25AF34F23
:104D80009081EE55FC408181891708F4918381E080
:104D90008093C60285E29DE0289FF001299FF00DD7
:104DA000389FF00D1124EF5DFF4E80E160810E947D
:104DB00077250E94E6255F981092EA02DF91CF9155
:104DC0001F910F91FF90EF90DF9008951F938091B6
:104DD000933683FF0FC01091F53310931C370E9458
:104DE000AE0B8093F533811729F081E08093F03585
:104DF00080932C011F91089580914802837090E068
:104E0000009719F0039754F523C060913E0270910A
:104E10003F0280E090E00E94168C20E030E040EC01
:104E200052E40E94CC8C20E030E040E752E40E9443
:104E30007D8B9B01AC0160E074E284EF99E40E94F9
:104E40007D8B0E94EA8B709389006093880008959F
:104E500084EF91E090938900809388000895E1E8C1
:104E6000F0E0108280818093800080818A6080835E
:104E70000E94FC26EFE6F0E0808182608083089546
:104E8000CF92EF920F938130910509F04CC06F5F84
:104E90007F4F09F071C086EF91E060E071E00E9401
:104EA000C8898DEF91E060E071E00E94C88984E0DC
:104EB00092E060E071E00E94C8898BE092E060E0DF
:104EC00071E00E94C88982E192E060E071E00E9496
:104ED000C88989E192E060E071E00E94C88980E2BF
:104EE00092E060E071E00E94C88987E292E060E0B1
:104EF00071E00E94C8898EE292E060E071E00E9459
:104F0000C88980E58093F6351092F73587E097E3FE
:104F100062E143E124E105E1A6E1EA2EF7E1CF2ECB
:104F20000E94A97E29C0892B39F56F5F7F4F21F53B
:104F30008EE292E00E94088B87E292E00E94088B4A
:104F400080E292E00E94088B89E192E00E94088B47
:104F500082E192E00E94088B8BE092E00E94088B35
:104F600084E092E00E94088B8DEF91E00E94088B14
:104F700086EF91E00E94088B0F91EF90CF900895FB
:104F800080E090E06FEF7FEF0E944027089581E07E
:104F900090E06FEF7FEF0E94402708950E94A18468
:104FA0002091633630916436409165365091663673
:104FB000621B730B840B950B66307105810591059F
:104FC00008F470C00E94A1846093633670936436C5
:104FD00080936536909366364091F6353091F7357B
:104FE00020919737222381F0213051F48DB38093A3
:104FF00099379DB380919837809589238DBB04C0E4
:105000008FB7F894809399374CBD3DBD5E9A1EBC16
:1050100000000DB407FEFDCF8EB5809359361EBC3F
:1050200000000DB407FEFDCF8EB580935B361EBC2D
:1050300000000DB407FEFDCF8EB580935D361EBC1B
:1050400000000DB407FEFDCF8EB580935F361EBC09
:1050500000000DB407FEFDCF8EB5809361365E98DB
:10506000222339F080919937213011F48DBB01C092
:105070008FBF93B190729093FB35E9E5F6E3AEE410
:10508000B6E320818181281709F42C93329611967A
:1050900086E3E336F807A9F78091FC35981711F4F9
:1050A0009093FD354091F6353091F7352091973743
:1050B000222381F0213051F48DB3809399379DB331
:1050C00080919837809589238DBB04C08FB7F89461
:1050D000809399374CBD3DBD5E9A1EBC00000DB457
:1050E00007FEFDCF8EB580935A361EBC00000DB46E
:1050F00007FEFDCF8EB580935C361EBC00000DB45C
:1051000007FEFDCF8EB580935E361EBC00000DB449
:1051100007FEFDCF8EB5809360361EBC00000DB437
:1051200007FEFDCF8EB5809362365E98222339F05C
:1051300080919937213011F48DBB01C08FBF83B1AD
:1051400080728093FC350895CF93DF93EC018881C2
:10515000877E888320E0672B09F021E098819E7F7D
:10516000922B9883892F86958170281701F192FDE3
:105170000EC0213061F4986098830E94A1846093EE
:1051800093377093943780939537909396378881AF
:1051900082FF05C080FD03C080618F7D8883888188
:1051A000982F9170990F990F8B7F892B8883888115
:1051B00082FF18C080FF16C00E94A18420919337FF
:1051C000309194374091953750919637621B730B0D
:1051D000840B950B695E73408040904018F0888185
:1051E000806288838881982F9170990F8D7F892B99
:1051F0008883DF91CF910895DF92EF92FF920F9312
:105200001F93CF93DF930E94CE27E0905036D0902B
:1052100052360091513610E0B8016470707087E822
:1052200096E30E94A428B8016870707089E896E33C
:105230000E94A428B801617070708FE996E30E9403
:10524000A428FF24B701627070708DE996E30E9474
:10525000A4280270107087EA96E3B8010E94A4287F
:10526000B7016470707085E996E30E94A428B701C5
:105270006870707087E996E30E94A428B70160788F
:10528000707085EA96E30E94A428CD2DD0E0BE017F
:105290006170707089EA96E30E94A428BE01627072
:1052A00070708BEA96E30E94A428B7016072707058
:1052B0008DE896E30E94A428B7016074707081EABB
:1052C00096E30E94A428B701607170708FE896E39E
:1052D0000E94A42821E0E222FF2481E996E3B7019D
:1052E0000E94A428BE016072707089E996E30E9452
:1052F000A428BE01607170708BE996E30E94A42817
:1053000070914F3660E080914E3690E0682B792B9B
:1053100083E996E30E94A42820918B36D695C79501
:10532000D695C795CE018170682F267E922F982B37
:1053300090938B36892F86958170681729F192FD9D
:105340000FC0613069F4296020938B360E94A184DC
:105350006093AD367093AE368093AF369093B0368F
:1053600080918B3682FF06C080FD04C080618F7DF6
:1053700080938B3680918B36982F9170990F990F6F
:105380008B7F892B80938B3680918B36982F9170F1
:10539000990F8D7F892B80938B3682FF18C00E94D6
:1053A000A1842091AD363091AE364091AF36509108
:1053B000B036621B730B840B950B695E73408040A3
:1053C000904028F080918B36806280938B3620E06D
:1053D00030E0F901EE0FFF1FE959F94C8081877E1B
:1053E00080832F5F3F4F2031310599F7DF91CF91B7
:1053F0001F910F91FF90EF90DF9008951F93CF932F
:10540000DF93182F883038F1599AC82FD0E0809157
:10541000352B90E025E23DE0829FF001839FF00D67
:10542000929FF00D1124EE53FC4FEC0FFD1F87816E
:10543000882311F48FE301C084E10E94161082B129
:10544000C85ADE4F8F719881892B82B988E290E02B
:105450000E940885599888E290E00E940885599A30
:10546000183038F5149AC12FD0E08091352B90E098
:1054700025E23DE0829FF001839FF00D929FF00DA9
:105480001124EE53FC4FEC0FFD1F8781882311F48C
:105490008FE301C084E10E94161082B1C05ADE4F32
:1054A0008F719881892B82B988E290E00E940885EB
:1054B000149888E290E00E940885149ADF91CF91B9
:1054C0001F9108950F931F93CF93DF93C8E0D0E00F
:1054D00005E21DE0599A8091352B90E0809FF00104
:1054E000819FF00D909FF00D1124EE53FC4FEC0FB7
:1054F000FD1F8781882311F48FE301C084E10E949E
:10550000161082B18F71FE01E85AFE4F9081892BEF
:1055100082B988E290E00E94088559982196CC30A3
:10552000D105C1F688E290E00E940885599AC0E052
:10553000D0E005E21DE0149A8091352B90E0809F29
:10554000F001819FF00D909FF00D1124EE53FC4F60
:10555000EC0FFD1F8781882311F48FE301C084E1E4
:105560000E94161082B18F71FE01E05AFE4F9081A9
:10557000892B82B988E290E00E94088514982196D0
:10558000C830D105C1F688E290E00E940885149ADF
:10559000DF91CF911F910F910895CF92DF92EF92FB
:1055A000FF920F931F93CF93DF938C01C8E0D0E05D
:1055B000F4ECCF2ED12CE5E2EE2EEDE0FE2EC8016C
:1055C0000C2E02C0969587950A94E2F780FF5EC084
:1055D000599AFE01E15BFD4F808190E02091352BCF
:1055E00030E0FC01EE0FFF1FE80FF91FCC9DC0015A
:1055F000CD9D900DDC9D900D1124E80FF91F2E9D7F
:10560000C0012F9D900D3E9D900D1124E80FF91FB4
:10561000E452FC4F808181FD02C024E10FC08091E3
:105620004202909143020C2E02C0969587950A94EF
:10563000E2F780FD02C02FE301C02FE78091F03335
:105640009091F1330C2E02C0969587950A94E2F75B
:1056500080FF0CC080914402909145020C2E02C044
:10566000969587950A94E2F780FD20E0822F0E94AC
:10567000161082B18F71FE01E85AFE4F9081892B7E
:1056800082B988E290E00E94088559982196CC3032
:10569000D10509F094CF88E290E00E940885599ADC
:1056A000C0E0D0E064ECC62ED12C55E2E52E5DE0E2
:1056B000F52EC8010C2E02C0969587950A94E2F744
:1056C00080FF5EC0149AFE01E15BFD4F808190E097
:1056D0002091352B30E0FC01EE0FFF1FE80FF91F82
:1056E000CC9DC001CD9D900DDC9D900D1124E80F47
:1056F000F91F2E9DC0012F9D900D3E9D900D1124F0
:10570000E80FF91FE452FC4F808181FD02C024E1C3
:105710000FC080914202909143020C2E02C09695D8
:1057200087950A94E2F780FD02C02FE301C02FE7BE
:105730008091F0339091F1330C2E02C096958795AD
:105740000A94E2F780FF0CC08091440290914502D8
:105750000C2E02C0969587950A94E2F780FD20E012
:10576000822F0E94161082B18F71FE01E05AFE4F07
:105770009081892B82B988E290E00E940885149874
:105780002196C830D10509F094CF88E290E00E94BC
:105790000885149ADF91CF911F910F91FF90EF90A0
:1057A000DF90CF9008951F93CF93DF9310E0C0E078
:1057B000D0E084E49AE3BE0140E00E944882219652
:1057C00084E49AE3BE0143E60E944882219684E481
:1057D0009AE3BE0144E60E944882219684E49AE35B
:1057E000BE0141E00E944882219684E49AE3BE0112
:1057F00043E00E9448822196CA30D105D1F61F5F4E
:105800001038A9F6DF91CF911F9108952F923F9202
:105810004F925F926F927F928F929F92AF92BF92C0
:10582000CF92DF92EF92FF920F931F93CF93DF936C
:105830009AE0899F802D1124C4EBD6E304E0A02ECA
:10584000B12CAC0EBD1EEE24FF24C82EDD241601A3
:105850000894211C311C12E0412E512C4C0C5D1C73
:10586000B3E06B2E712C6C0C7D1CA4E08A2E912C65
:105870008C0C9D1CB7016C0D7D1D84E49AE348815E
:105880000E944882B1016E0D7F1D84E49AE34A8133
:105890000E94488282010E0D1F1DF50161917191D8
:1058A000819191915F0120E030E048EC52E40E9448
:1058B000CC8C0E94EA8B9B01AC0184E49AE3B80192
:1058C000422F0E944882B3016E0D7F1D84E49AE34B
:1058D0004A890E944882B4016E0D7F1D84E49AE3D8
:1058E0004C890E944882219685E090E0E80EF91EDE
:1058F00096E3C63BD90709F0BDCFDF91CF911F9149
:105900000F91FF90EF90DF90CF90BF90AF909F905E
:105910008F907F906F905F904F903F902F90089561
:1059200084E49AE360EA7FE040E00E9448820895C0
:1059300084E49AE360EA7FE0409109360E9448825D
:1059400008954F925F926F927F928F929F92AF9243
:10595000BF92CF92DF92EF92FF920F931F93CF935C
:10596000DF939AE0899F802D1124C4EBD6E334E0C5
:10597000C32ED12CCC0EDD1E00E010E0E82EFF245B
:1059800027010894411C511C22E0622E712C6E0CE0
:105990007F1C93E0892E912C8E0C9F1C84E0A82EF6
:1059A000B12CAE0CBF1CB8016E0D7F1D84E49AE3D0
:1059B0000E944182853008F084E08883B201600F44
:1059C000711F84E49AE30E9441828F3F09F48EEFB5
:1059D0008A83B301600F711F84E49AE30E944182BD
:1059E000853608F084E6682F70E0882777FD80957B
:1059F000982F0E94188C20E030E048EC52E40E947E
:105A00007D8BF6016083718382839383B401600F81
:105A1000711F84E49AE30E944182811181E08A8BA4
:105A2000B501600F711F84E49AE30E9441828830BF
:105A300008F087E08C8B1C861E86188A0B5F1F4F30
:105A4000219684E090E0C80ED91E0A30110509F0B5
:105A5000AACFDF91CF911F910F91FF90EF90DF9030
:105A6000CF90BF90AF909F908F907F906F905F90FE
:105A70004F9008951092E2361092CA3680E00E944C
:105A8000A12C80E00E94C61681E00E94C6160895EF
:105A900084E49AE360EA7FE00E94418280930936C1
:105AA000823020F0109209360E94982C0895AF920F
:105AB000BF92CF92DF92EF92FF920F931F9390913C
:105AC000C0369F5F9093C0368091C1368F5F8093C0
:105AD000C1368091CA36882349F080E098E00E9460
:105AE000541080E098E00E9489102FC1892F90E027
:105AF0004091B63620E031E0241B3109821793072C
:105B00000CF48BC01092C0368091B4368430D9F535
:105B10008091C236882309F075C060E070E080E0B3
:105B200090E02FEF30E040E050E00E947888E09075
:105B3000B836F090B9360091BA361091BB360E9453
:105B4000188CA80197010E94CC8C5B016C01C801E4
:105B5000B70120E030E040E053EC0E94CC8C20E024
:105B600030E040E053E40E94158B9B01AC01C6017C
:105B7000B5010E94158B0E94EA8B54E0660F771FD7
:105B80005A95E1F73BC0F82FE0E08091C236E80F6C
:105B9000F11DEF5CFB4FE491E090B836F090B93620
:105BA0000091BA361091BB366E2F70E0882777FDD2
:105BB0008095982F0E94188CA80197010E94CC8C88
:105BC0005B016C01C801B70120E030E040E053EC1C
:105BD0000E94CC8C20E030E040E053E40E94158B22
:105BE0009B01AC01C601B5010E94158B20E030E09D
:105BF00040E851E40E94CC8C0E94EA8B70932A37D3
:105C0000609329378091293790912A370E94541048
:105C10008091C2368F5F8093C2368091C13690E00A
:105C20004091B73620E031E0241B310982179307F9
:105C30000CF48BC01092C1368091B5368430D9F502
:105C40008091C336882309F075C060E070E080E081
:105C500090E02FEF30E040E050E00E947888E09044
:105C6000BC36F090BD360091BE361091BF360E9412
:105C7000188CA80197010E94CC8C5B016C01C801B3
:105C8000B70120E030E040E053EC0E94CC8C20E0F3
:105C900030E040E053E40E94158B9B01AC01C6014B
:105CA000B5010E94158B0E94EA8B44E0660F771FB6
:105CB0004A95E1F73BC0F82FE0E08091C336E80F4A
:105CC000F11DEF5CFB4FE491E090BC36F090BD36E7
:105CD0000091BE361091BF366E2F70E0882777FD99
:105CE0008095982F0E94188CA80197010E94CC8C57
:105CF0005B016C01C801B70120E030E040E053ECEB
:105D00000E94CC8C20E030E040E053E40E94158BF0
:105D10009B01AC01C601B5010E94158B20E030E06B
:105D200040E851E40E94CC8C0E94EA8B70932837A3
:105D30006093273780912737909128370E948910E8
:105D40008091C3368F5F8093C33680914A02882347
:105D500029F190914B02809148028370813041F487
:105D6000E0913D02F0E0E05DF74FE491E69506C07A
:105D7000E0913D02F0E0E05DF74FE491F0E09F5FDD
:105D800090934B029150892F90E08E179F0734F02B
:105D90000E94AF0F10924B0210924A0280914B3634
:105DA0008F5F80934B361F910F91FF90EF90DF90A4
:105DB000CF90BF90AF9008951F920F920FB60F92A1
:105DC0000BB60F9211242F933F934F935F936F93D2
:105DD0007F938F939F93AF93BF93EF93FF930E9413
:105DE000572DFF91EF91BF91AF919F918F917F912F
:105DF0006F915F914F913F912F910F900BBE0F903C
:105E00000FBE0F901F9018952F923F924F925F9266
:105E10006F927F928F929F92AF92BF92CF92DF92BA
:105E2000EF92FF920F931F93DF93CF93CDB7DEB71F
:105E300028970FB6F894DEBF0FBECDBF8091EA025F
:105E40008823D1F08091B7038823B1F42091B30364
:105E50003091B4038091B5039091B60382179307F4
:105E600058F48091B803882339F45F981092EA02BD
:105E70001092B4031092B3038091423690E08823CD
:105E800009F491E09093423680914E0260E30E94C3
:105E90004E8D943041F48091790190E0882309F48B
:105EA00091E09093790180914E026CE00E944E8DBA
:105EB000943051F4E091B102F0E0E658FE4F1082C8
:105EC00010924536109244368091AB02882311F42B
:105ED0000C94A637E6EBF6E34FEF50E030E880890C
:105EE000882309F4A1C082898330F1F1843028F439
:105EF000813069F18230A0F50CC0853009F454C0BE
:105F00008530B8F1863009F457C0873009F067C092
:105F10005EC08091AA0290E083709070892B09F096
:105F20005EC080914E02813009F059C08091E43604
:105F3000882311F0348704C084858093E536148665
:105F400090E08091E436882309F591E01FC08091AC
:105F5000AA0290E083709070892B09F040C004C0C1
:105F60008091AA0280FD3BC080914E028130B9F53C
:105F70002AC090914E02913011F00C941D388091FE
:105F8000E436882311F00C941D3834879093E4365E
:105F900026C08091E436882311F184858093E5360C
:105FA00014861092E4361BC080914E0260E30E947A
:105FB0004E8D9923A1F407C080914E0290E08F711D
:105FC0009070892B61F484858093E53607C08091B9
:105FD0004E0268E10E944E8D992309F414862081B7
:105FE000233000F19091E536892F80588F3768F47F
:105FF000BA01691B7109653171052CF08289833002
:1060000010F42B5F0EC02F5F0CC0892F815087FDCD
:1060100009C0953128F08289833010F4255001C0E1
:10602000215020831092E536319676E3E83BF7075E
:1060300009F055CF8091480283708230E0F580915D
:106040003A028330D1F0843028F4813071F082300C
:1060500080F407C0853019F18530C8F0863059F5D5
:1060600022C080914E0260E60BC080914E0260E338
:1060700007C080914E0268E103C080914E026CE03F
:106080000E944E8D9923B9F4809149020FC08091EE
:106090004E0290E083709070892B69F404C0809167
:1060A0004E0280FD08C08091490290E0882309F4E7
:1060B00091E0909349021092A5021092A4021092CE
:1060C000BA038AE096E39A838983AFE5BBE2BC8397
:1060D000AB8336EB432E32E0532E27EC622E22E0C8
:1060E000722E9E838D8318861F8285E2282E8DE076
:1060F000382E01E0802E912CA12CB12CDF80209134
:10610000352BB0E1DB1681F4822F90E0829DF00107
:10611000839DF00D929DF00D1124EE53FC4FE25A39
:10612000F34FC190F0801DC0822F90E02F81388501
:1061300044EC50E0249FF001259FF00D349FF00DBA
:106140001124BC01629DC001639D900D729D900D54
:106150001124E80FF91FEE53FC4FE552FF4FC080AA
:10616000F2903296E08080914E029C2D9695292FD8
:1061700030E090E06C2D70E00E945A8D82179307FA
:1061800031F4EF81F885ED56FD4F71E07083809119
:106190004E0290E06C2D70E00E945A8D821793079A
:1061A00009F068C0EF81F885EE57FD4F80818F5F61
:1061B00080838081F81608F4108281E0E81681F06F
:1061C000E81640F092E0E916C9F0A3E0EA1609F0FB
:1061D00051C03DC0EF81F885EE57FD4F808108C06A
:1061E000EF81F885EE57FD4F8081BF2DB81B8B2FB7
:1061F000EF81F885EF58FD4F80833CC0EF81F88533
:10620000EF58FD4F80818F1509F01FC7F301808182
:10621000813009F01AC7108206C0D3018C918823FF
:1062200011F4E1E0EC93D3018C91EF81F885EE5706
:10623000FD4FAF81B885AF58BD4F882311F08081E5
:1062400004C08081EF2DE81B8E2F8C9313C02F2D5F
:1062500030E02F5F3F4F442737FD4095542F60E0DB
:1062600070E080E090E00E947888EF81F885EF5838
:10627000FD4F60832091352B4F2D50E0F0E1DF166C
:1062800079F530E080915F0290E0841795071CF06B
:1062900080E090E004C080915F0290E00196FC01F4
:1062A000EE0FFF1FE80FF91F229DD001239DB00DB7
:1062B000329DB00D1124EA0FFB1FEB5DFF4E908164
:1062C000929596959695937081818770880F880F27
:1062D000892B482F50E040515040AE5DBF4E40C02A
:1062E000622F70E0EF81F885E15BFD4F808190E0E7
:1062F000841795071CF080E090E003C0808190E057
:106300000196FC01EE0FFF1FE80FF91F2F81388562
:1063100044EC50E0249FD001259FB00D349FB00D78
:106320001124EA0FFB1F629D9001639D300D729D49
:10633000300D1124E20FF31FE452FC4F908192952F
:1063400096959695937081818770880F880F892B19
:10635000482F50E040515040A20FB31FA156BB4FF1
:10636000AC91A15020914E020F81188507521D4F0C
:10637000F8018081EA2FF0E0EE0FFF1FE80FF11D1A
:10638000EE0FFF1FEE5BFE4F80819181820F911D0A
:10639000841B950B6C2D70E00E946E8D892B09F08B
:1063A0009CC2EF81F885ED56FD4F8081882309F46A
:1063B00094C21082D8018C9190E0882309F491E076
:1063C000EF81F885E752FD4F9083EF81F885E6581D
:1063D000FE4FB1E0B083EB16A1F0EB1640F0E2E027
:1063E000EE16D1F0F3E0EF1609F051C03DC0EF8199
:1063F000F885E05AFD4F8081EF81F885E15BFD4F24
:106400002DC0EF81F885E05AFD4F8081F81AEF81A9
:10641000F885E15BFD4F26C0EF81F885E15BFD4F1C
:1064200080818F1508F41AC6D2018C91813009F051
:1064300015C61C9206C0F2018081882311F421E068
:106440002083D2018C91EF81F885E15BFD4FAF8114
:10645000B885A05ABD4F882319F08C91808317C04E
:106460008C91F81AF08213C02F2D30E02F5F3F4F30
:10647000442737FD4095542F60E070E080E090E0C5
:106480000E947888EF81F885E15BFD4F6083209161
:10649000352BEF81F885E15BFD4FB0E1DB16C1F4F0
:1064A000808190E030E0FC01EE0FFF1FE80FF91F44
:1064B000229DC001239D900D329D900D1124E80F67
:1064C000F91FEA5DFF4E608166956695669524C06A
:1064D000808190E030E0FC01EE0FFF1FE80FF91F14
:1064E0004F81588564EC70E0469FC001479F900D36
:1064F000569F900D1124E80FF91F229DC001239D86
:10650000900D329D900D1124E80FF91FE452FC4FBD
:106510006081669566956F70EF81F885E15BFD4F50
:10652000808182958F70AB81BC819C918917F9F035
:10653000908192959F709C9380913A2B882329F0AB
:10654000EF81F885E25BF44D908380914602909153
:1065500047028330910541F08730910529F0893059
:10656000910511F0049719F4B1E0B0932C0120913A
:10657000352BE0E1DE16C9F480915F0290E030E057
:10658000FC01EE0FFF1FE80FF91F229DC001239DA4
:10659000900D329D900D1124E80FF91FEB5DFF4E19
:1065A000808181708093BA0339C0EF81F885E15B07
:1065B000FD4F808190E030E0FC01EE0FFF1FE80FFF
:1065C000F91F4F815885A4ECB0E04A9FC0014B9F52
:1065D000900D5A9F900D1124E80FF91F229DC001C4
:1065E000239D900D329D900D1124E80FF91FE45268
:1065F000FC4F808180FF12C02091A4023091A5023F
:1066000081E090E00F8002C0880F991F0A94E2F7A2
:10661000822B932B9093A5028093A402EF81F8859F
:10662000E15BFD4F808190E08F709070892B09F0C5
:1066300048C0808190E02091352B30E0FC01EE0FC6
:10664000FF1FE80FF91F4F815885A4ECB0E04A9F67
:10665000C0014B9F900D5A9F900D1124E80FF91F18
:10666000229DC001239D900D329D900D1124E80FB5
:10667000F91FE452FC4F808120910236309103369D
:1066800080FD0DC0D501C4010F8004C0880F991F83
:10669000AA1FBB1F0A94D2F7282B392B0EC0D50195
:1066A000C4010F8004C0880F991FAA1FBB1F0A9442
:1066B000D2F7809590952823392330930336209381
:1066C0000236EF81F885E05AFD4F80818F5F80832D
:1066D0006B3008F4AAC0B0E1DB16B9F02091A40237
:1066E0003091A502D501C4010F8004C0880F991F05
:1066F000AA1FBB1F0A94D2F78095909582239323FB
:106700009093A5028093A40202C01092BA036D3048
:1067100091F16E3030F46B3059F06C3009F0D5C027
:1067200010C06E3009F440C06F3009F0CEC055C0C3
:1067300060E070E080E090E029E030E040E050E090
:1067400054C060E070E080E090E027E030E040E09E
:1067500050E00E9478889B01AC0161307105810591
:10676000910509F0B2C060E1D61609F04BC071E0A6
:106770007093BA03AAC060E070E080E090E024E08B
:1067800030E040E050E00E9478889B01AC0161302D
:1067900071058105910509F098C080E1D81691F541
:1067A00091E09093BA0391C060E070E080E090E0E7
:1067B00023E030E040E050E00E9478889B01AC018B
:1067C000613071058105910509F07FC0A0E1DA16FD
:1067D000C9F4B1E0B093BA0378C060E070E080E043
:1067E00090E022E030E040E050E00E9478889B0199
:1067F000AC01613071058105910509F066C0E0E1E9
:10680000DE1679F08091A4029091A5020F8004C059
:10681000220F331F441F551F0A94D2F7822B932B4C
:106820004DC0F1E0F093BA0350C0862F81508730FD
:1068300068F470E06F5F7F4FAD81BE818C9190E016
:106840000E946E8D892B09F440C015C0683049F450
:10685000ED81FE81808163E00E944E8D9923A9F530
:1068600018C0693061F4AD81BE818C9190E0837075
:106870009070892B51F5B0E1DB1671F424C06A30B9
:1068800021F5ED81FE81808190E087709070892BE9
:10689000E1F4F0E1DF16B9F02091A4023091A502F5
:1068A000D501C4010F8004C0880F991FAA1FBB1F08
:1068B0000A94D2F780959095822393239093A50212
:1068C0008093A40202C01092BA038091A402909116
:1068D000A5029093A7028093A60220E1D21609F4A4
:1068E0007DC04091352B50E0BFE4EB2EB2E0FB2E93
:1068F0006F817885E60EF71ED7012C9180914E02AC
:1069000030E0F901EE0FFF1FE20FF31F24EC30E03F
:10691000629F8001639F100D729F100D1124E00F84
:10692000F11F429D9001439D300D529D300D112469
:10693000E20FF31FE352FC4FE081E695E695E69502
:10694000F0E0EC5CFE4FE08190E06E2F70E00E9482
:106950005A8D892B09F042C0EE2309F43FC0809183
:10696000A6029091A7020F8002C0969587950A947F
:10697000E2F780FF33C0D7018C9190E0FC01EE0F6D
:10698000FF1FE80FF91FE00FF11FE20FF31FE452A2
:10699000FC4F808180FF22C04091A4025091A5024B
:1069A0002091A4023091A502D501C4010F8004C03A
:1069B000880F991FAA1FBB1F0A94D2F7282B392BC7
:1069C0003093A5022093A4028091A4029091A50285
:1069D000842B952B9093A5028093A402EF81F885D8
:1069E0003196F887EF832D813E812F5F3F4F3E83A5
:1069F0002D834B815C814F5F5F4F5C834B83089499
:106A0000411C511C0894611C711C719709F076CBD4
:106A1000809148028370823038F480914902882343
:106A200011F02C9A01C02C988091BA03882309F4A4
:106A30000AC18091F202882309F005C18091B70351
:106A4000882309F000C18091352BE82EFF24809126
:106A50005F0220915F0290E0FC01EE0FFF1FE80F44
:106A6000F91F85E29DE0E89EB001E99E700DF89E59
:106A7000700D1124E60FF71FE95DFF4E90819F70A6
:106A8000DB01AE53BC4FA35AB34FEC918CE0E89FAF
:106A9000F0011124E90FF11DE355FC4FE491E150A1
:106AA000F0E0EE0FFF1FE75EFB4F4591549130E0A1
:106AB000F901EE0FFF1FE20FF31FE60FF71FE95D6D
:106AC000FF4E2081269526952695922F9E7080E078
:106AD000480F591F5093BD034093BC0380915F0240
:106AE00012962C9130E090E0821793071CF080E022
:106AF00090E004C080915F0290E00196FC01EE0FEF
:106B0000FF1FE80FF91F85E29DE0BC01E69EC00172
:106B1000E79E900DF69E900D1124E80FF91FE95D98
:106B2000FF4EE081EF7080915F0290E08217930743
:106B30001CF020E030E006C080915F02282F30E09A
:106B40002F5F3F4FF0E0E355FC4FE491F0E0EE0F94
:106B5000FF1FE75EFB4F85919491F901EE0FFF1F38
:106B6000E20FF31F05E21DE0E09ED001E19EB00DB3
:106B7000F09EB00D1124EA0FFB1FE95DFF4E40812E
:106B8000469546954695342F3E7020E0820F931F20
:106B90009093BF038093BE032091BC033091BD034B
:106BA000A05EBF4E6C91821B930B70E00E946E8DB5
:106BB0007093C1036093C003C9010E94E10F5F9A03
:106BC00081E08093EA022091352B30E080915F02D2
:106BD00090E0FC01EE0FFF1FE80FF91F209FD0018E
:106BE000219FB00D309FB00D1124EA0FFB1FEB5D0C
:106BF000FF4E808186958F71A05EBF4EAC91A0360E
:106C000039F490E00196880F991F880F991F08C0EA
:106C100090E0A03321F40196880F991F01C00196DE
:106C20009093B6038093B5032091B5033091B603DA
:106C30008A2F90E02817390720F081E08093B8036D
:106C400002C01092B80380915F0290E02091352B32
:106C500030E0FC01EE0FFF1FE80FF91F85E29DE019
:106C6000DC012A9FC0012B9F900D3A9F900D1124AB
:106C7000E80FF91FE95DFF4E808187FF14C0809106
:106C8000B703882381F48091C0039091C1032091C0
:106C9000BC033091BD03820F931F9093BD0380937B
:106CA000BC030E94E10F2091333630913436211518
:106CB0003105C1F080914E02E0913236F0E0EE589D
:106CC000FE4F608190E070E00E945A8D892B51F454
:106CD0008091A4029091A502822B932B9093A50200
:106CE0008093A4028091A4029091A502892B61F166
:106CF0008091A4029091A5029093453680934436EA
:106D00008091A4029091A5020E94CD2A8091350223
:106D1000882349F08091A4029091A5029F779093D7
:106D2000A5028093A4022091A4023091A502809133
:106D3000F0339091F13380959095822393230E94B4
:106D4000770F81E080934A02E0914D2BF0E0E05A0A
:106D5000FD4F808190E09093330180933201109138
:106D6000352B612F70E085E29DE0689FF001699FFF
:106D7000F00D789FF00D1124E456FB4F20E030E039
:106D800041E0D901A05ABD4F9C918081891750F4F0
:106D90001C92A981BA818C918F5F8C938150833D25
:106DA00008F04C932F5F3F4FEC53FF4F89819A813E
:106DB00001969A8389832031310519F72091700259
:106DC00085E29DE0689FF001699FF00D789FF00DCE
:106DD0001124EF5DFF4E8081821768F410927002DB
:106DE00080911A368F5F80931A368150833D18F058
:106DF00081E080931A3640914D2B403161F485E259
:106E00009DE0689FF001699FF00D789FF00D1124BF
:106E1000E05EFF4E19C0242F30E084EC90E0289F04
:106E2000F001299FF00D389FF00D112485E29DE0BF
:106E3000DC016A9FC0016B9F900D7A9F900D112419
:106E4000E80FF91FE356FB4F2081E42FF0E0E05AF2
:106E5000FD4F8081882309F056C080914E0290E05A
:106E6000622F70E00E945A8D30E02150304082172E
:106E7000930709F048C0109233011092320110922A
:106E80005C378091372B8823F1F1809146029091F5
:106E900047028230910541F08530910529F081301B
:106EA000910511F0892B79F51092372B1092352B23
:106EB000112319F481E08093352B8091B5028093E2
:106EC000B3020E944F2681E08093E63680932C0126
:106ED00080E090E021E0FC01E05AFD4F1082FC01CF
:106EE000E752FD4F1082FC01EE57FD4F1082FC016E
:106EF000E65FF94C2083FC01ED56FD4F208301969F
:106F00008131910541F740913201509133018091D7
:106F1000352B90E025E23DE0829FF001839FF00D4C
:106F2000929FF00D1124EE53FC4F808190E0019769
:106F30004817590709F09BC080915C37882309F0F6
:106F400096C081E08093D80280935C378091AB0239
:106F5000882349F480914E026CE00E944E8D992363
:106F600011F40E94622A8091AB02882309F52091D6
:106F700033363091343621153105D1F080914E02EF
:106F8000E0913236F0E0EE58FE4F608190E070E024
:106F90000E945A8D892B61F4C9010E94CD2A8091EB
:106FA0003336909134360E94770F81E080934A0205
:106FB00080914E028F5F80934E028150803658F14F
:106FC00081E080934E028091AA028F5F8093AA0293
:106FD0008091AA02803110F01092AA028091AA0238
:106FE00090E083709070892BB1F400E010E0809104
:106FF000023690910336002E02C0969587950A942A
:10700000E2F780FF03C0802F0E94FE290F5F1F4F11
:107010000C30110561F78091EA02882359F18091C3
:10702000B803882339F58091B3039091B403019696
:107030009093B4038093B3031DC080914E028130BE
:1070400011F00C94EF2F0C94C92FEF81F885EF58B5
:10705000FD4F8081882309F0E6C8DFC8EF81F885FD
:10706000E15BFD4F8081882309F0EBC9E4C91092F0
:10707000D8026CCF28960FB6F894DEBF0FBECDBFF6
:10708000CF91DF911F910F91FF90EF90DF90CF9004
:10709000BF90AF909F908F907F906F905F904F9038
:1070A0003F902F9008951F920F920FB60F920BB63C
:1070B0000F9211240F931F932F933F934F935F933E
:1070C0006F937F938F939F93AF93BF93EF93FF93B0
:1070D00080914802837090E08130910549F08230C0
:1070E0009105E1F1892B09F0ABC00E94042FA8C0E3
:1070F00080912636882309F466C0109220361092BB
:107100001F361092263680914E02843520F48091ED
:107110004E028C3018F48CE580934E0280914E0222
:107120008C3038F080914E02843218F484E18093E0
:107130004E0280914E02843238F080914E028C33A0
:1071400018F48CE280934E0280914E028C33D8F179
:1071500080914E028435B8F584E433C080912636A0
:10716000882389F11092203610921F36109226360D
:1071700080914E02843520F480914E028C3010F4C0
:1071800010924E0280914E028C3038F080914E0267
:10719000843218F488E180934E0280914E0284324A
:1071A00038F080914E028C3318F480E380934E02C5
:1071B00080914E028C3338F080914E02843518F461
:1071C00088E480934E0200911F3610912036609122
:1071D00068017091690180916A0190916B0128E1C9
:1071E00030E040E050E00E94818D0217130720F04C
:1071F0001092203610921F3680911F3690912036C3
:10720000892B11F40E94042F80911B3690911C361B
:10721000A0911D36B0911E360196A11DB11D80931F
:107220001B3690931C36A0931D36B0931E3680916A
:107230001F369091203601969093203680931F360A
:10724000FF91EF91BF91AF919F918F917F916F913E
:107250005F914F913F912F911F910F910F900BBE16
:107260000F900FBE0F901F901895FF920F931F93D2
:10727000F82E07E017E3C8016F2D41E00E94867DDC
:10728000C8016BE378E00E945A86C8016F2D41E087
:107290000E94867D1F910F91FF9008950F931F9379
:1072A00007E017E3C80164E040E00E94867DC80162
:1072B00069E978E00E945A8681E08093EC011F9191
:1072C0000F9108950F931F9307E017E3C80164E03F
:1072D00040E00E94867DC80163EA78E00E945A86F9
:1072E00081E08093EC011F910F91089587E097E36F
:1072F00062EB78E00E945A8608950F931F9307E08F
:1073000017E3C80160E040E00E94867DC80161E5A6
:1073100078E00E945A86C80160E041E00E94867DC4
:107320000E947639C80160E041E00E94867DC80174
:1073300060E478E00E945A861F910F9108950F93A0
:107340001F9307E017E3C80160E040E00E94867DDC
:10735000C80163E778E00E945A86C80160E041E016
:107360000E94867D0E947639C80160E041E00E945B
:10737000867DC80162E678E00E945A861F910F91CF
:1073800008950F931F93CF93DF93C0E0D0E0082FB1
:1073900010E006C087E097E361EA0E947D862196AF
:1073A000C017D107BCF3DF91CF911F910F910895C2
:1073B00088E00E943539E091E236F0E0EC54F94C77
:1073C00084898330D1F1843030F4813009F449C0AC
:1073D0008230E0F54DC08530C9F0853000F186304F
:1073E00061F0873009F04AC087E097E360E00E94CF
:1073F0007C7D87E097E361E031C087E097E360E060
:107400000E947C7D87E097E361E011C087E097E30D
:1074100060E00E947C7D87E097E363E01FC087E027
:1074200097E360E00E947C7D87E097E363E00E9441
:107430007C7D87E097E362E011C087E097E360E03E
:107440000E947C7D87E097E366E008C087E097E3D1
:1074500060E00E947C7D87E097E367E00E947C7D8E
:10746000089587E097E36FEA78E00E945A860895CE
:1074700087E097E36CEA78E00E945A8608951F93AC
:107480002091B1024091352B203171F4242F30E04E
:1074900085E29DE0289FF001299FF00D389FF00DB7
:1074A0001124E05EFF4E19C030E050E084EC90E023
:1074B000289FF001299FF00D389FF00D112485E2DF
:1074C0009DE09C01429FC001439F900D529F900DF3
:1074D0001124E80FF91FE356FB4F108188E00E944A
:1074E0003539183109F1193130F41C3059F01031A7
:1074F00009F044C010C0103371F11036A9F11032F8
:10750000E9F51BC087E097E360E00E947C7D87E09F
:1075100097E364E031C087E097E360E00E947C7D00
:1075200087E097E361E011C087E097E360E00E94A5
:107530007C7D87E097E361E01FC087E097E360E030
:107540000E947C7D87E097E363E00E947C7D87E07A
:1075500097E362E011C087E097E360E00E947C7DE2
:1075600087E097E363E008C087E097E360E00E946C
:107570007C7D87E097E366E00E947C7D1F91089503
:10758000CF92DF92EF92FF920F931F93CF93DF93EF
:10759000EC018B017A01690166EF71E00E94E288DB
:1075A000882321F587E097E360E041E00E94867D33
:1075B00087E097E362ED78E00E945A868C819D8196
:1075C000029720F487E097E361E003C087E097E348
:1075D00060E041E00E94867D87E097E3BE010E9463
:1075E000238886EF91E0BE010E94DB8AC8016DEF1F
:1075F00071E00E94E2888823E1F487E097E364E089
:1076000041E00E94867D87E097E36DEC78E00E9480
:107610005A8687E097E364E041E00E94867D87E038
:1076200097E3B8010E9423888DEF91E0B8010E9492
:10763000DB8AC70164E072E00E94E288882329F5B2
:1076400087E097E368E041E00E94867D87E097E36A
:1076500068EC78E00E945A86F70184819581029750
:1076600020F487E097E369E003C087E097E368E0F0
:1076700041E00E94867D87E097E3B7010E9423885E
:1076800084E092E0B7010E94DB8AC6016BE072E001
:107690000E94E288882329F587E097E36CE041E0C7
:1076A0000E94867D87E097E363EC78E00E945A862B
:1076B000F60184819581029720F487E097E36DE0DD
:1076C00003C087E097E36CE041E00E94867D87E09D
:1076D00097E3B6010E9423888BE092E0B6010E94F6
:1076E000DB8ADF91CF911F910F91FF90EF90DF9098
:1076F000CF9008958F929F92AF92BF92CF92DF92D8
:10770000EF92FF920F931F93DF93CF93CDB7DEB726
:10771000CF57D3400FB6F894DEBF0FBECDBF8091D8
:10772000ED018823A1F087E097E36091F00141E04B
:107730000E94867D809179018823F1F487E097E3A8
:1077400061E071E00E94828710922E371EC0809106
:107750002E378823D1F48091EE0190E020914602EB
:10776000309147028217930781F487E097E3609195
:10777000F00141E00E94867D87E097E36EE272E0CF
:107780000E94238881E080932E378091EE0190E063
:1077900020914602309147028217930711F0109210
:1077A000ED0180912C01882311F40C944251109228
:1077B0002C018091F501882309F472C087E097E3DA
:1077C00060E040E00E94867D87E097E36EE47AE027
:1077D0000E945A8687E097E360E041E00E94867D40
:1077E0000E94763987E097E362E041E00E94867D5F
:1077F00087E097E36CE47AE00E945A8687E097E39B
:1078000065E041E00E94867D87E00E94C13987E003
:1078100097E36EE041E00E94867D87E097E36AE4AB
:107820007AE00E945A862091B1024091352B203196
:1078300071F4242F30E085E29DE0289FF001299F1C
:10784000F00D389FF00D1124EE5DFF4E19C030E0B1
:1078500050E084EC90E0289FF001299FF00D389FC4
:10786000F00D112485E29DE09C01429FC001439FE1
:10787000900D529F900D1124E80FF91FE156FB4F18
:1078800060816C5F87E097E341E00E94867D87E03E
:1078900097E36BED0E947D868BE090E00C943E5167
:1078A0008091F401882309F475C087E097E360E0D4
:1078B00040E00E94867D80914602909147020297A7
:1078C00029F487E097E369E37AE004C087E097E36F
:1078D00068E27AE00E945A8687E097E360E041E040
:1078E0000E94867D0E94763987E097E363E041E05D
:1078F0000E94867D2091B1024091352BDE01A9586E
:10790000BC4F2031B9F4242F30E085E29DE0289F60
:10791000F001299FF00D389FF00D1124ED5DFF4E11
:107920008081E82FF0E0EE0FFF1FE551FD4F6591DC
:10793000749122C030E050E084EC90E0289FF00188
:10794000299FF00D389FF00D112485E29DE0BC01C8
:10795000469FC001479F900D569F900D1124E80F40
:10796000F91FE256FB4F8081E82FF0E0EE0FFF1F7A
:10797000E551FD4F65917491CD010E94190887E092
:1079800097E3BE0169587C4F0E9482878AE090E0AD
:107990000C943E51809146029091470286309105A9
:1079A00011F40C940B4987309105D4F48230910581
:1079B00009F42FC28330910554F4009711F40C940C
:1079C000834E019711F00C9442510C945A4D84301F
:1079D000910509F458C5059714F00C94154D2EC364
:1079E0008930910511F40C944D4A8A30910554F474
:1079F0008730910511F40C940D46089711F00C9402
:107A0000425110C08D30910511F40C94544F8E30BA
:107A1000910511F40C942F500C9711F00C944251D5
:107A20000C947A458091AE029091AF020897A9F02C
:107A30008BE092E066E071E00E94FC89BC0184E08A
:107A400092E00E94DB8ABC018DEF91E00E94DB8A0C
:107A5000BC0186EF91E00E94DB8A8091F1018130C8
:107A600029F0823011F00C944251BBC08091AE02DB
:107A70009091AF02089761F480914101813041F407
:107A800080912D01882321F48091EC018823D1F18C
:107A900088E090E09093AF028093AE028091F10174
:107AA0008093410110922D011092EC0187E097E341
:107AB00060E040E00E94867D87E097E367E17AE03E
:107AC0000E945A868091EF01E82FF0E0EE0FFF1F31
:107AD000E557FD4F659174918E010F5F1F4FC801EF
:107AE0000E941908E091EF01F0E0E25DFE4F87E0AF
:107AF00097E3608140E00E94867D87E097E3B801CC
:107B00000E948287809148028370E82FF0E0EE0F98
:107B1000FF1FE55AFC4F659174917E010894E11CAA
:107B2000F11CC7010E94190882E192E0B7010E948E
:107B3000FC898E010B5F1F4F6091400270914102E2
:107B4000C8014AE00E94158A89E192E0B8010E94CA
:107B5000DB8AC8010E94088B8E01045F1F4FC80199
:107B600060913D024AE00E94778A80E292E0B8018B
:107B70000E94DB8AC8010E94088B80913A02E82F9C
:107B8000F0E0EE0FFF1FE35BFC4F65917491C701BE
:107B90000E94190887E292E0B7010E94FC89F3E194
:107BA000AF2EB12CAC0EBD1EC50162E172E00E9489
:107BB000F28AEAE1CE2ED12CCC0EDD1EC60169E19F
:107BC00072E00E94F28A71E2E72EF12CEC0EFD1EAB
:107BD000C70160E272E00E94F28A8E01085D1F4FC9
:107BE000FFC080914101823049F480912D018823AA
:107BF00029F48091EC01882309F44DC082E0809340
:107C0000410110922D011092EC0187E097E360E0B2
:107C100040E00E94867D87E097E36BE07AE00E9477
:107C20005A868091B4028093303787E097E36FE7FC
:107C30000E947D8687E097E368E07AE00E945A869A
:107C40006091B40270E06F5F7F4F87E097E34AE096
:107C500050E00E946F878091EF01E82FF0E0EE0F77
:107C6000FF1FED56FD4F659174918E010F5F1F4F01
:107C7000C8010E941908E091EF01F0E0E25DFE4FBB
:107C800087E097E3608140E00E94867D87E097E38C
:107C9000B8010E948287909130378091B402981782
:107CA00009F187E097E36FE040E00E94867D87E07E
:107CB00097E366E07AE00E945A8687E097E36EE0F9
:107CC00040E00E94867D6091B40270E06F5F7F4F5C
:107CD00087E097E34AE050E00E946F878091B4020A
:107CE0008093303780913602E82FF0E0EE0FFF1FCF
:107CF000EF55FC4F659174918E010F5F1F4FC801C6
:107D00000E94190882E192E0B8010E94FC898091EA
:107D10003502E82FF0E0EE0FFF1FEB55FC4F6591A9
:107D20007491C8010E94190889E192E0B8010E948B
:107D3000FC89E0914402F09145020090B40202C037
:107D4000F695E7950A94E2F7E170F070EE0FFF1FE9
:107D5000EB55FC4F65917491C8010E94190880E2AF
:107D600092E0B8010E94FC89E0914202F091430246
:107D70000090B40202C0F695E7950A94E2F7E1702C
:107D8000F070EE0FFF1FE755FC4F65917491C8012D
:107D90000E94190887E292E0B8010E94FC899FE2E4
:107DA000A92EB12CAC0EBD1EC50162E172E00E948D
:107DB000F28A86E3C82ED12CCC0EDD1EC60169E105
:107DC00072E00E94F28A0DE3E02EF12CEC0EFD1E13
:107DD000C70160E272E00E94F28A8E010C5B1F4FC5
:107DE000C80167E272E00E94F28AC501B601A701EC
:107DF00098010E94C03AC8010E94088BC7010E94E6
:107E0000088BC6010E94088BC5010E94088B0C9448
:107E1000425187E097E360E040E00E94867D8091D8
:107E2000F201882309F445C087E097E365EF79E024
:107E30000E945A8687E097E360E041E00E94867DD9
:107E40000E94763987E097E364E041E00E94867DF6
:107E5000E091B102F0E0E25BF44D608170E06F5FB1
:107E60007F4F87E097E34AE050E00E946F8787E00A
:107E700097E36BE041E00E94867D8091352B90E096
:107E800025E23DE0829FF001839FF00D929FF00D6F
:107E90001124EE53FC4F608170E06F5F7F4F87E0ED
:107EA00097E34AE050E00E946F8781E08093F301FE
:107EB00077C08091AE029091AF02029749F4809111
:107EC000F301882329F48091EC01882309F468C028
:107ED00082E090E09093AF028093AE021092F301A3
:107EE0001092EC0187E097E364EE79E00E945A86F5
:107EF00087E097E360E041E00E94867D0E9476394A
:107F000087E097E362E041E00E94867D6091B202E3
:107F10006F5B87E097E30E947D866091B30270E01B
:107F20006F5F7F4F8091B20290E014E0880F991F3D
:107F30001A95E1F7681B790B87E097E34AE050E078
:107F40000E946F878091B3028093303787E097E378
:107F500069E041E00E94867D87E097E365E00E944A
:107F60007C7D87E097E368E071E00E9482878091E2
:107F70004802837039F087E097E360EE79E00E9471
:107F80005A860AC060913E0270913F0287E097E3F3
:107F90004AE050E00E940C8780913E0280932F3788
:107FA0009091B30280913037981719F182E00E94C6
:107FB00035396091B2026F5B87E097E30E947D865E
:107FC0006091B30270E06F5F7F4F8091B20290E0EA
:107FD000B4E0880F991FBA95E1F7681B790B87E029
:107FE00097E34AE050E00E946F878091B30280934C
:107FF000303780912F3790E020913E0230913F0240
:108000008217930711F40C944251809148028370B7
:1080100011F00C9442518BE00E94353960913E0280
:1080200070913F0287E097E34AE050E00E940C879E
:1080300080913E0280932F370C9442518091AE0282
:108040009091AF020397C1F08BE092E066E071E09F
:108050000E94FC89BC0184E092E00E94DB8ABC01A2
:108060008DEF91E00E94DB8ABC0186EF91E00E94D7
:10807000DB8A81E00E943F3A8091AE029091AF028C
:10808000039741F480912D01882321F48091EC0124
:10809000882381F187E097E360E040E00E94867DDD
:1080A00087E097E36FEC79E00E945A868091EF01B8
:1080B000E82FF0E0EE0FFF1FE553FD4F659174913F
:1080C0008E010F5F1F4FC8010E941908E091EF0158
:1080D000F0E0E25DFE4F87E097E3608140E00E94C0
:1080E000867D87E097E3B8010E94828710922D0178
:1080F0001092EC018E01055B1F4FE091B102F0E0A0
:10810000E15AF44D608170E06F5F7F4FC8014AE033
:108110000E94468ACE018E5A9F4FB8010E94FD8A66
:1081200080913A2B882311F460E201C06EE7E2E50A
:10813000CE2ED12CCC0EDD1EC6010E9480898C0172
:1081400079E5E72EF12CEC0EFD1EE091B102F0E096
:10815000E25BF44D608170E06F5F7F4FC7014AE0E2
:108160000E94468AC801B7010E949189BC018E0114
:10817000005A1F4FC8010E94F28A82E192E0B801C2
:108180000E94DB8AC8010E94088BC7010E94088BED
:10819000C6010E940E8BCE01855B9F4F0E94088B0B
:1081A0002091B1024091352B203171F4242F30E021
:1081B00085E29DE0289FF001299FF00D389FF00D8A
:1081C0001124EF5DFF4E19C030E050E084EC90E0E8
:1081D000289FF001299FF00D389FF00D112485E2B2
:1081E0009DE09C01429FC001439F900D529F900DC6
:1081F0001124E80FF91FE456FB4F8081682F70E0CF
:108200006F5F7F4F8E0109591F4FC8014AE00E94DE
:10821000468A89E192E0B8010E94DB8AC8010E9487
:10822000088B80E292E060E070E00E94FC8940915F
:10823000B102403139F48E0102591F4FC8016AE082
:1082400071E092C080910936882309F481C0E42F3F
:10825000F0E0EE0FFF1FE757FC4F65917491CE01E0
:1082600001960E9419084091B1024C3090F580911E
:10827000352B90E025E23DE0829FF001839FF00DD9
:10828000929FF00D1124EE53FC4FE40FF11D8781F6
:10829000882311F460E201C06BE25CE7C52ED12CAB
:1082A000CC0EDD1EC6010E94C28A45E7E42EF12CE9
:1082B000EC0EFD1EC701BE016F5F7F4F0E94C88993
:1082C000C601B7010E949189BC018E010D571F4F55
:1082D0008AC04F3041F480913502882321F08E010D
:1082E00006571F4F3EC08091352B90E025E23DE0C0
:1082F000829FF001839FF00D929FF00D1124EE53A9
:10830000FC4FE40FF11D8781882311F460E201C066
:108310006BE238E9C32ED12CCC0EDD1EC6010E94C3
:10832000C28A21E9E22EF12CEC0EFD1E6091B10211
:1083300070E06F5F7F4FC7014AE00E94468AC60126
:10834000B7010E949189BC018E0101561F4F4BC09D
:108350004F30A9F480913502882389F08E010A55A7
:108360001F4FC8016DE071E00E94C88987E292E06A
:10837000B8010E94DB8AC8010E94088B45C0809129
:10838000352B90E025E23DE0829FF001839FF00DC8
:10839000929FF00D1124EE53FC4FE40FF11D8781E5
:1083A000882311F460E201C06BE294EBC92ED12C5A
:1083B000CC0EDD1EC6010E94C28A8DEAE82EF12C89
:1083C000EC0EFD1E6091B10270E06F5F7F4FC70140
:1083D0004AE00E94468AC601B7010E949189BC0109
:1083E0008E0105541F4FC8010E94F28A87E292E075
:1083F000B8010E94DB8AC8010E94088BC7010E9455
:10840000088BC6010E940E8B02ECA02EB12CAC0E84
:10841000BD1EC50162E172E00E94F28A19ECC12E14
:10842000D12CCC0EDD1EC60169E172E00E94F28AF9
:10843000B0EDEB2EF12CEC0EFD1EC70160E272E0F8
:108440000E94F28A8E0109521F4FC80167E272E052
:108450000E94F28AC501B601A70198010E94C03AA4
:10846000C8010E94088BC7010E94088BC6010E94A8
:10847000088BC5010E94088B80E00E943F3A83E090
:1084800090E00C943E518091B1022091AE02309167
:10849000AF02803109F001C124303105A9F08BE031
:1084A00092E066E071E00E94FC89BC0184E092E009
:1084B0000E94DB8ABC018DEF91E00E94DB8ABC0147
:1084C00086EF91E00E94DB8A8091AE029091AF022C
:1084D000049741F480912D01882321F48091EC01CF
:1084E0008823A1F187E097E360E040E00E94867D69
:1084F00087E097E36EEB79E00E945A868091EF0166
:10850000E82FF0E0EE0FFF1FED51FD4F65917491E4
:108510008E010F5F1F4FC8010E941908E091EF0103
:10852000F0E0E25DFE4F87E097E3608140E00E946B
:10853000867D87E097E3B8010E9482878091BB0324
:108540008093410110922D011092EC018091352B06
:1085500090E025E23DE0829FF001839FF00D929F25
:10856000F00D1124E15EFF4E8081E82FF0E0EE0F68
:10857000FF1FED50FD4F659174917E010894E11C41
:10858000F11CC7010E9419088E0102521F4FC80139
:10859000B7010E94C88982E192E0B8010E94DB8A9B
:1085A000C8010E94088B8091F535E82FF0E0EE0FAE
:1085B000FF1FEF58FC4F65917491C7010E94190885
:1085C0008E010B511F4FC801B7010E94C88989E174
:1085D00092E0B8010E94DB8AC8010E94088B8E01DC
:1085E00004511F4F60915E0170E063507040C801FC
:1085F0004AE00E94468A80E292E0B8010E94DB8A4B
:10860000C8010E94088B8E010D501F4FC80160E009
:1086100071E00E94C88987E292E0B8010E94DB8A7B
:10862000C8010E94088B5AEFA52EB12CAC0EBD1EBE
:10863000C50162E172E00E94F28A41E0C42ED42EAC
:10864000CC0EDD1EC60169E172E00E94F28A38E0BC
:10865000E32E31E0F32EEC0EFD1EC70160E272E066
:108660000E94F28A8E01015F1E4FC80167E272E02C
:108670000E94F28AC501B601A70198010E94C03A82
:10868000C8010E94088BC7010E94088BC6010E9486
:10869000088BC5010E94088B29C224303105C1F026
:1086A0008BE092E066E071E00E94FC89BC0184E00E
:1086B00092E00E94DB8ABC018DEF91E00E94DB8A90
:1086C000BC0186EF91E00E94DB8A81E00E943F3A84
:1086D0008091AE029091AF02049741F480912D01F8
:1086E000882321F48091EC01882381F187E097E3CE
:1086F00060E040E00E94867D87E097E36DEA79E0E4
:108700000E945A868091EF01E82FF0E0EE0FFF1FE4
:10871000E553FD4F659174918E010F5F1F4FC801A6
:108720000E941908E091EF01F0E0E25DFE4F87E062
:1087300097E3608140E00E94867D87E097E3B8017F
:108740000E94828710922D011092EC018E010A5E28
:108750001E4FE091B102F0E0E15AF44D608170E00B
:108760006F5F7F4FC8014AE00E94468ACE01835E58
:108770009E4FB8010E94FD8A80913A2B882311F404
:1087800060E201C06EE79DE1C92E91E0D92ECC0ECA
:10879000DD1EC6010E9480898C0184E2E82E81E002
:1087A000F82EEC0EFD1EE091B102F0E0E25BF44D1C
:1087B000608170E06F5F7F4FC7014AE00E94468A88
:1087C000C801B7010E949189BC018E01055D1E4F51
:1087D000C8010E94F28A82E192E0B8010E94DB8A1D
:1087E000C8010E94088BC7010E94088BC6010E9425
:1087F0000E8BCE018A5E9E4F0E94088B2091B102A3
:108800004091352B203171F4242F30E085E29DE03A
:10881000289FF001299FF00D389FF00D1124EF5D86
:10882000FF4E19C030E050E084EC90E0289FF0014A
:10883000299FF00D389FF00D112485E29DE0BC01C9
:10884000469FC001479F900D569F900D1124E80F41
:10885000F91FE456FB4F8081682F70E06F5F7F4FF8
:108860008E010E5C1E4FC8014AE00E94468A89E1D3
:1088700092E0B8010E94DB8AC8010E94088B80E266
:1088800092E060E070E00E94FC894091B1024031CA
:1088900039F48E01075C1E4FC8016AE071E096C092
:1088A00080910936882309F485C0E42FF0E0EE0FAB
:1088B000FF1FE757FC4F65917491CE0101960E940E
:1088C00019084091B1024C30A0F58091352B90E011
:1088D00025E23DE0829FF001839FF00D929FF00D15
:1088E0001124EE53FC4FE40FF11D8781882311F40E
:1088F00060E201C06BE2B7E4CB2EB1E0DB2ECC0E20
:10890000DD1EC6010E94C28AA0E4EA2EA1E0FA2E72
:10891000EC0EFD1EC701BE016F5F7F4F0E94C8892C
:10892000C601B7010E949189BC018E01025B1E4FF6
:108930008EC04F3041F480913502882321F08E01A2
:108940000B5A1E4F40C08091352B90E025E23DE050
:10895000829FF001839FF00D929FF00D1124EE5342
:10896000FC4FE40FF11D8781882311F460E201C000
:108970006BE2F3E6CF2EF1E0DF2ECC0EDD1EC6015A
:108980000E94C28AECE5EE2EE1E0FE2EEC0EFD1E0A
:108990006091B10270E06F5F7F4FC7014AE00E94B3
:1089A000468AC601B7010E949189BC018E01065911
:1089B0001E4F4DC04F30A9F480913502882389F0B5
:1089C0008E010F581E4FC8016DE071E00E94C889EA
:1089D00087E292E0B8010E94DB8AC8010E94088BFE
:1089E00047C08091352B90E025E23DE0829FF00169
:1089F000839FF00D929FF00D1124EE53FC4FE40F76
:108A0000F11D8781882311F460E201C06BE27FE7EA
:108A1000C72E71E0D72ECC0EDD1EC6010E94C28A81
:108A200068E7E62E61E0F62EEC0EFD1E6091B102C5
:108A300070E06F5F7F4FC7014AE00E94468AC6011F
:108A4000B7010E949189BC018E010A571E4FC801CF
:108A50000E94F28A87E292E0B8010E94DB8AC80194
:108A60000E94088BC7010E94088BC6010E940E8BD2
:108A70005DE8A52E51E0B52EAC0EBD1EC50162E12C
:108A800072E00E94F28A44E9C42E41E0D42ECC0E5A
:108A9000DD1EC60169E172E00E94F28A3BE9E32E25
:108AA00031E0F32EEC0EFD1EC70160E272E00E9481
:108AB000F28A8E010E551E4FC80167E272E00E94D5
:108AC000F28AC501B601A70198010E94C03AC80107
:108AD0000E94088BC7010E94088BC6010E94088B68
:108AE000C5010E94088B80E00E943F3A84E090E03C
:108AF0000C943E518091AE029091AF020C9721F4FC
:108B00008091EC018823B9F187E097E360E040E0D1
:108B10000E94867D0E94763987E097E362E040E01C
:108B20000E94867D87E097E368EA79E00E945A8692
:108B300087E097E360E041E00E94867D0E947639FD
:108B400087E097E362E041E00E94867D87E097E35B
:108B500065EA79E00E945A86E0913236F0E0E95207
:108B6000F74FE49187E097E36E2F4AE050E00E94D0
:108B70001D871092EC01E0913236F0E0E952F74F98
:108B8000E4918E0107551E4FC8016E2F4AE00E94E6
:108B9000778A86EF91E0B8010E94E288F82EC8013A
:108BA0000E94088BFF20A9F587E097E364E041E08D
:108BB0000E94867D87E097E361EA79E00E945A8609
:108BC00087E097E364E041E00E94867DE0913236E1
:108BD000F0E0E952F74FE49187E097E36E2F4AE027
:108BE00050E00E941D87E0913236F0E0E952F74FE5
:108BF000E4918E0100551E4FC8016E2F4AE00E947D
:108C0000778A86EF91E0B8010E94DB8AC8010E9452
:108C1000088B8CE090E00C943E518091BB0388233C
:108C200021F0813009F0F3C2E3C18091AE0290914E
:108C3000AF02079721F4809141018823A9F08BE0CE
:108C400092E066E071E00E94FC89BC0184E092E061
:108C50000E94DB8ABC018DEF91E00E94DB8ABC019F
:108C600086EF91E00E94DB8A8091AE029091AF0284
:108C7000079771F49091BB0380914101981741F4DB
:108C800080912D01882321F48091EC018823A1F1AA
:108C900087E097E360E040E00E94867D87E097E30D
:108CA00060E979E00E945A868091EF01E82FF0E0B8
:108CB000EE0FFF1FE555FD4F659174918E010F5F1B
:108CC0001F4FC8010E941908E091EF01F0E0E25D3A
:108CD000FE4F87E097E3608140E00E94867D87E059
:108CE00097E3B8010E9482878091BB038093410182
:108CF00010922D011092EC018E0109541E4FE0914B
:108D0000B102F0E0E15AF44D608170E06F5F7F4F97
:108D1000C8014AE00E94468ACE0182549E4FB801A3
:108D20000E94FD8A80913A2B882311F460E201C0F1
:108D30006EE79EEBC92E91E0D92ECC0EDD1EC6014A
:108D40000E9480898C0185ECE82E81E0F82EEC0EE3
:108D5000FD1EE091B102F0E0E25BF44D608170E055
:108D60006F5F7F4FC7014AE00E94468AC801B70182
:108D70000E949189BC018E0104531E4FC8010E94BC
:108D8000F28A82E192E0B8010E94DB8AC8010E9467
:108D9000088BC7010E94088BC6010E940E8BCE0172
:108DA00089549E4F0E94088B2091352B30E0809192
:108DB0004C0290E0FC01EE0FFF1FE80FF91FA5E247
:108DC000CA2EADE0DA2E2C9DD0012D9DB00D3C9D1C
:108DD000B00D1124EA0FFB1FE95DFF4E90819F70DB
:108DE000A15EBF4EEC918CE0E89FF0011124E90FE9
:108DF000F11DE355FC4FE491F0E0EE0FFF1FE15948
:108E0000FC4F659174917E010894E11CF11CC7012F
:108E10000E9419088E010D521E4FC801B7010E9411
:108E2000C88989E192E0B8010E94DB8AC8010E94EA
:108E3000088B80914C0290E02091352B30E0FC01B2
:108E4000EE0FFF1FE80FF91F2C9DC0012D9D900D07
:108E50003C9D900D1124E80FF91FE95DFF4E8081C4
:108E600082958770E82FF0E0EE0FFF1FEF59FC4F5F
:108E700065917491C7010E9419088E0106521E4F18
:108E8000C801B7010E94C88980E292E0B8010E943F
:108E9000DB8AC8010E94088B2091352B30E080913D
:108EA0004C0290E0FC01EE0FFF1FE80FF91F2C9D14
:108EB000D0012D9DB00D3C9DB00D1124EA0FFB1F7C
:108EC000EB5DFF4E608166956F71262F2F5FA05E70
:108ED000BF4EAC91A03619F4220F220F03C0A0336D
:108EE00009F4220FCE018F519E4F2A1729F462E117
:108EF00071E00E94C88906C070E06F5F7F4F4AE052
:108F00000E94468A8E010F511E4F87E292E0B801FF
:108F10000E94DB8AC8010E94088B28EEA22E21E065
:108F2000B22EAC0EBD1EC50162E172E00E94F28A53
:108F30009FEEC92E91E0D92ECC0EDD1EC60169E14F
:108F400072E00E94F28A86EFE82E81E0F82EEC0EA5
:108F5000FD1EC70160E272E00E94F28A8E0103509A
:108F60001E4FC80167E272E00E94F28AC501B60195
:108F7000A70198010E94C03AC8010E94088BC7014E
:108F80000E94088BC6010E94088BC5010E94088BB5
:108F900087E097E36FE041E00E94867D80914C027C
:108FA00090E02091352B30E0FC01EE0FFF1FE80F21
:108FB000F91F85E29DE0AC01249FC001259F900D23
:108FC000349F900D1124E80FF91FE95DFF4E808159
:108FD00087FF07C087E097E36EE879E00E945A8632
:108FE00016C187E097E366E171E00E9482870FC1B6
:108FF0008091AE029091AF02079721F480914101D8
:109000008130A9F08BE092E066E071E00E94FC897B
:10901000BC0184E092E00E94DB8ABC018DEF91E00C
:109020000E94DB8ABC0186EF91E00E94DB8A80917E
:10903000AE029091AF02079771F49091BB038091BB
:109040004101981741F480912D01882321F48091EA
:10905000EC018823A1F187E097E360E040E00E9403
:10906000867D87E097E36DE779E00E945A868091DC
:10907000EF01E82FF0E0EE0FFF1FED51FD4F65917E
:1090800074918E010F5F1F4FC8010E941908E09173
:10909000EF01F0E0E25DFE4F87E097E3608140E0A2
:1090A0000E94867D87E097E3B8010E9482878091C5
:1090B000BB038093410110922D011092EC0180912D
:1090C000352B90E025E23DE0829FF001839FF00D7B
:1090D000929FF00D1124E15EFF4E8081E82FF0E0B9
:1090E000EE0FFF1FED50FD4F659174917E010894C6
:1090F000E11CF11CC7010E9419088E010C5F1D4F75
:10910000C801B7010E94C88982E192E0B8010E94BB
:10911000DB8AC8010E94088B8091F535E82FF0E0CA
:10912000EE0FFF1FEF58FC4F65917491C7010E942D
:1091300019088E01055F1D4FC801B7010E94C8893B
:1091400089E192E0B8010E94DB8AC8010E94088B85
:109150008E010E5E1D4F60915E0170E063507040A5
:10916000C8014AE00E94468A80E292E0B8010E946B
:10917000DB8AC8010E94088B8E01075E1D4FC80163
:1091800060E071E00E94C88987E292E0B8010E9425
:10919000DB8AC8010E94088BF0E2AF2EF2E0BF2EFE
:1091A000AC0EBD1EC50162E172E00E94F28AE7E2E8
:1091B000CE2EE2E0DE2ECC0EDD1EC60169E172E0AD
:1091C0000E94F28A7EE2E72E72E0F72EEC0EFD1E80
:1091D000C70160E272E00E94F28A8E010B5C1D4FB3
:1091E000C80167E272E00E94F28AC501B601A701D8
:1091F00098010E94C03AC8010E94088BC7010E94D2
:10920000088BC6010E94088BC5010E94088B87E06D
:1092100090E00C943E518091AE029091AF0206977F
:10922000A9F08BE092E066E071E00E94FC89BC014D
:1092300084E092E00E94DB8ABC018DEF91E00E9405
:10924000DB8ABC0186EF91E00E94DB8AE091E23686
:10925000F0E0EC54F94C928980912D37981771F019
:1092600084E092E066E071E00E94FC89E091E236E1
:10927000F0E0EC54F94C828980932D378091AE0256
:109280009091AF02069741F480912D01882321F43B
:109290008091EC018823B1F187E097E360E040E042
:1092A0000E94867D87E097E36CE679E00E945A860B
:1092B0008091EF01E82FF0E0EE0FFF1FED55FD4F1D
:1092C000659174918E010F5F1F4FC8010E941908AC
:1092D000E091EF01F0E0E25DFE4F87E097E360810F
:1092E00040E00E94867D87E097E3B8010E94828774
:1092F00086E090E09093AF028093AE0210922D0131
:109300001092EC01E091E236F0E0EC54F94C8081EF
:10931000E82FF0E0EE0FFF1FEB5DFC4F65917491BD
:109320007E010894E11CF11CC7010E9419088E01FE
:10933000045C1D4F6091E23670E06F5F7F4FC801A3
:109340004AE00E94468A82E192E0B8010E94DB8AEC
:10935000C8010E94088B8E010D5B1D4FC801B7012B
:109360000E94C88989E192E0B8010E94DB8AC801A5
:109370000E94088B8091E236E82FF0E0EC54F94C23
:1093800082899E01265B3D4F882331F0C90160E050
:1093900070E00E94C88908C0628170E06F5F7F4FF3
:1093A000C9014AE00E94468A8E01065B1D4F80E299
:1093B00092E0B8010E94DB8AC8010E94088B8E01EE
:1093C0000F5A1D4FE091E236F0E0EE0FFF1FEE0F57
:1093D000FF1FE854F94C608171818281938120E004
:1093E00030E048EC52E40E94CC8C0E94EA8B9B0156
:1093F000AC01C801622F4AE00E94778A87E292E0BE
:10940000B8010E94DB8AC8010E94088B38E5A32EB0
:1094100032E0B32EAC0EBD1EC50162E172E00E94C7
:10942000F28A2FE5C22E22E0D22ECC0EDD1EC6011E
:1094300069E172E00E94F28A96E6E92E92E0F92E46
:10944000EC0EFD1EC70160E272E00E94F28A8E01FE
:1094500003591D4FC80167E272E00E94F28AC501FC
:10946000B601A70198010E94C03AC8010E94088B6A
:10947000C7010E94088BC6010E94088BC5010E948B
:10948000088BE091E236F0E0EC54F94C82898823B5
:1094900009F4F8C60E94D839F5C68091AE029091C1
:1094A000AF020997A9F08BE092E066E071E00E94BC
:1094B000FC89BC0184E092E00E94DB8ABC018DEF54
:1094C00091E00E94DB8ABC0186EF91E00E94DB8A7A
:1094D00087E097E360E040E00E94867D8091B102E2
:1094E0002091AE023091AF02803109F044C02930A2
:1094F000310569F480912D01882349F480912B373F
:10950000803129F48091EC01882309F475C087E04B
:1095100097E36BE579E00E945A868091EF01E82F8E
:10952000F0E0EE0FFF1FED53FD4F659174918E013A
:109530000F5F1F4FC8010E941908E091EF01F0E092
:10954000E25DFE4F87E097E3608140E00E94867D08
:1095500087E097E3B8010E94828789E090E09093CA
:10956000AF028093AE021092EC0110922D0180E1C7
:1095700080932B3741C02930310561F480912D0152
:10958000882341F480912B37803121F08091EC01C8
:10959000882391F187E097E36AE479E00E945A8694
:1095A0008091EF01E82FF0E0EE0FFF1FE554FD4F33
:1095B000659174918E010F5F1F4FC8010E941908B9
:1095C000E091EF01F0E0E25DFE4F87E097E360811C
:1095D00040E00E94867D87E097E3B8010E94828781
:1095E00089E090E09093AF028093AE021092EC017C
:1095F00010922D0110922B372091352B30E04091A5
:10960000B102C42EDD2480914C0290E0DC01AA0F4F
:10961000BB1FA80FB91F84EC90E0C89EB001C99E83
:10962000700DD89E700D11246A0F7B1F85E29DE09E
:10963000289F7001299FF00C389FF00C11246E0DAB
:109640007F1DFB01E352FC4F8080869486948694B4
:109650004031F1F4FD01EE0DFF1DDF01AB5DBF4EAA
:109660009C91929596959695937011968C91877092
:10967000880F880F892BA82EBB2460EF7FEFA60EE2
:10968000B71EEA5DFF4E908096949694969419C00A
:10969000FB01E452FC4F2081922F9295969596956E
:1096A000937081818770880F880F892BA82EBB2427
:1096B00080EF9FEFA80EB91E922E969496949FE08D
:1096C00099228E010C581D4FEFE5FBE2CE0EDF1EF6
:1096D000F601608170E06F5F7F4FC8014AE00E9431
:1096E000468ACE0185589D4FB8010E94FD8A80911F
:1096F0003A2B882311F460E201C06EE7ABE7CA2E73
:10970000A2E0DA2ECC0EDD1EC6010E9480898C01FB
:10971000F2E8EF2EF2E0FF2EEC0EFD1EE091B1021A
:10972000F0E0E25BF44D608170E06F5F7F4FC70156
:109730004AE00E94468AC801B7010E949189BC0193
:109740008E0107571D4FC8010E94F28A82E192E004
:10975000B8010E94DB8AC8010E94088BC7010E94E1
:10976000088BC6010E940E8BCE018C589D4F0E9423
:10977000088BB7FC30C0E7E9CE2EE2E0DE2ECC0E3F
:10978000DD1EC60168E171E00E94E28970E9E72E02
:1097900072E0F72EEC0EFD1EC701B5014AE00E94F3
:1097A000468AC601B7010E949189BC018E0102560A
:1097B0001D4FC8010E94F28A89E192E0B8010E941F
:1097C000DB8AC8010E94088BC7010E94088BC60172
:1097D0000E940E8B10C08E010B551D4FC801B501A4
:1097E0004AE00E94468A89E192E0B8010E94DB8A41
:1097F000C8010E94088BE92DF0E0EE0FFF1FEB5F20
:10980000FC4F659174918E010F5F1F4FC8010E943C
:10981000190880E292E0B8010E94FC892091352B62
:1098200030E080914C0290E0FC01EE0FFF1FE80F4A
:10983000F91F85E29DE0289FD001299FB00D389F38
:10984000B00D1124EA0FFB1FEB5DFF4E60816695A2
:109850006F71262F2F5FA05EBF4EAC91A03619F41A
:10986000220F220F03C0A03309F4220F8091B1020E
:109870008031E1F4CE0184559D4F2A1729F462E12D
:1098800071E00E94C88906C070E06F5F7F4F4AE0B8
:109890000E94468A8E0104551D4F87E292E0B8016E
:1098A0000E94DB8AC8010E94088B51C041ECC42E83
:1098B00042E0D42ECC0EDD1E882041F4C6016AE1C0
:1098C00071E00E94C889EE24FF2428C03AEBE32E01
:1098D00032E0F32EEC0EFD1EC7016EE171E00E9436
:1098E000E2898E010D541D4FE82DF0E0EC5CFE4F37
:1098F000608180E891E070E00E946E8DC8014AE0CE
:109900000E94468AC701B8010E949189BC01C60124
:109910000E94F28AEE24E394FF24F3948E010F5305
:109920001D4F87E292E0B8010E94DB8AC8010E94C5
:10993000088BFF2029F0CE018D549D4F0E94088B8B
:10994000EE2029F0CE0186549D4F0E940E8B28EC0C
:10995000A22E22E0B22EAC0EBD1EC50162E172E065
:109960000E94F28A9FECC92E92E0D92ECC0EDD1E09
:10997000C60169E172E00E94F28A86EDE82E82E07B
:10998000F82EEC0EFD1EC70160E272E00E94F28A22
:109990008E0103521D4FC80167E272E00E94F28AF5
:1099A000C501B601A70198010E94C03AC8010E94F2
:1099B000088BC7010E94088BC6010E94088BC50155
:1099C0000E94088B8091B102803109F05BC487E06E
:1099D00097E36FE041E00E94867D80914C0290E029
:1099E0002091352B30E0FC01EE0FFF1FE80FF91F2F
:1099F00085E29DE0AC01249FC001259F900D349F1E
:109A0000900D1124E80FF91FE95DFF4E808187FF5B
:109A100005C087E097E368E479E049C087E097E311
:109A200066E171E00E9482872DC485E090E090930A
:109A3000AF028093AE0287E097E360E040E00E94CF
:109A4000867D87E097E367E379E00E945A8687E0A6
:109A500097E360E041E00E94867D0E94763987E0CE
:109A600097E362E041E00E94867D8091CA368823B8
:109A700029F087E097E363E379E004C087E097E3A8
:109A800060E379E00E945A8687E097E36AE041E06C
:109A90000E94867D8091F202882329F087E097E377
:109AA0006CE279E004C087E097E369E279E00E9424
:109AB0005A86E8C38091AE029091AF020197A9F057
:109AC0008BE092E066E071E00E94FC89BC0184E0DA
:109AD00092E00E94DB8ABC018DEF91E00E94DB8A5C
:109AE000BC0186EF91E00E94DB8A8091AE029091EA
:109AF000AF02019741F480912D01882321F48091D8
:109B0000EC01882381F187E097E360E040E00E9468
:109B1000867D87E097E368E179E00E945A8680912C
:109B2000EF01E82FF0E0EE0FFF1FED52FD4F6591C2
:109B300074918E010F5F1F4FC8010E941908E091B8
:109B4000EF01F0E0E25DFE4F87E097E3608140E0E7
:109B50000E94867D87E097E3B8010E948287109279
:109B60002D011092EC018E010C511D4F6091F533C7
:109B700070E06F5F7F4FC8014AE00E94468A82E131
:109B800092E0B8010E94DB8AC8010E94088B8E0116
:109B900005511D4F6091F6337091F7336F5F7F4F22
:109BA000C8014AE00E94468A89E192E0B8010E9419
:109BB000DB8AC8010E94088BB2EFCB2EB2E0DB2E0D
:109BC000CC0EDD1EE091F633F091F733EC50FC4CF7
:109BD000618562956F706F5BC6010E94A98AE12C56
:109BE000A3E0FA2EEC0EFD1EC701B6010E94FD8A0D
:109BF000E091F633F091F733EC50FC4C21858E0167
:109C000007501D4F622F70E06F5F7F4F822F82954C
:109C10008F7090E0F4E0880F991FFA95E1F7681BC8
:109C2000790BC8014AE00E94468AC701B8010E9428
:109C30009189BC0180E292E00E94DB8AC8010E9407
:109C4000088BC7010E940E8BC6010E94088B8EE212
:109C500092E060E272E00E94DB8A88E08093F0018B
:109C60008E01095F1C4F6091FA337091FB336F5F77
:109C70007F4FC8014AE00E94158A87E292E0B8014E
:109C80000E94DB8AC8010E94088BEEE0AE2EE3E062
:109C9000BE2EAC0EBD1EC50162E172E00E94F28ACA
:109CA00075E1C72E73E0D72ECC0EDD1EC60169E12B
:109CB00072E00E94F28A6CE1E62E63E0F62EEC0E72
:109CC000FD1EC70160E272E00E94F28A8E010D5D06
:109CD0001C4FC80167E272E00E94F28AC501B6011A
:109CE000A70198010E94C03AC8010E94088BC701D1
:109CF0000E94088BC6010E94088BC5010E94088B38
:109D000081E090E0BBC28091AE029091AF02892BBE
:109D1000C9F480912D018823A9F48091EC01882356
:109D200089F48091303790E02091F6333091F73309
:109D30008217930739F490912F378091F533981754
:109D400009F4ADC087E097E360E040E00E94867DC3
:109D50000E94763987E097E360E040E00E94867DCC
:109D600087E097E36BE079E00E945A866091F533D3
:109D700070E06F5F7F4F87E097E34AE050E00E941A
:109D80006F878091F53380932F3787E097E360E00A
:109D900041E00E94867D0E94763987E097E360E08B
:109DA00041E00E94867D87E097E366E079E00E94CB
:109DB0005A868091F633809330376091F6337091F4
:109DC000F73377FF02C060E070E06F5F7F4F87E09E
:109DD00097E34AE050E00E946F8787E097E368E0EE
:109DE00041E00E94867D87E097E360E079E00E9491
:109DF0005A865AE2C52E53E0D52ECC0EDD1EE091D8
:109E0000F633F091F733EC50FC4C618562956F703E
:109E10006F5BC6010E94A98A48E3E42E43E0F42E5A
:109E2000EC0EFD1EC701B6010E94FD8AE091F633DB
:109E3000F091F733EC50FC4C21858E010F5C1C4FE8
:109E4000622F70E06F5F7F4F822F82958F7090E05E
:109E500034E0880F991F3A95E1F7681B790BC80128
:109E60004AE00E94468AC701B8010E949189BC015C
:109E700080E292E00E94DB8AC8010E94088BC70141
:109E80000E940E8BC6010E94088B87E097E360E278
:109E900072E00E94238810922D011092EC01109222
:109EA000AF021092AE02EEC18091AE029091AF026D
:109EB0000D97A9F08BE092E066E071E00E94FC89CA
:109EC000BC0184E092E00E94DB8ABC018DEF91E04E
:109ED0000E94DB8ABC0186EF91E00E94DB8A8091C0
:109EE000AE029091AF020D9741F480912D0188232D
:109EF00021F48091EC01882381F110922D011092C0
:109F0000EC0187E097E360E040E00E94867D87E017
:109F100097E36FEE78E00E945A868091EF01E82F78
:109F2000F0E0EE0FFF1FE552FD4F659174918E0139
:109F30000F5F1F4FC8010E941908E091EF01F0E088
:109F4000E25DFE4F87E097E3608140E00E94867DFE
:109F500087E097E3B8010E9482878E01015C1C4F65
:109F6000C801609135364AE00E94778A82E192E02A
:109F7000B8010E94DB8AC8010E94088B8E010A5B2F
:109F80001C4FC801609136364AE00E94778A89E109
:109F900092E0B8010E94DB8AC8010E94088B8E0102
:109FA000035B1C4FC801609137364AE00E94778AF4
:109FB00080E292E0B8010E94DB8AC8010E94088B0F
:109FC0008E010C5A1C4FC801609138364AE00E943D
:109FD000778A87E292E0B8010E94DB8AC8010E947A
:109FE000088B9BE5A92E93E0B92EAC0EBD1EC501D2
:109FF00062E172E00E94F28A82E6C82E83E0D82EE7
:10A00000CC0EDD1EC60169E172E00E94F28A09E60B
:10A01000E02E03E0F02EEC0EFD1EC70160E272E0C0
:10A020000E94F28A8E0100591C4FC80167E272E05B
:10A030000E94F28AC501B601A70198010E94C03AA8
:10A04000C8010E94088BC7010E94088BC6010E94AC
:10A05000088BC5010E94088B8DE090E00FC18091B4
:10A06000AE029091AF020E9729F48091EC01882303
:10A0700009F46CC01092EC0187E097E360E040E0E7
:10A080000E94867D87E097E36EED78E00E945A8615
:10A0900087E097E360E041E00E94867D0E94763988
:10A0A00087E097E362E041E00E94867D60914C0288
:10A0B00070E06F5F7F4F87E097E34AE050E00E94D7
:10A0C0006F8787E097E36AE041E00E94867D809198
:10A0D0004C0290E02091B10230E04091352B50E0ED
:10A0E000FC01EE0FFF1FE80FF91F84EC90E0BC01AC
:10A0F000269FC001279F900D369F900D1124E80FD9
:10A10000F91F85E29DE09C01429FC001439F900D95
:10A11000529F900D1124E80FF91FE252FC4F60810D
:10A120006F7770E0882777FD8095982F0E94188CB4
:10A130002AE037ED43E25DE30E94CC8CAB01BC0129
:10A1400087E097E322E030E00E94208880914C0273
:10A1500090E02091B10230E04091352B50E0FC01BD
:10A16000EE0FFF1FE80FF91FA4ECEA2EF12C2E9D35
:10A17000C0012F9D900D3E9D900D1124E80FF91FF9
:10A1800005E21DE0409FC001419F900D509F900D42
:10A190001124E80FF91FE252FC4F20812F7730E0A5
:10A1A00080912C3790E02817390709F465C087E0C3
:10A1B00097E36AE041E00E94867D80914C0290E046
:10A1C0002091B10230E04091352B50E0FC01EE0FC0
:10A1D000FF1FE80FF91F2E9DC0012F9D900D3E9D82
:10A1E000900D1124E80FF91F409FC001419F900D71
:10A1F000509F900D1124E80FF91FE252FC4F60812F
:10A200006F7770E0882777FD8095982F0E94188CD3
:10A210002AE037ED43E25DE30E94CC8CAB01BC0148
:10A2200087E097E322E030E00E94208880914C0292
:10A2300090E02091B10230E04091352B50E0FC01DC
:10A24000EE0FFF1FE80FF91F2E9DC0012F9D900DEF
:10A250003E9D900D1124E80FF91F409FC001419FC2
:10A26000900D509F900D1124E80FF91FE252FC4F02
:10A2700080818F7780932C378EE090E09093AF02AF
:10A280008093AE02C158DC4F0FB6F894DEBF0FBE0C
:10A29000CDBFCF91DF911F910F91FF90EF90DF9095
:10A2A000CF90BF90AF909F908F9008959F92AF9264
:10A2B000BF92CF92DF92EF92FF920F931F93DF93A3
:10A2C000CF9300D000D00F92CDB7DEB78091460279
:10A2D000909147028230910561F10C9751F1809184
:10A2E000EF0190E061E070E00E940811282F80915A
:10A2F000460290914702049749F48091B10280315F
:10A3000029F4822F233030F082E004C0822F2430E1
:10A3100008F083E08093EF019091EF01809159372D
:10A32000981739F09093593781E080932D018093ED
:10A330002C018091F501882309F4B6C00091B10287
:10A340004091352B0031A1F4842F90E025E23DE0CF
:10A350008C01029FC001039F900D129F900D11244C
:10A360008E5D9F4E61E041E027E009EB13E01FC0E6
:10A3700010E084EC90E09C01029FC001039F900DCF
:10A38000129F900D112450E025E23DE0B901469F57
:10A390009001479F300D569F300D1124820F931F5F
:10A3A000055C144D81569B4F61E041E027E00E941F
:10A3B00064118091873682FD07C08091460290919A
:10A3C0004702029709F070C05091B1024091352BBD
:10A3D0005031A1F4242F30E085E29DE0289FF00168
:10A3E000299FF00D389FF00D1124EE53FC4FE05AD9
:10A3F000F34F8081E056FC4083831FC0242F30E060
:10A4000085E29DE0289FD001299FB00D389FB00DB7
:10A410001124252F30E084EC90E0289FF001299F43
:10A42000F00D389FF00D1124EA0FFB1FE156FB4F92
:10A430008081AE53BC4F13968C9320E030E004EC47
:10A4400010E065E27DE0FF24F3948091352B90E0ED
:10A45000209FF001219FF00D309FF00D1124DC01B1
:10A46000A69FC001A79F900DB69F900D1124E80FE5
:10A47000F91FE156FB4FDC01AE53BC4FAD014D5F00
:10A480005F4F13968C9113978083F901E55CF44D2F
:10A49000F0822F5F3F4F20313105B9F6FD01E05AC0
:10A4A000F34FDA018C9180838091F401882309F4C1
:10A4B000B8C00091B1024091352B0031A1F4842F36
:10A4C00090E025E23DE0FC01E29FC001E39F900D9A
:10A4D000F29F900D11248D5D9F4E61E040E023E0DE
:10A4E00009EB13E01FC010E084EC90E09C01029F98
:10A4F000C001039F900D129F900D112450E025E2A2
:10A500003DE0B901469F9001479F300D569F300DA9
:10A510001124820F931F055C144D82569B4F61E0FE
:10A5200040E023E00E9464118091873682FD07C0DD
:10A530008091460290914702029709F072C02091E3
:10A54000B1024091352B203169F450E085E29DE065
:10A55000489FF001499FF00D589FF00D1124ED5DCB
:10A56000FF4E19C050E030E084EC90E0289FF001ED
:10A57000299FF00D389FF00D112485E29DE0DC014C
:10A580004A9FC0014B9F900D5A9F900D1124E80FD8
:10A59000F91FE256FB4F208185E29DE0489FF001C4
:10A5A000499FF00D589FF00D1124EE53FC4F22836C
:10A5B00020E030E004EC10E065E27DE0FF24F3945D
:10A5C0008091352B90E0209FF001219FF00D309F6E
:10A5D000F00D1124AC01469FC001479F900D569F7E
:10A5E000900D1124E80FF91FE256FB4FDC01AE532A
:10A5F000BC4FAD014E5F5F4F12968C9112978083D6
:10A60000F901E55CF44DF0822F5F3F4F20313105B9
:10A61000B9F6FD01EF59F34FDA018C918083F09286
:10A62000B90380914602909147028630910509F462
:10A6300014C787309105A4F48230910571F18330FD
:10A6400091052CF4019711F00C948F6160C5833053
:10A65000910509F4D5C0049711F00C948F61C3C221
:10A660008930910511F40C949C5D8A30910554F465
:10A670008730910511F40C944C5B089711F00C9401
:10A680008F61BFC58C30910511F40C945B610D97FF
:10A6900011F00C948F610C94726180918D3682FF61
:10A6A0006AC08091352B90E0F5E2EF2EFDE0FF2EA1
:10A6B0008E9DF0018F9DF00D9E9DF00D1124EE53A7
:10A6C000FC4FD080CF0161E040E02FE308E31BE2C4
:10A6D0000E9464118091352B90E08E9DF0018F9D3A
:10A6E000F00D9E9DF00D1124EE53FC4F80818D15D1
:10A6F00091F120E030E064EC70E045E25DE011E0D3
:10A700008091352B90E0269FF001279FF00D369F1A
:10A71000F00D1124DC01A49FC001A59F900DB49FF2
:10A72000900D1124E80FF91FE456FB4FDC01AE53E6
:10A73000BC4F8C918083F901E55CF44D10832F5F51
:10A740003F4F20313105E1F6FD01E15AF34F8C9185
:10A7500080831093B9038091B102082F10E0025B4F
:10A76000144DF801F0808F2D90E061E070E00E94C0
:10A7700008110C94535E80914802837059F48091C3
:10A780003E0290913F0261E00E94EA1190933F02E5
:10A7900080933E0280913E0290913F024F9730F4A9
:10A7A0008EE190E090933F0280933E0280913E02C2
:10A7B00090913F028A3F910530F08AEF90E09093AC
:10A7C0003F0280933E0220913E0230913F028091F1
:10A7D0005637909157372817390711F40C948F6129
:10A7E00030935737209356370E94FC2681E08093A0
:10A7F0002C0180914802837009F471C50C948F611B
:10A800008091EF018130B9F0813038F08230E1F190
:10A81000833011F00C948F619DC180919B3683FD34
:10A8200002C00C94425E8091893682FF02C00C9473
:10A83000425E0C942B5E0091B1024091352B0031A9
:10A84000A1F4842F90E025E23DE0FC01E29FC001ED
:10A85000E39F900DF29F900D11248F5D9F4E61E05C
:10A8600040E02FE309EB13E077C210E084EC90E0C6
:10A870009C01029FC001039F900D129F900D112417
:10A8800050E025E23DE057C22091B1024091352BC6
:10A89000203171F4242F30E085E29DE0289FF00103
:10A8A000299FF00D389FF00D1124E05EFF4E19C076
:10A8B00030E050E084EC90E0289FF001299FF00DFB
:10A8C000389FF00D112485E29DE0DC014A9FC00114
:10A8D0004B9F900D5A9F900D1124E80FF91FE356DE
:10A8E000FB4F10811831A9F0193128F41C30A9F060
:10A8F0001031B1F410C0103341F0103619F010329D
:10A9000079F405C01092A4360BC081E007C082E044
:10A9100005C083E003C084E001C085E08093A436D5
:10A920008091A43661E00E943911863008F085E0FC
:10A930008093A43680913837882371F488E397E3B5
:10A940000E942286892B41F08091A436809355374E
:10A9500088E397E30E942C869091A4368091553726
:10A96000981711F40C948F619093553781E0809380
:10A970002C01E091B102E03119F48093B90304C0D5
:10A98000F0E0E55CF44D80838091A4368230A9F03C
:10A99000833028F4882351F0813011F509C08430C8
:10A9A000A1F0843060F08530D9F415C010E601C004
:10A9B00010E3EE24EFE1FE2E13C010E2FACF18E10F
:10A9C00074E0E72E6BE1F62E0BC010E158E0E52EA7
:10A9D00047E1F42E05C01CE03AE0E32E25E1F22E1B
:10A9E0008091B1026E2D4F2D0E943B138091B102D8
:10A9F000803191F48091352B90E025E23DE0829FFB
:10AA0000F001839FF00D929FF00D1124E05EFF4E48
:10AA1000812F60810E94EE0B2091B1024091352B75
:10AA2000203171F4242F30E085E29DE0289FF00171
:10AA3000299FF00D389FF00D1124E05EFF4E19C0E4
:10AA400030E050E084EC90E0289FF001299FF00D69
:10AA5000389FF00D112485E29DE09C01429FC001CA
:10AA6000439F900D529F900D1124E80FF91FE3565C
:10AA7000FB4F10838091913682FF70C15091B102DB
:10AA80004091352B5031A1F4242F30E085E29DE038
:10AA9000289FF001299FF00D389FF00D1124EE53EF
:10AAA000FC4FE25AF34F8081EE55FC4081831FC07A
:10AAB000242F30E085E29DE0289FD001299FB00D32
:10AAC000389FB00D1124252F30E084EC90E0289FB2
:10AAD000F001299FF00D389FF00D1124EA0FFB1FA4
:10AAE000E356FB4F8081AE53BC4F11968C9300E030
:10AAF00010E094ECA92EB12C85E2C82E8DE0D82E62
:10AB0000992493948091352B90E00A9DD0010B9D60
:10AB1000B00D1A9DB00D11248C9DF0018D9DF00D8E
:10AB20009C9DF00D1124AE0FBF1FA356BB4FEE53DB
:10AB3000FC4F81818C93802F6E2D4F2D0E943B13F3
:10AB4000F801E55CF44D90820F5F1F4F0031110555
:10AB5000C9F65CC280919B3683FFD2C24091B1029C
:10AB60008091352B90E025E23DE0829FF001839FAC
:10AB7000F00D929FF00D1124EE53FC4FE40FF11DE8
:10AB80008781882309F4A1C240E050E0A4ECB0E042
:10AB900065E27DE08091B10290E02091352B30E0BC
:10ABA000FA01EE0FFF1FE40FF51F8C010A9FC00191
:10ABB0000B9F900D1A9F900D1124E80FF91F269FEF
:10ABC000C001279F900D369F900D1124E80FF91FAB
:10ABD000E452FC4F8081826080834F5F5F4F40343E
:10ABE0005105C1F672C20091B1026091EF010031CE
:10ABF00009F065C08091352B90E025E23DE0829F11
:10AC0000F001839FF00D929FF00D1124E15EFF4E45
:10AC10008081613051F1613028F0623011F00C9484
:10AC20008F6138C061E00E943911482F893008F0E7
:10AC300048E080915437481739F04093543781E009
:10AC40008093B90380932C018091352B90E025E20D
:10AC50003DE0829FF001839FF00D929FF00D112443
:10AC6000E15EFF4E40830C948F618091F53561E089
:10AC70000E943911982F8C3008F09BE09093F535A5
:10AC800080915337981711F40C948F619093533738
:10AC90000C946E6180915E0161E00E943911982FE1
:10ACA000883008F097E090935E01809152379817B2
:10ACB00011F40C948F61909352370C946E61613053
:10ACC00051F1613040F0623009F44CC0633011F052
:10ACD0000C948F61B5C180919B3683FF71C58091C3
:10ACE000893682FD6DC590E080913A2B882309F466
:10ACF00091E090933A2B992351F0E091B102F0E06A
:10AD0000DF01A15AB44D8C91E25BF44D808381E068
:10AD100080932C0155C510E084EC90E09C01029FCB
:10AD2000C001039F900D129F900D11242091352B8F
:10AD300030E045E25DE0B901649F9001659F300D10
:10AD4000749F300D1124820F931F055C144D84569F
:10AD50009B4F61E040E02FE30E9464110E94E625D2
:10AD60000C948F61402F50E02091352B30E084EC23
:10AD700090E0489FF001499FF00D589FF00D11247D
:10AD800085E29DE0DC012A9FC0012B9F900D3A9F38
:10AD9000900D1124E80FF91FE356FB4F1081183175
:10ADA000A9F0193128F41C30A9F01031B1F410C009
:10ADB000103341F0103619F0103279F405C01092BA
:10ADC000A4360BC081E007C082E005C083E003C069
:10ADD00084E001C085E08093A4368091A43661E0D0
:10ADE0000E943911863008F085E08093A436809166
:10ADF0004037882371F480E497E30E942286892BF0
:10AE000041F08091A4368093513780E497E30E940B
:10AE10002C869091A43680915137981711F40C9498
:10AE20008F619093513781E080932C01E091B102C2
:10AE3000E03119F48093B90304C0F0E0E55CF44D0F
:10AE400080838091A4368230A9F0833028F488234F
:10AE500051F0813011F509C08430A1F0843060F0E8
:10AE60008530D9F415C010E601C010E3EE24EFE1FF
:10AE7000FE2E13C010E2FACF18E174E0E72E6BE16A
:10AE8000F62E0BC010E158E0E52E47E1F42E05C088
:10AE90001CE03AE0E32E25E1F22E8091B1026E2D06
:10AEA0004F2D0E943B138091B102803191F480912B
:10AEB000352B90E025E23DE0829FF001839FF00D6D
:10AEC000929FF00D1124E05EFF4E812F60810E9461
:10AED000EE0B2091B1024091352B203171F4242FDB
:10AEE00030E085E29DE0289FF001299FF00D389F1A
:10AEF000F00D1124E05EFF4E19C030E050E084EC0C
:10AF000090E0289FF001299FF00D389FF00D11244B
:10AF100085E29DE09C01429FC001439F900D529F9E
:10AF2000900D1124E80FF91FE356FB4F1083809119
:10AF3000913682FF13CF5091B1024091352B5031A1
:10AF4000A1F4242F30E085E29DE0289FF001299FA5
:10AF5000F00D389FF00D1124EE53FC4FE25AF34FE1
:10AF60008081EE55FC4081831FC0242F30E085E2B4
:10AF70009DE0289FD001299FB00D389FB00D11246E
:10AF8000252F30E084EC90E0289FF001299FF00D00
:10AF9000389FF00D1124EA0FFB1FE356FB4F808111
:10AFA000AE53BC4F11968C9300E010E094ECA92EA8
:10AFB000B12C85E2C82E8DE0D82E992493948091EF
:10AFC000352B90E00A9DD0010B9DB00D1A9DB00D60
:10AFD00011248C9DF0018D9DF00D9C9DF00D112490
:10AFE000AE0FBF1FA356BB4FEE53FC4F81818C9316
:10AFF000802F6E2D4F2D0E943B13F801E55CF44D20
:10B0000090820F5F1F4F00311105C9F680E16E2D50
:10B010004F2D0E943B138091352B90E025E23DE0BF
:10B02000829FF001839FF00D929FF00D1124EE534B
:10B03000FC4F8181E25AF34F80839092B9038ECE08
:10B0400080919B3683FF5CC08091352B90E025E298
:10B050003DE0829FF001839FF00D929FF00D11243F
:10B06000EE53FC4FE00FF11D8781882371F140E022
:10B0700050E0A4ECB0E065E27DE08091B10290E0A8
:10B080002091352B30E0FA01EE0FFF1FE40FF51F82
:10B090008C010A9FC0010B9F900D1A9F900D1124E7
:10B0A000E80FF91F269FC001279F900D369F900D36
:10B0B0001124E80FF91FE452FC4F808182608083E5
:10B0C0004F5F5F4F40345105C1F68091352B90E0C2
:10B0D0004091B10225E23DE0829FF001839FF00D97
:10B0E000929FF00D1124EE53FC4FE40FF11D90E000
:10B0F0008781882309F491E0978381E080932C0174
:10B1000081EB92E061E040E020E10C948B61809162
:10B11000B302E091F633F091F733EC50FC4C91859B
:10B12000981741F081E08093ED0180914602809371
:10B13000EE0102C01092ED018091EF01813091F09B
:10B14000813038F0823029F1833011F00C948F6116
:10B1500041C085EF93E361E040E02FE000EF15E3AD
:10B160000C948D6180919B3682FF05C086EF93E33E
:10B170006AE070E004C086EF93E361E070E040E0D5
:10B1800050E023EF31E000E010E00E949C120C94AC
:10B190008F618091F6339091F73383509C4C61E03E
:10B1A00040E02FE701EF15E30E94641180919B3688
:10B1B00082FD02C00C948F61E091F633F091F73379
:10B1C000EC50FC4C81858093B50281E08093362B56
:10B1D0000C948F6180919B3682FF05C08AEF93E3C8
:10B1E0006AE070E004C08AEF93E361E070E040E061
:10B1F00050E023EF31E000E010E00E9427120C94B1
:10B200008F618091F101813029F0823011F00C942E
:10B210008F6183C08091EF01813089F1813040F0EE
:10B22000823009F46BC0833011F00C948F616CC0D4
:10B2300080914802837061E00E943911582F537049
:10B24000533009F452E0852F8370409148024C7FBF
:10B25000482B40934802252F30E08091503790E0F2
:10B260002817390711F40C948F61509350374460BC
:10B270004093480281E0809337020C946F61809183
:10B2800040029091410261E00E94EA119C018E31DE
:10B29000910518F42EE130E005C08B3F910510F0C8
:10B2A0002AEF30E0309341022093400280914F37E3
:10B2B00090E02817390711F40C948F6120934F37D1
:10B2C0000E94FC26809140029091410290933F029F
:10B2D00080933E0281E08093370280932C0180911D
:10B2E000C636882319F080E00E94C6168091C736C2
:10B2F000882311F40C948F6181E016C18DE392E0F4
:10B3000061E042E02AE005C08AE392E061E040E0CB
:10B3100026E007E312E00C948D618091EF0181300B
:10B3200061F0813038F0823071F0833011F00C948C
:10B330008F614EC086E392E002C085E392E061E057
:10B3400040E021E0E6CF80914402909145020090D8
:10B35000B40202C0969587950A94E2F781708983BA
:10B36000CE01019661E040E021E007E312E00E9497
:10B37000641189814091B4022091440230914502C8
:10B38000882391F081E090E0A0E0B0E004C0880F55
:10B39000991FAA1FBB1F4A95D2F7282B392B309330
:10B3A000450220934402BBC781E090E0A0E0B0E0FA
:10B3B00004C0880F991FAA1FBB1F4A95D2F780951A
:10B3C0009095822393239093450280934402A7C7CC
:10B3D00080914202909143020090B40202C096957F
:10B3E00087950A94E2F781708983CE01019661E026
:10B3F00040E021E007E312E00E946411898140915E
:10B40000B4022091420230914302882391F081E0FE
:10B4100090E0A0E0B0E004C0880F991FAA1FBB1FF6
:10B420004A95D2F7282B392B3093430220934202BE
:10B4300076C781E090E0A0E0B0E004C0880F991FDB
:10B44000AA1FBB1F4A95D2F780959095822393231C
:10B45000909343028093420262C78091EF01813052
:10B4600071F0813030F0823099F0833009F057C7A5
:10B470005EC082EE96E361E040E021E04CC780913F
:10B48000E23690E08C54994C61E040E024E030C01A
:10B4900080919B3683FF11C08091E236E82FF0E067
:10B4A000EC54F94C90E08289882309F491E0928B66
:10B4B00081E08093E33680932C018091E236282F3F
:10B4C00030E0F901EC54F94C82898823A1F4809191
:10B4D00087362E5F3F4F82FF05C0C9018C54994CBF
:10B4E0006AE004C0C9018C54994C61E040E02EEF41
:10B4F00003EE16E312C7813009F011C7F488C901C1
:10B500008853994C61E040E027E003EE16E30E9487
:10B5100064119091E236E92FF0E0EC54F94C848903
:10B520008F1509F4FCC6892F0E94C616F8C68091B3
:10B5300087360091E23682FF11C010E0000F111F24
:10B54000000F111F0854194CD8016D917D918D91F8
:10B550009C912DEC3CEC4CEC5DE310C010E0000F36
:10B56000111F000F111F0854194CD8016D917D91C6
:10B570008D919C912AE037ED43E25CE30E94DA1260
:10B58000F80160837183828393838091E236C82EB1
:10B59000DD24F601EE0FFF1FEE0FFF1FE854F94CFC
:10B5A000E080F18002811381C801B70120E030E022
:10B5B00040E050E00E94798B88235CF40F2EF0E08D
:10B5C000EF2EF0E0FF2EF0E00F2FF0E01F2FF02D18
:10B5D00014C0C801B70120E030E040E85FE30E94FA
:10B5E000C88C181654F40F2EF0E0EF2EF0E0FF2E6A
:10B5F000F0E80F2FFFE31F2FF02DCC0CDD1CCC0C3F
:10B60000DD1C28EB36E3C20ED31ED601ED92FD926F
:10B610000D931C931397E091E236F0E0EE0FFF1FBD
:10B62000EE0FFF1FE20FF31FE080F1800281138114
:10B63000C801B70120914B3730914C3740914D37BD
:10B6400050914E370E94798B882369F0E0924B37F6
:10B65000F0924C3700934D3710934E3781E0809332
:10B66000E33680932C0180919B3683FF58C6E0918E
:10B67000E236F0E0EE0FFF1FEE0FFF1FE854F94C2B
:10B6800080E090E0A0E8BFE380839183A283B3834E
:10B6900081E08093E33623C62091352B30E0809102
:10B6A0004C0290E0DC01AA0FBB1FA80FB91F85E276
:10B6B0009DE0F901E89F9001E99F300DF89F300D62
:10B6C0001124A20FB31FFD01E95DFF4E8081F82F09
:10B6D000FF70FD83829587708983215E3F4EF9015B
:10B6E0001081AB5DBF4E0C9106950F718091BB032D
:10B6F000813009F053C08091EF01813049F18130F0
:10B7000020F0823009F04AC035C0812F61E00E94EC
:10B710003911182F893008F018E080914A3718172E
:10B7200039F010934A3781E08093B90380932C015C
:10B730008091352B90E025E23DE0829FF001839FD0
:10B74000F00D929FF00D1124E15EFF4E108326C094
:10B750008091F53561E00E943911982F8C3008F006
:10B760009BE09093F535809149379817B9F0909305
:10B77000493711C080915E0161E00E943911982F14
:10B78000883008F097E090935E01809148379817D1
:10B7900029F09093483781E080932C018091BB037E
:10B7A000882309F0BCC58091EF018130E9F0813038
:10B7B00038F0823009F41CC1833009F0B0C599C15A
:10B7C00080913A2B882309F0AAC58091B102082FF5
:10B7D00010E0025B144DD801FC908F2D61E00E94B7
:10B7E0003911F801808361C223B122702093FE35A4
:10B7F00093B191709093FF35222371F480910036BC
:10B80000882351F0992321F4EE24EA94FE2C06C0FB
:10B8100071E0E72EF12C02C0EE24FF2420930036C5
:10B82000E114F10409F47BC58091873682FFAFC033
:10B830008091352B90E025E23DE0829FF001839FCF
:10B84000F00D929FF00D1124EF5DFF4E008180916D
:10B85000893682FD02C040E02EC080915E2B81308F
:10B8600061F0813028F0823079F08330D9F413C050
:10B870000031C0F040E00FE016C0003218F040E1A7
:10B880000FE111C040E10FC0003318F040E20FE2B9
:10B890000AC040E208C0003418F040E30FE303C0E0
:10B8A00040E301C040E080914C02841710F008177B
:10B8B00010F440934C022091352B30E0812F90E022
:10B8C000FC01EE0FFF1FE80FF91FEE0FFF1FEE0F39
:10B8D000FF1FBF0168547C4F542FAA24A394BB249C
:10B8E000B39485E29DE0289FD001299FB00D389F39
:10B8F000B00D1124E355FC4FE491CE2EDD24FB0165
:10B900008491682F70E029C0252F30E0F901EE0FF7
:10B91000FF1FE20FF31FEA0FFB1FE95DFF4EE081FF
:10B920008E2F8F7090E08C159D0521F4E295E770C5
:10B9300009F4AA248617970779F4F901EE0FFF1F7F
:10B94000E20FF31FEA0FFB1FE95DFF4E8081829536
:10B950008770873009F4BB245F5F0517A8F6142FA2
:10B9600013C0F1E0EF16F10419F4BB2041F40BC051
:10B970002FEFE2162FEFF20631F4AA2021F0812FEB
:10B98000B7010E94CF0C1F5F011758F72DC080919F
:10B99000913683FF24C020E030E065E27DE04D81F8
:10B9A0004F708091352B90E0F901EE0FFF1FE20FF1
:10B9B000F31FDC01A69FC001A79F900DB69F900DBD
:10B9C0001124E80FF91FE95DFF4E8081807F842BF1
:10B9D00080832F5F3F4F2034310519F705C08091D8
:10B9E0004C02B7010E94CF0C81E08093B90377C469
:10B9F0008091913683FF4EC023B122702093FE3593
:10BA000093B191709093FF35222361F480910036B9
:10BA1000882341F0992319F48FEF9FEF05C081E04F
:10BA200090E002C080E090E0209300368093EC022A
:10BA30008823C9F140E050E065E27DE08091352B3C
:10BA400090E0FA01EE0FFF1FE40FF51F8C01069F37
:10BA5000C001079F900D169F900D1124E80FF91F4C
:10BA6000E95DFF4E2081822F82958F709091EC02CC
:10BA7000890F87708295807F2F78282B20834F5FD6
:10BA80005F4F40345105D1F681E08093B903809334
:10BA90002C0109C0CE01019661E040E027E009EBEE
:10BAA00013E00E94641180919B3683FF02C083E003
:10BAB000898380914C0290E02091352B30E0FC018D
:10BAC000EE0FFF1FE80FF91F85E29DE0AC01249FF8
:10BAD000C001259F900D349F900D1124E80FF91F90
:10BAE000E95DFF4E998197709295907F80818F7864
:10BAF000DFC3802F0E94911120914C0230E04091D1
:10BB0000352B50E0F901EE0FFF1FE20FF31F25E286
:10BB10003DE0B901469F9001479F300D569F300D83
:10BB20001124E20FF31FEB5DFF4E8F71880F9081A0
:10BB3000917C982B9083F3C31C822091B102409199
:10BB4000352B80914C02203199F590E0242F30E084
:10BB5000FC01EE0FFF1FE80FF91F85E29DE0D90100
:10BB6000A89F9001A99F300DB89F300D1124E20FBE
:10BB7000F31FDF01AB5DBF4E4C91942F92959695CC
:10BB80009695937011968C918770880F880F892BEA
:10BB90008983205E3F4ED9013C91EA5DFF4E808152
:10BBA0008695869586958A83842F86958F7141C068
:10BBB00090E030E050E0FC01EE0FFF1FE80FF91FAE
:10BBC00084EC90E08901089F9001099F300D189F37
:10BBD000300D1124E20FF31F85E29DE0BA01689F4A
:10BBE000A001699F500D789F500D1124E40FF51F9F
:10BBF000DF01A452BC4F9C91692F629566956695B2
:10BC0000637011968C918770880F880F862B8983BB
:10BC1000240F351F23563B4FD9013C91969596959D
:10BC20009F709A83E352FC4F808186958695869516
:10BC30008B839091EF01913009F44CC0913038F032
:10BC4000923009F478C1933009F069C361C28091E0
:10BC50009B3683FF17C090E080913A2B882309F42C
:10BC600091E090933A2B992351F0E091B102F0E0EA
:10BC7000DF01A15AB44D8C91E25BF44D808381E0E9
:10BC800080932C0180913A2B882309F048C380913E
:10BC9000B102082F10E0025B144DF801F0808F2DE7
:10BCA00061E00E943911D8018C938091B102E82F94
:10BCB000F0E0E25BF44D8081843008F083E0808323
:10BCC000E091B102F0E0E25BF44D8081F81609F0FA
:10BCD00005C325C3383199F0393128F43C30D9F007
:10BCE000303119F512C0303321F0303611F03032D6
:10BCF000E1F4CE01019661E040E02FE111C0CE01F8
:10BD0000019661E044E02BE10BC0CE01019661E0B9
:10BD100048E027E105C0CE01019661E04AE025E157
:10BD20008E010C5F1F4F0E94641180919B3683FF30
:10BD300006C080E1898381E08C8380932C018C8113
:10BD4000882309F46AC0A091B1024091352B8091FB
:10BD50004C026981A03151F590E0242F30E0FC01C4
:10BD6000EE0FFF1FE80FF91F85E29DE08C01209F79
:10BD7000C001219F900D309F900D1124E80FF91FF5
:10BD8000EB5DFF4E962F9295990F990F907C8081D5
:10BD90008F73892B80836695669567708181887F14
:10BDA000862B818381E08093B90337C090E0B0E0B7
:10BDB000242F30E0FC01EE0FFF1FE80FF91F84EC89
:10BDC00090E0AC01A49FC001A59F900DB49F900D81
:10BDD0001124E80FF91F85E29DE08C01209FC0012E
:10BDE000219F900D309F900D1124E80FF91FE45210
:10BDF000FC4F962F9295990F990F907C80818F73AD
:10BE0000892B80836695669567708181887F862BF4
:10BE10008183A55CB44D81E08C938091913683FF42
:10BE20007EC28091352B90E025E23DE0829FF001BB
:10BE3000839FF00D929FF00D1124EE53FC4F8981EA
:10BE400085838091B102803199F520E030E045E2B0
:10BE50005DE08091352B90E0F901EE0FFF1FE20FBE
:10BE6000F31F849FD001859FB00D949FB00D1124C6
:10BE7000EA0FFB1FEB5DFF4EAE53BC4F15969C9136
:10BE800015979295990F990F907C80818F73892BCC
:10BE9000808315969C919695969597708181887F61
:10BEA000892B81832F5F3F4F2034310591F6F0C0FD
:10BEB00040E050E014ECE12EF12C05E21DE0209171
:10BEC000352B30E08091B102682F70E0FA01EE0F5F
:10BED000FF1FE40FF51F6E9DC0016F9D900D7E9DAD
:10BEE000900D1124E80FF91F209FD001219FB00D64
:10BEF000309FB00D1124EA0FFB1FE452FC4FAE53EC
:10BF0000BC4F15969C9115979295990F990F907C1F
:10BF100080818F73892B808315969C919695969539
:10BF200097708181887F892B81834F5F5F4F403479
:10BF3000510529F6E7C0CE01029661E040E02FE00E
:10BF40008E010C5F1F4F0E94641180919B3683FF0E
:10BF500005C01A8281E08C8380932C018C81882318
:10BF600009F458C0A091B1024091352B80914C0248
:10BF70006A81A03109F590E0242F30E0FC01EE0F3A
:10BF8000FF1FE80FF91F85E29DE08C01209FC00193
:10BF9000219F900D309F900D1124E80FF91FEA5D4D
:10BFA000FF4E660F660F660F80818770862B808339
:10BFB00081E08093B9032EC090E0B0E0242F30E000
:10BFC000FC01EE0FFF1FE80FF91F84EC90E0AC01BD
:10BFD000A49FC001A59F900DB49F900D1124E80F60
:10BFE000F91F85E29DE08C01209FC001219F900DEB
:10BFF000309F900D1124E80FF91FE452FC4F6F7031
:10C00000660F660F8081837C862B8083A55CB44D90
:10C0100081E08C938091913683FF81C18091352B93
:10C0200090E025E23DE0829FF001839FF00D929F1A
:10C03000F00D1124EE53FC4F8A8184838091B1026C
:10C04000803151F520E030E045E25DE08091352B14
:10C0500090E0D901AA0FBB1FA20FB31F849FF0016C
:10C06000859FF00D949FF00D1124AE0FBF1FAA5DA8
:10C07000BF4EEE53FC4F9481990F990F990F8C91FD
:10C080008770892B8C932F5F3F4F20343105F1F659
:10C0900081E08093B90343C140E050E094ECE92E85
:10C0A000F12C05E21DE02091352B30E08091B102AA
:10C0B000682F70E0DA01AA0FBB1FA40FB51F6E9D99
:10C0C000C0016F9D900D7E9D900D1124A80FB91F8A
:10C0D000209FF001219FF00D309FF00D1124AE0F35
:10C0E000BF1FA452BC4FEE53FC4F94819F70990F19
:10C0F000990F8C91837C892B8C934F5F5F4F4034D9
:10C10000510589F6655C744D81E0DB018C9307C1B4
:10C110000091B102003161F50E949111482F809188
:10C120009B3683FF06C081E08093B90380932C0186
:10C130004CE080914C0290E02091352B30E0FC01E6
:10C14000EE0FFF1FE80FF91F85E29DE08C01209F95
:10C15000C001219F900D309F900D1124E80FF91F11
:10C16000EB5DFF4E4F71440F8081817C842BA1C019
:10C17000E0E4F1E02CE08081381721F02150319784
:10C180002223C9F7215010E0055C144DCE0103961F
:10C1900061E040E00E94641180919B3683FF0AC0F9
:10C1A0001B82E091B102F0E0E55CF44D81E0808318
:10C1B00080932C018091913683FF4CC08091352B68
:10C1C00090E025E23DE0829FF001839FF00D929F79
:10C1D000F00D1124EE53FC4F8B81868340E050E03C
:10C1E000B4ECEB2EF12C05E21DE02091352B30E074
:10C1F0008091B102682F70E0FA01EE0FFF1FE40F8B
:10C20000F51F6E9DC0016F9D900D7E9D900D1124B8
:10C21000E80FF91F209FD001219FB00D309FB00D76
:10C220001124EA0FFB1FE352FC4FAE53BC4F16968E
:10C230009C91990F990F990F80818770892B80832A
:10C240004F5F5F4F4034510581F6655C744D81E06E
:10C25000DB018C9380914C0290E02091B10230E0A0
:10C260004091352B50E0FC01EE0FFF1FE80FF91F46
:10C2700084EC90E08C01209FC001219F900D309FA5
:10C28000900D1124E80FF91F85E29DE09C01429F6B
:10C29000C001439F900D529F900D1124E80FF91F8C
:10C2A000E352FC4F9B81990F990F990F8081877002
:10C2B000892B808334C08091323690E061E070E059
:10C2C0000E940811982F873008F096E0909332363C
:10C2D00080915837981719F19093583781E08093DF
:10C2E0002C011DC08091EF01813051F0813028F088
:10C2F000823049F0833099F409C085E396E308C0A1
:10C3000086E396E305C087E396E302C088E396E3FD
:10C3100069E140E024E600E010E00E9464110F9023
:10C320000F900F900F900F90CF91DF911F910F9171
:10C33000FF90EF90DF90CF90BF90AF909F900895C7
:10C34000CF92DF92EF92FF920F931F937B018C01AC
:10C3500084EAC82E88E3D82E980144275527205B0D
:10C36000C601622F0E94E27E5527412F302F2F2DCC
:10C37000C601622F0E946E7FC6016E2D0E946E7FE5
:10C380001F910F91FF90EF90DF90CF9008953F9213
:10C390004F925F926F927F928F929F92AF92BF92D5
:10C3A000CF92DF92EF92FF920F931F932091FA3377
:10C3B0003091FB33220F232F221F330B3195322E66
:10C3C000E82EFF2400E010E030E040E050E0E1E83B
:10C3D000AE2EE9E0BE2EC12CD12CA20EB31EC41E7F
:10C3E000D51ED801C70172E0880F991FAA1FBB1F75
:10C3F0007A95D1F7A80EB91ECA1EDB1E67E0AA0CFB
:10C40000BB1CCC1CDD1C6A95D1F729013A0127E041
:10C41000440C551C661C771C2A95D1F78824C6014C
:10C42000B5010E94A061831401F599240AC0E92D89
:10C43000F0E0EC50FC4C84EA98E361850E946E7F4A
:10C440009394292D30E040E050E08091FA339091B0
:10C45000FB33A0E0B0E084199509A609B7092817B5
:10C4600039074A075B0718F30EC09924E92DF0E05D
:10C47000EC50FC4C84EA98E361850E946E7F9394B3
:10C4800080E8981699F784EA98E30E94B17F6AE001
:10C4900070E080E090E00E94AF848394381408F04C
:10C4A000BECF99E0EE0CFF1C001F111F9A95D1F72B
:10C4B00083E792ECA4E0B0E0E80EF91E0A1F1B1F10
:10C4C000C801B7010E94A06184EA98E36091FA3341
:10C4D0000E946E7F6091FB3384EA98E30E946E7F36
:10C4E00084EA98E30E94B17F6AE070E080E090E027
:10C4F0000E94AF841F910F91FF90EF90DF90CF903B
:10C50000BF90AF909F908F907F906F905F904F9073
:10C510003F900895CF92DF92EF92FF920F931F9377
:10C5200060E070EC84E090E00E94A06104EA18E30F
:10C53000609148026370C8010E946E7FC8016091DB
:10C5400040020E946E7FC801609139020E946E7F96
:10C55000C801609138020E946E7FC80160913A0262
:10C560000E946E7FC80160913D020E946E7FC801EB
:10C57000609136020E946E7FB8E4EB2EB2E0FB2E93
:10C58000C801609135020E946E7FAAEFCA2EAFEFFC
:10C59000DA2ECE0CDF1CC801F60160810E946E7F8E
:10C5A000F6016181C8010E946E7F8CEF9FEFE80E5B
:10C5B000F91EC801F70160810E946E7FF701618159
:10C5C000C8010E946E7FC8010E94B17F6AE070E0DE
:10C5D00080E090E00E94AF841F910F91FF90EF9058
:10C5E000DF90CF9008959F92AF92BF92CF92DF924B
:10C5F000EF92FF920F931F938091480282FF3BC0FE
:10C60000837090E081309105D9F082309105F1F08E
:10C61000892B61F5809140029091410290933F02F5
:10C6200080933E028091C636882319F080E00E94F4
:10C63000C6168091C736882319F081E00E94C6167D
:10C640000E942F2781E08093710110C080E293E067
:10C65000A0E0B0E08093680190936901A0936A0123
:10C66000B0936B010E942F271092710180914802B4
:10C670008B7F8093480280913702882351F080910C
:10C680008B3683FF06C00E948A62109237020E9496
:10C6900062398091460290914702089711F01092FA
:10C6A000370280914802837009F485C090901F374B
:10C6B00083E68915E0F1E0906801F090690100914E
:10C6C0006A0110916B016091203770912137809140
:10C6D0002237909123370E94168C5B016C0189E60A
:10C6E00090E0A0E0B0E0E80EF91E0A1F1B1F60E614
:10C6F0007AEE80E090E0A80197010E94818DCA0146
:10C70000B9010E94168C9B01AC01C601B5010E94C3
:10C71000158B0E94EA8B60932037709321378093AA
:10C72000223790932337939490921F371CC06091C7
:10C73000203770912137809122379091233724E65A
:10C7400030E040E050E00E94818D30933F02209322
:10C750003E0210921F37109220371092213710920C
:10C7600022371092233720913E0230913F02809170
:10C770001D3790911E37281B390B37FF03C03095AA
:10C7800021953F4F25313105B4F08091C63688237D
:10C7900019F080E00E94C6168091C736882319F0F0
:10C7A00081E00E94C61680913E0290913F029093D4
:10C7B0001E3780931D371F910F91FF90EF90DF90F0
:10C7C000CF90BF90AF909F9008952F923F924F923D
:10C7D0005F927F928F929F92AF92BF92CF92DF92A1
:10C7E000EF92FF920F931F93DF93CF9300D000D06F
:10C7F000CDB7DEB7062FC82EDD24EE24FF2460312E
:10C8000009F41EC1262E332444245524C701B60141
:10C8100023E130E040E050E00E942F8D620D731D57
:10C82000841D951DE7E0660F771F881F991FEA9505
:10C83000D1F70E94A0617724802E99249A82898260
:10C8400084EC90E0889E5001899EB00C989EB00CBC
:10C8500011244CC0872D90E0FC01EE0FFF1FE80F64
:10C86000F91FEA0DFB1DE20FF31FDF01A452BC4FBD
:10C870002C91022F0695017010E0000F111F822FDE
:10C88000869586958F7090E0880F991F880F991F65
:10C89000082B192B822F817090E0082B192B2295E1
:10C8A00026952695237011968C918770880F880F96
:10C8B000822B90E0A6E0880F991FAA95E1F7082B3C
:10C8C000192BE352FC4F8081887F8C831B822B8144
:10C8D0003C81022B132B84EA98E3602F0E946E7F29
:10C8E00084EA98E3612F0E946E7F73948091352BC8
:10C8F00090E0F5E28F2EFDE09F2E889D9001899DAE
:10C90000300D989D300D1124F501E20FF31FE45610
:10C91000FB4F8081871508F09DCF84EA98E30E9441
:10C92000B17F6AE070E080E090E00E94AF84C701D0
:10C93000B60120E839E040E050E00E942F8D7B01F5
:10C940008C0180E098E0A0E0B0E0E80EF91E0A1F3C
:10C950001B1FC201B10126E030E040E050E00E9420
:10C960002F8DE60EF71E081F191FC801B7010E9480
:10C97000A06184EA98E360E00E946E7F8091352B8D
:10C9800090E0889DF001899DF00D989DF00D112497
:10C99000EA0DFB1DE456FB4F84EA98E360810E9498
:10C9A0006E7F8091352B90E0889DF001899DF00D80
:10C9B000989DF00D1124EA0DFB1DE356FB4F84EA10
:10C9C00098E360810E946E7F8091352B90E0889D76
:10C9D000F001899DF00D989DF00D1124EA0DFB1DCD
:10C9E000E156FB4F84EA98E360810E946E7F80915C
:10C9F000352B90E0889DF001899DF00D989DF00DFC
:10CA00001124EA0DFB1DE256FB4F84EA98E3608196
:10CA10000E946E7F8091352B90E0889DF001899D6A
:10CA2000F00D989DF00D1124EE53FC4FA981BA81B1
:10CA3000EA0FFB1F84EA98E367810E946E7FF5C0CE
:10CA4000C701B60120E839E040E050E00E942F8D98
:10CA50006B017C016058774F8F4F9F4F0E94A06100
:10CA60008091352B90E005E21DE0809FF001819FD1
:10CA7000F00D909FF00D1124EF5DFF4E84EA98E3D6
:10CA800060810E946E7F8091352B90E0809FF00145
:10CA9000819FF00D909FF00D1124E05EFF4E84EA1F
:10CAA00098E360810E946E7F8091352B90E0809F9B
:10CAB000F001819FF00D909FF00D1124EE5DFF4E6F
:10CAC00084EA98E360810E946E7F8091352B90E02C
:10CAD000809FF001819FF00D909FF00D1124ED5D7E
:10CAE000FF4E84EA98E360810E946E7F8091352B2F
:10CAF00090E0809FF001819FF00D909FF00D112438
:10CB0000E15EFF4E84EA98E360810E946E7F00E060
:10CB1000E5E2AE2EEDE0BE2E11C0802F90E0FC01CC
:10CB2000EE0FFF1FE80FF91FE20FF31FE95DFF4E45
:10CB3000608184EA98E30E946E7F0F5F8091352BBD
:10CB400090E08A9D90018B9D300D9A9D300D1124AF
:10CB5000F901EF5DFF4E80818017F8F684EA98E3D3
:10CB60000E94B17F6AE070E080E090E00E94AF84B4
:10CB7000C701B6016050774F8F4F9F4F0E94A06151
:10CB8000FF2465E2C62E6DE0D62E3EC08F2D90E0CC
:10CB9000FC01EE0FFF1FE80FF91FE20FF31FDF018B
:10CBA000AB5DBF4E2C91022F06950F7110E0000F68
:10CBB000111F422F429546954695437011968C91D0
:10CBC0008770880F880F842B90E036E0880F991FBC
:10CBD0003A95E1F7082B192B217030E0022B132B2B
:10CBE000EA5DFF4E808198EF992E982288240829CB
:10CBF000192984EA98E3602F0E946E7F84EA98E303
:10CC0000612F0E946E7FF3948091352B90E08C9D74
:10CC100090018D9D300D9C9D300D1124F901EF5D2B
:10CC2000FF4E80818F1508F0B1CF84EA98E30E940F
:10CC3000B17F6AE070E080E090E00E94AF840F90E6
:10CC40000F900F900F90CF91DF911F910F91FF9058
:10CC5000EF90DF90CF90BF90AF909F908F907F909C
:10CC60005F904F903F902F9008952F923F924F9258
:10CC70005F927F928F929F92AF92BF92CF92DF92FC
:10CC8000EF92FF920F931F93DF93CF9300D000D0CA
:10CC9000CDB7DEB77724C8C0003109F43FC0C70163
:10CCA000B6010E94A06110E084EA98E362E00E946D
:10CCB0006E7F84EA98E364E00E946E7F1F5F103409
:10CCC00099F784EA98E30E94B17F6AE070E080E01F
:10CCD00090E00E94AF84C501B4010E94A06184EA83
:10CCE00098E361E00E946E7F84EA98E36FE00E941F
:10CCF0006E7F84EA98E368E10E946E7F84EA98E39D
:10CD000061E00E946E7F84EA98E360E00E946E7F9B
:10CD100084EA98E360E00E946E7F44C069817A8172
:10CD20008B819C810E94A06184EA98E36FE00E945D
:10CD30006E7F84EA98E368E10E946E7F84EA98E35C
:10CD400061E00E946E7F84EA98E360E00E946E7F5B
:10CD500084EA98E360E00E946E7F10E084EA98E342
:10CD600060E30E946E7F1F5F1034C1F784EA98E38E
:10CD70000E94B17F6AE070E080E090E00E94AF84A2
:10CD8000C201B1010E94A06110E084EA98E368E169
:10CD90000E946E7F84EA98E364E00E946E7F1F5FCA
:10CDA000103499F784EA98E30E94B17F6AE070E05A
:10CDB00080E090E00E94AF840F5F86E090E0A0E00A
:10CDC000B0E0880E991EAA1EBB1E80E890E0A0E08D
:10CDD000B0E0C80ED91EEA1EFB1E013109F05CCF7F
:10CDE000272D26952695269581E090E0A0E0B0E0DD
:10CDF00004C0880F991FAA1FBB1F2A95D2F79C0158
:10CE0000AD0180915A3790915B37822B932B909391
:10CE10005B3780935A3760E070E040E00E942F0F4C
:10CE2000739490E8791651F1672D70E080E090E0FE
:10CE300020E839E040E050E00E942F8D6B017C013A
:10CE4000812CA8E09A2EA12CB12C860E971EA81E2C
:10CE5000B91EDC01CB018058974FAF4FBF4F89837C
:10CE60009A83AB83BC83212CF9E03F2E412C512CBB
:10CE70002C0C3D1C4E1C5F1C00E00ECF60E070ECE3
:10CE800084E090E00E94A06184EA98E360E00E9460
:10CE90006E7F84EA98E368E70E946E7F84EA98E3F5
:10CEA00061E00E946E7F84EA98E361E00E946E7FF9
:10CEB00084EA98E361E00E946E7F84EA98E30E942E
:10CEC000B17F6AE070E080E090E00E94AF8484EA85
:10CED00098E367E570E00E94EC7E84EA98E36FEFE8
:10CEE0000E946E7F84EA98E36DEF0E946E7F84EA71
:10CEF00098E360E00E946E7F84EA98E361E00E941C
:10CF00006E7F84EA98E363E00E946E7F84EA98E390
:10CF10000E94B17F6AE070E080E090E00E94AF8400
:10CF20000F900F900F900F90CF91DF911F910F9165
:10CF3000FF90EF90DF90CF90BF90AF909F908F9039
:10CF40007F905F904F903F902F9008953F924F9227
:10CF50005F926F927F928F929F92AF92BF92CF9289
:10CF6000DF92EF92FF920F931F93A82EBB24CC2445
:10CF7000DD2486017501F9E0EE0CFF1C001F111F76
:10CF8000FA95D1F783E792ECA4E0B0E0E80EF91E41
:10CF90000A1F1B1FC801B7010E94A06184EA98E321
:10CFA0000E94B17F78010027112790E5E90E84EAFD
:10CFB00098E36E2D42E00E94C67F84EA98E30E94C7
:10CFC000FF7E8C0184EA98E30E94FF7E382F20E0E8
:10CFD0001070022B132B1093FB330093FA33045F72
:10CFE000114020F01092FB331092FA338091FA3303
:10CFF0009091FB33880F892F881F990B9195582E9C
:10D00000282F30E040E050E061E8662E69E0762E9F
:10D01000812C912C620E731E841E951E92E0AA0C28
:10D02000BB1CCC1CDD1C9A95D1F76A0C7B1C8C1C9C
:10D030009D1C87E0660C771C881C991C8A95D1F78B
:10D04000C401AA27BB2710E5412E480E59016A01E9
:10D05000B7E0AA0CBB1CCC1CDD1CBA95D1F73A2C4E
:10D06000FF24C401B3010E94A06184EA98E30E94F6
:10D07000B17FF51461F54091FA33431984EA98E3DE
:10D08000642D0E94C67FEE240EC00E2D10E084EAAF
:10D0900098E30E94FF7EF801EC50FC4C81878138B8
:10D0A00008F01186E3942E2D30E040E050E08091AE
:10D0B000FA339091FB33A0E0B0E08A199B09AC09E8
:10D0C000BD09281739074A075B07F8F218C084EA38
:10D0D00098E3642D40E80E94C67FEE240E2D10E0F8
:10D0E00084EA98E30E94FF7EF801EC50FC4C8187B3
:10D0F000813808F01186E394B0E8EB1679F7F394E1
:10D100005F1408F0AECF1F910F91FF90EF90DF906A
:10D11000CF90BF90AF909F908F907F906F905F90D7
:10D120004F903F9008950F931F9360E070EC84E060
:10D1300090E00E94A06184EA98E30E94B17F84EAB3
:10D1400098E364E540E80E94C67F84EA98E30E9481
:10D15000FF7E982F9370933009F492E09370809142
:10D1600048028C7F892B8093480284EA98E30E94CE
:10D17000FF7E90E08E31910518F48EE190E005C0BD
:10D180008B3F910510F08AEF90E0909341028093DD
:10D19000400284EA98E30E94FF7E882311F481E034
:10D1A00003C0813108F080E18093390284EA98E37A
:10D1B0000E94FF7E882311F481E003C0813108F0D2
:10D1C00080E18093380284EA98E30E94FF7E8430F5
:10D1D00008F083E080933A0284EA98E30E94FF7E9D
:10D1E000823010F482E003C08B3008F08AE0809334
:10D1F0003D0284EA98E30E94FF7E811181E08093E2
:10D20000360284EA98E30E94FF7E811181E08093D8
:10D21000350284EA98E30E94FF7E8C0184EA98E359
:10D220000E94FF7E382F20E01070022B132B1093EA
:10D230004302009342020050104130F08FEF9FE014
:10D24000909343028093420284EA98E30E94FF7E17
:10D250008C0184EA98E30E94FF7E382F20E0107052
:10D26000022B132B109345020093440200501041EF
:10D2700030F08FEF9FE090934502809344021F911E
:10D280000F9108950E94936810924E0210923301FC
:10D29000109232011092F10183E090E090934702E6
:10D2A0008093460280E00E945A850E949688809171
:10D2B0006800816080936800D89A80916B008360D9
:10D2C00080936B001092CD008FE18093CC00809111
:10D2D000CA0086608093CA008091C90088698093E3
:10D2E000C9001092F2028091400290914102909305
:10D2F0003F0280933E0280914802837090E081302B
:10D30000910529F08230910541F0892B51F40E945A
:10D310002F2781E08093710104C00E942F27109273
:10D320007101809148028B7F80934802809149026D
:10D33000882311F02C9A01C02C988091352B90E015
:10D3400025E23DE0829FF001839FF00D929FF00D5A
:10D350001124DF01A95DBF4E4C91942F9F70E15EB7
:10D36000FF4EE0818CE0E89FF0011124E90FF11DF0
:10D37000E355FC4FE491E150F0E0EE0FFF1FE75E54
:10D38000FB4F85919491469546954695342F3E7076
:10D3900020E0820F931F0E94E10F08952F923F9289
:10D3A0004F925F926F927F928F929F92AF92BF92B5
:10D3B000CF92DF92EF92FF920F931F93DF93CF9361
:10D3C000CDB7DEB76E970FB6F894DEBF0FBECDBFF8
:10D3D000062F90E0A0E0B0E0BC01CD0120E839E0EC
:10D3E00040E050E00E942F8D5B016C01612C78E0E1
:10D3F000772E812C912C6A0C7B1C8C1C9D1CA60109
:10D4000095012058374F4F4F5F4F29873A874B87F9
:10D410005C87CA01AA27BB27382F305B3E83D60121
:10D42000C5018050974FAF4FBF4F8A839B83AC831A
:10D43000BD83CD01AA27BB27E82FE05BE98310E07D
:10D4400085E29DE09C01029FC001039F900D129F09
:10D45000900D1124AC0144565B4F5E8F4D8FDC0163
:10D46000A753BC4FB887AF83222433242C018E539B
:10D470009C4FFC01E15AF34FFC8BEB8B9C01225A31
:10D48000334F3E8B2D8BAC01405A534F588F4F8BEF
:10D49000DC01AF59B34FBA8FA98FFC01E35AF34FA8
:10D4A000FC8FEB8FF0E12F16310409F4D5C0C401D5
:10D4B000B3010E94A06184EA98E30E94B17F9401C5
:10D4C00044275527205B84EA98E3622F46E00E94B8
:10D4D000C67F84EA98E30E94FF7E84EA98E30E9474
:10D4E000FF7EAD8DBE8D8C9384EA98E30E94FF7E13
:10D4F000ED8DFE8D818384EA98E30E94FF7EAD8DE1
:10D50000BE8D13968C9384EA98E30E94FF7EED8D86
:10D51000FE8D828384EA98E30E94FF7EAF81B88506
:10D520008C93ED8DFE8DE080FF240894E11CF11CAE
:10D53000EE0CFF1C0027F7FC0095102FC601B5016B
:10D540000E94A06184EA98E30E94B17F960144277B
:10D550005527205B84EA98E3622F4E2D0E94C67FF8
:10D56000EE2444EC50E0249E9001259E300D349E24
:10D57000300D11243A8B298B68C084EA98E30E940D
:10D58000FF7E8C0184EA98E30E94FF7E8E871D86D1
:10D59000A80150708D859E85482B592B6E2D70E00B
:10D5A000FB01EE0FFF1FE60FF71FA989BA89EA0FEB
:10D5B000FB1FE40DF51DE452FC4F242F2170308138
:10D5C0003C7FCA0182709070969587958170880F14
:10D5D000322B382BCA018C7390709695879596954F
:10D5E00087958F70282F220F220F337C322B3083A8
:10D5F000882311F4337C3083FB01EE0FFF1FE60F0D
:10D60000F71F29893A89E20FF31FE40DF51DDF01A9
:10D61000A452BC4FCA01807C977076E0969587959E
:10D620007A95E1F7382F3295330F330F307C2C91F8
:10D630002F73232B2C9386958695E352FC4F252F31
:10D64000287F8770822B8083E394AD8DBE8D8C9173
:10D650008E1508F092CFD0C069857A858B859C8520
:10D660000E94A06184EA98E30E94B17F84EA98E373
:10D670006E8140E80E94C67F84EA98E30E94FF7EA4
:10D68000EB89FC89808384EA98E30E94FF7EAD8960
:10D69000BE898C9384EA98E30E94FF7EEF89F88D1F
:10D6A000808384EA98E30E94FF7EA98DBA8D8C93D3
:10D6B00084EA98E30E94FF7EEB8DFC8D80838930A5
:10D6C00008F088E0AB8DBC8D8C9300E022C084EA2A
:10D6D00098E30E94FF7E202F30E0F901EE0FFF1F3C
:10D6E000E20FF31FE40DF51DE95DFF4E282F30E03A
:10D6F0002077307054E0359527955A95E1F72770DB
:10D700002295207F982F90788F70282B292B2083AB
:10D710000F5FEB89FC89E080E016C8F66A817B81A7
:10D720008C819D810E94A06184EA98E30E94B17F70
:10D730002E2D30E02F5F3F4F220F331F442737FD40
:10D740004095542F84EA98E36981422F0E94C67F56
:10D75000EE244CC084EA98E30E94FF7E8C0184EAA8
:10D7600098E30E94FF7E888B1F8610702F85388972
:10D77000022B132B8E2D90E0AC01440F551F480F48
:10D78000591F440D551DFA01EB5DFF4E702F71704E
:10D79000C8018E739070969587958F71880F980148
:10D7A000207C3770B6E036952795BA95E1F7622F61
:10D7B0006295660F660F607C872B862B808326958B
:10D7C0002695812F869586958695FA01EA5DFF4E0E
:10D7D000982F990F990F990F2770292B2083815E1D
:10D7E0008F71803110F027702083E394AB89BC895E
:10D7F0008C918E1508F0AECF0894211C311CED8D54
:10D80000FE8DEC53FF4FFE8FED8F26E030E040E0C1
:10D8100050E0620E731E841E951E4F8158854F5F27
:10D820005F4F58874F8380E890E0A0E0B0E0A80EFB
:10D83000B91ECA1EDB1E91E12916310409F032CE51
:10D840006E960FB6F894DEBF0FBECDBFCF91DF91BD
:10D850001F910F91FF90EF90DF90CF90BF90AF900E
:10D860009F908F907F906F905F904F903F902F9000
:10D87000089580ED84B982EF8AB98CEF81B989E08F
:10D8800061E00E947C8512B85F980E94AF7C8FEFA8
:10D890000E948D7C84EA98E30E94CA7F0895FF92DB
:10D8A0000F931F93CF93DF9300E0C5E2DDE06CE0C0
:10D8B000F62E7EC16CE070E080E090E00E94568819
:10D8C000162F80913536823381F1833320F48931EC
:10D8D00009F097C007C08B3409F44AC0843609F0B8
:10D8E00090C069C067E070E080E090E00E945688D8
:10D8F000613071058105910509F083C08091352B58
:10D9000090E08C9F90018D9F300D9C9F300D1124D5
:10D91000F901E15EFF4EE081EF9DF0011124E10F7E
:10D92000F11DE355FC4F44915CC064E070E080E081
:10D9300090E00E945688613071058105910509F0DB
:10D9400060C08091352B90E08C9F90018D9F300DB1
:10D950009C9F300D1124F901E15EFF4EE081EF9DA7
:10D96000F0011124E10FF11DE355FC4F449139C042
:10D9700063E070E080E090E00E94568861307105BD
:10D980008105910509F03DC08091352B90E08C9F79
:10D9900090018D9F300D9C9F300D1124F901E15EA7
:10D9A000FF4EE081EF9DF0011124E10FF11DE355E1
:10D9B000FC4F449116C08091352B90E08C9F9001D4
:10D9C0008D9F300D9C9F300D1124F901E15EFF4EBB
:10D9D000E081EF9DF0011124E10FF11DE355FC4FB3
:10D9E0004491802F90E0FC01EE0FFF1FE80FF91F1C
:10D9F000E20FF31FE95DFF4E4F708081807F842B23
:10DA0000808368E070E080E090E00E945688162FE6
:10DA100080913636823379F0833318F48931C1F539
:10DA200005C08B3469F0843699F515C067E070E065
:10DA300080E090E009C064E070E080E090E004C025
:10DA400063E070E080E090E00E94568861307105EC
:10DA500081059105E9F4202F30E08091352B90E08D
:10DA6000F901EE0FFF1FE20FF31F9C012C9FC00175
:10DA70002D9F900D3C9F900D1124E80FF91FE95D3B
:10DA8000FF4E17701295107F80818F78812B8083D5
:10DA900062E070E080E090E00E945688162F80914E
:10DAA0003736823379F0833318F48931B1F505C004
:10DAB0008B3469F0843689F515C067E070E080E04A
:10DAC00090E009C064E070E080E090E004C063E0B2
:10DAD00070E080E090E00E94568861307105810519
:10DAE0009105D9F4202F30E08091352B90E0F90199
:10DAF000EE0FFF1FE20FF31F9C012C9FC0012D9F13
:10DB0000900D3C9F900D1124E80FF91FEB5DFF4E27
:10DB1000117080818E7F812B80836AE070E080E0CD
:10DB200090E028E130E040E050E00E947888162F35
:10DB300080913836823379F0833318F48931B9F51E
:10DB400005C08B3469F0843691F515C067E070E04C
:10DB500080E090E009C064E070E080E090E004C004
:10DB600063E070E080E090E00E94568861307105CB
:10DB700081059105E1F4202F30E08091352B90E074
:10DB8000F901EE0FFF1FE20FF31F9C012C9FC00154
:10DB90002D9F900D3C9F900D1124E80FF91FEB5D18
:10DBA000FF4E1F71110F8081817C812B80830F5F5D
:10DBB0008091352B90E08C9FF0018D9FF00D9C9F04
:10DBC000F00D1124EF5DFF4E8081801708F072CEBA
:10DBD000DF91CF911F910F91FF9008958F929F92A7
:10DBE000AF92BF92CF92DF92EF92FF920F931F936B
:10DBF000CF93DF9381E060E070E00E948008909313
:10DC0000B3368093B2368091AB02882379F080914D
:10DC1000460290914702089749F483E090E0909380
:10DC200047028093460281E080932C018091460256
:10DC3000909147028430910531F00C9721F01092B9
:10DC4000B0021092F43580912936882379F00E9431
:10DC5000A18460932B3670932C3680932D3690934D
:10DC60002E3681E080932A361092293680912A360A
:10DC70008823F1F08091AB028823D1F00E94A18427
:10DC800020912B3630912C3640912D3650912E36E6
:10DC9000621B730B840B950B61597140804090405F
:10DCA00038F081E0809328361092710110922A3664
:10DCB0008091993682FF21C080919B3683FF1DC0E1
:10DCC00080914602909147020597B9F08091B30286
:10DCD0006091352B0E94CE690E944F268091B3023D
:10DCE0000E94A12CEBE3FBE211923BE2EB34F30741
:10DCF000D9F71092B9031092E3368091A93683FFC9
:10DD00000CC08091873682FD08C080917101882304
:10DD100021F080914802837049F080912736882352
:10DD200029F480910436882309F44AC081E0809365
:10DD3000AB021092400110923136109227361092A9
:10DD4000043610924E021092B4031092B303109254
:10DD5000AA021092E4362C982C9A10924902109242
:10DD6000AC36109233011092320180E090E021E055
:10DD7000FC01E05AFD4F1082FC01E752FD4F10827A
:10DD8000FC01EA54FD4F2083FC01EE57FD4F108249
:10DD9000FC01E65FF94C2083FC01ED56FD4F20832A
:10DDA00001968131910521F78091C636882311F0C3
:10DDB0001092C2368091C736882311F01092C33674
:10DDC00080913136882341F08091AB02882321F085
:10DDD000109231361092AC368091AB3683FF0CC076
:10DDE0008091873682FD08C080917101882321F0DF
:10DDF00080914802837049F080910536882329F488
:10DE000080912836882309F454C05F981092EA0262
:10DE1000109249021092B0021092B6031092B5030C
:10DE20008091312B882359F091E09093332B80918E
:10DE3000322B8093B5028093B3029093362B80915E
:10DE40000536882311F01092AC368091283688234D
:10DE500011F01092AC3610922836109205361091BF
:10DE6000AC361F5F1093AC36113019F0123009F543
:10DE700017C0109340011092AB020E94622A0E94C8
:10DE8000622A0E94622A0E94622A809135028823B7
:10DE900081F080E090E80E94770F10934A0209C059
:10DEA0001092400181E08093AB021092AC36109248
:10DEB0004E028091873682FF36C08091953683FF6F
:10DEC00004C08091B1020E9430218091973683FF77
:10DED00004C08091B1020E942F238091A73683FF56
:10DEE00009C08CE090E0909347028093460281E065
:10DEF00080932C018091913683FFF3C0809146027C
:10DF000090914702019739F081E090E090934702A9
:10DF10008093460204C0109247021092460281E0AC
:10DF200080932C01DEC0809146029091470282309E
:10DF3000910569F48091953683FF02C00E94751F98
:10DF40008091973683FF3AC00E94BF1F37C083304D
:10DF50009105B9F48091953683FF08C08091B10294
:10DF60000E94BA1C8091B10280934C2B809197360D
:10DF700083FF24C08091B10260914C2B0E94B81D98
:10DF80001DC00997D9F48091953683FF08C0809110
:10DF90004C0280934D028091B10280934C2B809172
:10DFA000973683FF0BC080914C2B60914D024091BE
:10DFB0004C020E94BB1B81E080932C0180919D3616
:10DFC00083FF12C08091460290914702039719F097
:10DFD00083E090E002C082E090E09093470280935B
:10DFE000460281E080932C018091A73683FF1CC0FC
:10DFF0008091460290914702049719F084E090E0E6
:10E0000002C083E090E090934702809346028091A3
:10E01000B102803121F481E08093F43502C0109286
:10E02000F43581E080932C0120918F3623FF17C0B7
:10E0300080914602909147028530910581F090933E
:10E04000AD028093AC0285E090E09093470280930C
:10E050004602206420938F3681E080932C0120912A
:10E060008F3624FF23C026FF0AC08091460290917C
:10E0700047020597D9F42F7B20938F3617C08091E4
:10E08000460290914702059789F48091F23390916E
:10E09000F333892B59F48091AC029091AD029093A7
:10E0A00047028093460281E080932C0180914602D2
:10E0B00090914702059721F01092F3331092F233BA
:10E0C0008091460290914702089711F01092F10159
:10E0D00080914602909147020797029710F01092A4
:10E0E000F1018091A93683FF1DC08091873682FFA0
:10E0F00019C08091AB028823A9F488E090E0909346
:10E100004702809346028091F1018F5F8093F10175
:10E11000833018F081E08093F1011092EF0181E0EB
:10E1200080932C019091A136969596959695917035
:10E1300041F08091873682FD04C081E08093F50133
:10E1400007C08091A13684FF06C01092F50181E0DE
:10E1500080932C0110C0992371F08091873682FF43
:10E160000AC08091B102803131F48DE090E090934B
:10E170004702809346028091A53683FF04C081E068
:10E180008093F40105C084FF05C01092F40181E082
:10E1900080932C012091460230914702C9010397D8
:10E1A000029768F02730310551F02930310539F0F8
:10E1B0002630310521F02C30310509F0AAC58091B7
:10E1C000B2369091B336892B11F41092B13680910A
:10E1D000893682FF3EC08091933683FF0DC083E075
:10E1E00090E090934702809346020E94AE0B80938A
:10E1F000B10281E080932C0180918B3683FF0CC0AB
:10E2000087E090E0909347028093460280E18093FC
:10E21000B10281E080932C0180919B3683FF0CC07A
:10E2200083E090E0909347028093460280E18093E0
:10E23000B10281E080932C018091993683FF09C05F
:10E2400086E090E0909347028093460281E08093BD
:10E250002C018091993683FF1CC08091B1028031DE
:10E26000C1F48091893682FD14C087E090E09093DC
:10E27000470280934602809101368093BB0391E070
:10E2800090932C018F5F80930136823010F01092B2
:10E2900001368091460290914702079711F0109243
:10E2A000013680919B3683FF11C080914602909188
:10E2B0004702079759F41092013683E090E090935B
:10E2C00047028093460281E080932C0180919F3623
:10E2D00082FF91C08091AB02882309F48CC0209109
:10E2E000B1024091352B203109F043C080915F028B
:10E2F00090E0242F30E0FC01EE0FFF1FE80FF91F24
:10E3000085E29DE0A901489F9001499F300D589FEB
:10E31000300D1124E20FF31FEB5DFF4E80818E7FE5
:10E32000808380915F0290E0FC01EE0FFF1FE80FF9
:10E33000F91FE20FF31FDF01AB5DBF4E8C918E7FA3
:10E340008C93EA5DFF4E8081877080839C9111964B
:10E350008C911197887F846011968C93119791709E
:10E3600098619C9381E08093B9035F981092EA02D0
:10E3700042C030E0D901A15BBD4F8C9190E050E0EC
:10E38000FC01EE0FFF1FE80FF91F84EC90E0289FBF
:10E39000B001299F700D389F700D1124E60FF71FF3
:10E3A00085E29DE0EA01C89FA001C99F500DD89F5A
:10E3B000500D1124E40FF51FE452FC4F80818E7F35
:10E3C00080838C9190E0FC01EE0FFF1FE80FF91F96
:10E3D000E60FF71FE40FF51FDF01A452BC4F8C912D
:10E3E00083708C93E352FC4F84E08083255C344D32
:10E3F00081E0F90180838091873682FF0DC0809192
:10E400009F3683FF09C08091B102803119F00E94CC
:10E41000D61E02C00E94211F80918D3682FF0BC143
:10E420008091933683FF07C18091873682FF6EC04B
:10E430008091352B90E025E23DE0829F8001839F13
:10E44000100D929F100D11240E531C4FD801FC90FB
:10E450000E94AE0BE091B102F0E0E25BF44D9081DE
:10E460009295907F980FE801988320E030E064EC6B
:10E4700070E045E25DE011E08091352B90E0269F51
:10E48000F001279FF00D369FF00D1124DC01A49FB1
:10E49000C001A59F900DB49F900D1124E80FF91FA6
:10E4A000E456FB4FDC01AE53BC4F8C918083F901E5
:10E4B000E55CF44D10832F5F3F4F20313105E1F6CD
:10E4C000FD01E15AF34F8C9180831093B903809141
:10E4D0003602813009F0ACC010E0C5E2DDE0809189
:10E4E000352B90E08C9FF0018D9FF00D9C9FF00DDF
:10E4F0001124EE53FC4F4081F41620F4812F6F2D30
:10E500000E9419201F5F113151F792C08091B10212
:10E510004091352B8031C1F5842F90E0C5E2DDE0DC
:10E520008C9F80018D9F100D9C9F100D11240F5DFD
:10E530001F4EF801F0800E94AE0B2091B102E22F35
:10E54000F0E0E25BF44D90819295907F980FD801B6
:10E550009C9381E08093B90380913602813009F069
:10E5600065C08091352B90E08C9FF0018D9FF00D60
:10E570009C9FF00D1124EF5DFF4E4081F41608F0D2
:10E5800055C0822F6F2D50C0242F30E090E004EC56
:10E59000E02EF12C8E9DF0018F9DF00D9E9DF00DD3
:10E5A0001124C5E2DDE02C9F80012D9F100D3C9FC2
:10E5B000100D1124E00FF11FE456FB4FD0800E9494
:10E5C000AE0B5091B102A52FB0E0AE9D9001AF9D72
:10E5D000300DBE9D300D1124020F131F04561B4F2A
:10E5E000FD01E25BF44D90819295907F980FF801C8
:10E5F0009083A55CB44D81E08C938091360281308C
:10E60000A9F48091352B90E08C9FF0018D9FF00D47
:10E610009C9FF00D1124E20FF31FE456FB4F408145
:10E62000D41620F4852F6D2D0E9419200E94E62516
:10E6300081E080932C018091873682FF5DC08091BC
:10E64000893683FF59C04091B1024E3009F454C05D
:10E650004F3009F451C0403109F44EC08091352B40
:10E6600090E025E23DE0829FF001839FF00D929FB4
:10E67000F00D1124EE53FC4FE40FF11D8781882328
:10E6800081F1178240E050E0A4ECB0E065E27DE06B
:10E690008091B10290E02091352B30E0FA01EE0F2D
:10E6A000FF1FE40FF51FEC01CA9FC001CB9F900D27
:10E6B000DA9F900D1124E80FF91F269FC001279FB4
:10E6C000900D369F900D1124E80FF91FE452FC4F76
:10E6D0008081826080834F5F5F4F40345105C1F677
:10E6E00002C081E0878381E080932C01E091B10238
:10E6F000F0E0E55CF44D8083809146029091470202
:10E700008330910539F08730910521F089309105EA
:10E7100009F031C18091933684FF04C01092B13664
:10E720001092263780918D3682FDF3C28091893612
:10E7300082FDEFC28091873682FD15C0809146022E
:10E7400090914702039779F48091B1022091B236FB
:10E750003091B336803121F4C9010E943D0A03C0D3
:10E76000C9010E94EA088091933683FF79C08091A5
:10E770004602909147028930910519F0079709F0F8
:10E780006FC00E94AE0BE091B102F0E0E25BF44D8D
:10E7900090819295907F980F90934C02809187364C
:10E7A00082FF5BC08091460290914702099709F071
:10E7B00054C060E070E0C4ECD0E0A5E2BDE0809120
:10E7C000B2369091B336062E02C0969587950A947C
:10E7D000E2F780FF3CC08091B1024091352BFB01F4
:10E7E000EE0FFF1F803189F4842F90E0E60FF71FB2
:10E7F0009C012A9FC0012B9F900D3A9F900D1124E0
:10E80000E80FF91FEB5DFF4E1AC0242F30E090E0B7
:10E81000E60FF71FAC014C9FC0014D9F900D5C9F10
:10E82000900D1124E80FF91F2A9FC0012B9F900D16
:10E830003A9F900D1124E80FF91FE452FC4F90E02D
:10E84000808180FF91E080818E7F892B80836F5F44
:10E850007F4F6031710509F0B2CF81E080932C01C8
:10E8600080914602909147028930910541F00797C7
:10E8700009F062C08091B102803109F05DC00E9450
:10E88000CC0B082F0E94AE0B10E0081B11090130C1
:10E89000110509F081C680912637882309F07CC6CE
:10E8A0002091352B30E080914C0290E0FC01EE0F7E
:10E8B000FF1FE80FF91F85E29DE0DC012A9FC001E0
:10E8C0002B9F900D3A9F900D1124E80FF91F22C045
:10E8D0000E94CC0B682F8091352B90E025E23DE023
:10E8E000829FA001839F500D929F500D1124FA0129
:10E8F000EF5DFF4E80816817F9F4809126378823F9
:10E90000D9F4862F90E0FC01EE0FFF1FE80FF91FEE
:10E91000E40FF51FE95DFF4E90E0808187FF91E0F5
:10E9200097959927979580818F77892B808381E0B0
:10E930008093263780932C018091873682FFE9C12E
:10E940008091933683FFE5C189E090E09093470280
:10E95000809346020E94AE0BE091B102F0E0E25BD0
:10E96000F44D90819295907F980F90934C0281E0A6
:10E9700080932C01CEC18430910509F03AC1809179
:10E98000AB02882361F080918B3683FF08C090E052
:10E990008091B002882309F491E09093B0028091B5
:10E9A0009F3682FF53C0A091B1024091352BA03118
:10E9B000F9F480915F0290E0242F30E0FC01EE0F2B
:10E9C000FF1FE80FF91F85E29DE0EC012C9FC001BD
:10E9D0002D9F900D3C9F900D1124E80FF91FEB5DCA
:10E9E000FF4E80818E7F808381E08093B9032EC0AB
:10E9F000B0E0FD01E15BFD4F808190E0242F30E02D
:10EA0000FC01EE0FFF1FE80FF91F84EC90E0AC0152
:10EA1000A49FC001A59F900DB49F900D1124E80FF5
:10EA2000F91F85E29DE0EC012C9FC0012D9F900D08
:10EA30003C9F900D1124E80FF91FE452FC4F808198
:10EA40008E7F8083A55CB44D81E08C9380918D3660
:10EA500082FD0AC08091893682FD06C08091F4351E
:10EA6000882369F00E94FE1340E050E0A4EC8A2E57
:10EA7000912CF5E2AF2EFDE0BF2E01E064C0C0E0B6
:10EA8000D0E0E1E0EE2EF12C8091B2369091B336D9
:10EA90000C2E02C0969587950A94E2F7282F2170D4
:10EAA000FE01EE0FFF1FE959F94C90819E7F922BDA
:10EAB0009083892F86958170281799F192FD31C036
:10EAC000213079F587010C2E02C0000F111F0A9426
:10EAD000E2F7C8010E94CD2AC8010E94770F80ED9D
:10EAE00097E00E94088580E090E00E94770F809177
:10EAF000AB028823B1F08091B002813091F4FE0125
:10EB0000EF58FD4F8081FE0166E0EE0FFF1F6A9512
:10EB1000E1F7E80FF11DEE0FFF1FE059F44DF18210
:10EB2000E082FE01EE0FFF1FE959F94C8081982F1A
:10EB30009170990F8D7F892B80832196C031D105EB
:10EB400009F0A2CF91CFFA01E05AFD4F80818823CE
:10EB500009F048C010E0489DE001499DD00D589D46
:10EB6000D00D11246A0136E0CC0CDD1C3A95E1F79A
:10EB70002BE3E22E2BE2F22EE40EF51E21C0212F14
:10EB800030E0D601A20FB31FAA0FBB1FA059B44D8E
:10EB90008D919C911197892B91F0F901EE0FFF1F38
:10EBA000E20FF31FEC0FFD1FE60FF71FE452FC4FBF
:10EBB000808183608083F70100831D921C921F5F18
:10EBC0008091352B90E08A9DB0018B9D700D9A9DB0
:10EBD000700D1124FE01E60FF71FE456FB4F8081F4
:10EBE000181768F24F5F5F4F4031510509F0ABCF06
:10EBF00090C00C9709F08DC08091B2369091B336D9
:10EC000090933436809333368091AB02882309F495
:10EC100080C080918B3683FF08C090E08091B00265
:10EC2000882309F491E09093B0028091B002882388
:10EC300009F46FC040E050E0E4ECEE2EF12C05E268
:10EC40001DE0CC24C39477E0D72E80913336909189
:10EC50003436042E02C0969587950A94E2F780FF19
:10EC600052C0DA01A15BBD4F8C9190E02091352B11
:10EC700030E0FC01EE0FFF1FE80FF91F4E9DB001C1
:10EC80004F9D700D5E9D700D1124E60FF71F209FA4
:10EC9000E001219FD00D309FD00D1124EC0FFD1FFE
:10ECA000E452FC4F808181608083209132362223A0
:10ECB000B1F08C9190E0FC01EE0FFF1FE80FF91FFF
:10ECC000E60FF71FEC0FFD1FE352FC4F9D2D921B2B
:10ECD000990F990F990F80818770892B0FC08C91A4
:10ECE00090E0FC01EE0FFF1FE80FF91FE60FF71F82
:10ECF000EC0FFD1FE352FC4F808187708083FA0187
:10ED0000E55CF44DC0824F5F5F4F4031510509F023
:10ED10009CCF8091460290914702029709F083C1EF
:10ED20008091893682FF3EC08091933683FF0DC06B
:10ED300083E090E090934702809346020E94AE0BDE
:10ED40008093B10281E080932C0180918B3683FF08
:10ED50000CC087E090E0909347028093460280E1E8
:10ED60008093B10281E080932C0180919B3683FFD8
:10ED70000CC083E090E0909347028093460280E1CC
:10ED80008093B10281E080932C018091993683FFBA
:10ED900009C086E090E0909347028093460281E0AC
:10EDA00080932C0180918D3682FF54C080919336E0
:10EDB00083FF50C00091352B10E00E94AE0B25E27E
:10EDC0003DE0029FD001039FB00D129FB00D1124B2
:10EDD000AE53BC4FE091B102F0E0E25BF44D9081A4
:10EDE0009295907F980F9C9320E030E0C4ECD0E0A7
:10EDF00065E27DE041E08091352B90E02C9FF001B1
:10EE00002D9FF00D3C9FF00D1124DC01A69FC00149
:10EE1000A79F900DB69F900D1124E80FF91FE4569F
:10EE2000FB4FDC01AE53BC4F8C918083E091B1026B
:10EE3000F0E0E55CF44D40832F5F3F4F203131051A
:10EE4000D1F6FD01E15AF34F8C9180834093B903D1
:10EE500040932C0180918D3683FF04C081E0809324
:10EE6000F20105C084FF05C01092F20181E0809399
:10EE70002C0180919F3683FF0CC08091933682FFD6
:10EE800008C09091B3028091B502981711F40E94C6
:10EE90000D208091953682FF1BC08091933683FFB1
:10EEA00017C00E94AE0B0091B2020295007F080FBE
:10EEB0000E944E3910E0802F612F0E94E563802F61
:10EEC0000E94062C1F5F1131B1F781E080932C0165
:10EED0008091933684FF0AC080918D3682FD06C0F2
:10EEE0001092B13610922537109224372091B23605
:10EEF0003091B3362115310509F475C080918D36F6
:10EF000082FD71C0809124379091253728173907E9
:10EF100009F469C0309325372093243780919136C6
:10EF200082FF1AC00E94AE0B873010F087E002C04B
:10EF30000E94AE0B8093B2028091B3029091B20214
:10EF40009295907F8F70980F9093B5028091B30245
:10EF5000891709F045C047C08091893682FD43C0BA
:10EF60008091953682FD3FC00E94CC0B882309F129
:10EF70000E94CC0B182F0E94AE0B181B1093312B44
:10EF80000E94AE0B9091B2029295907F980F909351
:10EF9000322B9093B50221E02093B1368091B302D9
:10EFA0008917B1F48091AB02882391F02093332B21
:10EFB00011C08091B136882369F40E94AE0B909104
:10EFC000B2029295907F980F9093B5021092312BD8
:10EFD0001092332B9091B3028091B502981719F0DB
:10EFE00081E08093362B9091B3028091B50289170E
:10EFF000D1F42091312B2223B1F08091AB028823F0
:10F0000091F08091332B9091322B980F9093B50211
:10F0100091E09093362B8F5F8093332B8150821732
:10F0200010F01092332B809146029091470281306C
:10F03000910519F40E94E6268CC0892B09F087C03F
:10F040000E94E6268091F2358823C1F48091AB02BC
:10F050008823A1F41092F7331092F6339091FD3388
:10F060009093B5028091B302891719F081E08093E3
:10F07000362B81E080932C018093F2358091D80269
:10F08000882309F443C02091FA333091FB332115D2
:10F090003105E1F11092D8028091F335882391F087
:10F0A0001092F7331092F6339091FD339093B5029E
:10F0B0008091B302891719F081E08093362B10926A
:10F0C000F33521C08091F6339091F73301969093F8
:10F0D000F7338093F63301978217930720F010924D
:10F0E000F7331092F633E091F633F091F733EC50AA
:10F0F000FC4C91859093B5028091B302891719F069
:10F1000081E08093362B81E080932C0180919F36A3
:10F1100083FF1FC08091AB02882321F081E08093A0
:10F12000F33517C01092F7331092F6339091FD33F8
:10F130009093B5028091B302891719F081E0809312
:10F14000362B81E080932C018093F23502C010921F
:10F15000F23580914602909147020897D9F4809148
:10F16000F1018230B9F48091EF018250823090F445
:10F170008091933683FF07C00E94AE0B8093B40248
:10F1800081E080932C018091B4028B3018F08BE0E9
:10F190008093B40280914602909147020D9709F046
:10F1A0004BC08091913683FF05C00E944F6C81E077
:10F1B0008093B9038091893682FF3EC08091933657
:10F1C00083FF0DC083E090E0909347028093460256
:10F1D0000E94AE0B8093B10281E080932C0180915C
:10F1E0008B3683FF0CC087E090E0909347028093BA
:10F1F000460280E18093B10281E080932C018091EE
:10F200009B3683FF0CC083E090E09093470280938D
:10F21000460280E18093B10281E080932C018091CD
:10F22000993683FF09C086E090E09093470280936F
:10F23000460281E080932C01809146029091470222
:10F240000E9769F48091933684FF09C083E090E0C3
:10F25000909347028093460281E080932C01809135
:10F26000F035882349F08091F5330E94A66710920B
:10F27000F03581E080932C018091362B8823B1F109
:10F280001092362B81E080932C01EBE3FBE211928C
:10F29000BBE2EB34FB07D9F71092382B1092B9037D
:10F2A0008091873682FD04C08091AB02882389F467
:10F2B0008091B5026091352B0E94CE698091B50294
:10F2C0008093B3020E944F268091B3020E94A12C2A
:10F2D0000DC060E08091352B882309F461E08091B6
:10F2E000B5020E94CE6981E08093372B8091372B45
:10F2F0008823A1F08091AB02882381F41092372BF0
:10F3000090E08091352B882309F491E09093352B80
:10F310000E944F268091B3020E94A12C8091E63674
:10F32000882331F08091B3020E94A12C1092E6361E
:10F3300080918B3683FF16C08091893682FD12C082
:10F34000CBE3DBE210E08881882341F018828091D2
:10F35000B302612F0E94E5630E9462391F5F21960C
:10F36000103189F78091B9038823B9F080918B36E9
:10F3700083FF13C08091893682FD0FC080914602C1
:10F3800090914702049749F01092B9038091B3021B
:10F3900060E10E94E5630E9462398091E336882330
:10F3A000A1F080918B3683FF10C08091893682FD59
:10F3B0000CC08091460290914702049731F0109260
:10F3C000E3368091B3020E94062C8091F1358823A8
:10F3D000A1F080918B3683FF10C08091893682FD29
:10F3E0000CC08091460290914702049731F0109230
:10F3F000F1358091F5330E94C76180918B3684FF8F
:10F4000003C081E080932C018091460290914702D5
:10F41000059709F0C7C08091893682FD63C080914D
:10F420008F3682FD06C08091B2369091B3360E942D
:10F43000F90A8091873682FF35C080918F3683FD2F
:10F4400004C080919F3683FF07C01092F133109261
:10F45000F0331092CA3615C080919B3683FF22C0CC
:10F460008091392B882381F08091F202882349F41E
:10F470001092F1331092F0331092F2021092392B65
:10F480000EC01092F2020BC01092F20281E0809343
:10F49000392B8FEF9FEF9093F1338093F03381E01E
:10F4A00080932C018091993683FF0BC090E080916E
:10F4B000CA36882309F491E09093CA3681E080939C
:10F4C0002C0180919B3683FF1EC08091873682FD80
:10F4D0001AC090E08091F202882309F491E09093A1
:10F4E000F2020EC08091933683FF0DC083E090E05E
:10F4F00090934702809346020E94AE0B8093B10224
:10F5000081E080932C019091B3028091B50289171C
:10F51000D1F42091312B2223B1F08091AB028823CA
:10F5200091F08091332B9091322B980F9093B502EC
:10F5300091E09093362B8F5F8093332B815082170D
:10F5400010F01092332B80918F3684FF15C02091DC
:10F55000F2333091F3332115310571F08091F0339E
:10F560009091F133822793279093F1338093F03376
:10F570001092F3331092F23380918F3682FF12C0D3
:10F580006091F2337091F33380E00E948008909391
:10F59000F3338093F23306C00E94AE0B882309F048
:10F5A000CBC996C9DF91CF911F910F91FF90EF903A
:10F5B000DF90CF90BF90AF909F908F9008958091F3
:10F5C000AB02882311F4109205360E94FC280E9499
:10F5D00056510E94FD160E94F3620E94EE6D0E9439
:10F5E0007A3B0E94951B0895FF920F931F930E94F0
:10F5F000396CE8E6F6E31082329686E3E838F807DD
:10F60000D1F71092AC361092A43610929A3610921E
:10F61000903684EA98E367E570E00E94EC7E84EA25
:10F6200098E36FEF0E946E7F84EA98E36DEF0E948B
:10F630006E7F84EA98E30E94B17F84EA98E367E5ED
:10F6400070E043E050E00E94C27F84EA98E30E94A9
:10F65000FF7E082F84EA98E30E94FF7EF82E84EA5A
:10F6600098E30E94FF7E10E00F0D111D080F111D81
:10F670000430110531F00E949F390E9435660E94C6
:10F68000D32B0E94BE1080910736843051F40E9423
:10F690007D398FE70E94161080E094E00E94E10F10
:10F6A000F8CF80910636833041F40E949F390E9442
:10F6B00035660E94D32B0E94902C0E94482D809189
:10F6C0000836803F51F490E080910936882309F490
:10F6D00091E0909309360E94982C0E944269809193
:10F6E0006800816080936800D89A80916B00836085
:10F6F00080936B0080E06091352B0E94CE690E9460
:10F700004F2680E090E00E94770F0E94751F80E0F6
:10F710000E94A6671092B1008091B1008093B00062
:10F720008091B00082608093B0008091B1008260CF
:10F730008093B1008FE78093B30080917000826066
:10F74000809370000E943A2D789487E097E360E000
:10F750004BE65AE00E94BC7D87E097E361E043E717
:10F760005AE00E94BC7D87E097E362E04BE75AE0F5
:10F770000E94BC7D87E097E363E043E85AE00E9483
:10F78000BC7D87E097E364E04BE85AE00E94BC7DD3
:10F7900087E097E365E043E95AE00E94BC7D87E09B
:10F7A00097E360E142E020E00E94EC7D87E097E390
:10F7B00060E00E947C7D87E097E361E00E947C7DB1
:10F7C00087E097E362E00E947C7D87E097E364E056
:10F7D00040E00E94867D87E097E364EC0E947D868E
:10F7E00087E097E36EED0E947D8687E097E367ED03
:10F7F0000E947D8687E097E361ED0E947D8687E029
:10F8000097E369E040E00E94867D87E097E36CEB38
:10F810000E947D8687E097E360EB0E947D8687E00B
:10F8200097E369EB0E947D8687E097E36FEB0E9488
:10F830007D8687E097E36BEB0E947D8687E097E308
:10F8400060EB0E947D8687E097E360E041E00E94E4
:10F85000867D87E097E363E00E947C7D87E097E305
:10F8600064E00E947C7D87E097E365E00E947C7DF8
:10F8700087E097E366E041E00E94867D87E097E3BA
:10F880006BED7AE00E945A8660ED77E080E090E0D0
:10F890000E94AF8487E097E360E04BE95AE00E9462
:10F8A000BC7D87E097E361E043EA5AE00E94BC7DBB
:10F8B00087E097E362E04BEA5AE00E94BC7D87E074
:10F8C00097E363E043EB5AE00E94BC7D87E097E357
:10F8D00064E04BEB5AE00E94BC7D87E097E365E073
:10F8E00043EC5AE00E94BC7D87E097E366E04BEC76
:10F8F0005AE00E94BC7D87E097E367E043ED5AE061
:10F900000E94BC7D87E097E360E142E020E00E9436
:10F91000EC7D1F910F91FF900895982F809197375C
:10F920008230E0F42FB7F894913029F0913060F0F4
:10F93000923029F402C092E008C094E006C082E050
:10F94000809397372FBF089591E081E08093973798
:10F9500080919837892B809398372FBF089584E042
:10F9600061E00E94E08584E061E00E947C858CB5C6
:10F9700080618CBD8CB580648CBD87E061E00E94A5
:10F980007C8585E061E00E947C8508950F931F933C
:10F990008C01FC01868160E00E94E08581E090E0BE
:10F9A0000E940885F801868161E00E94E08581E07F
:10F9B00090E00E940885F801868160E00E94E08561
:10F9C00084E690E00E9408851F910F910895CF92E0
:10F9D000DF92EF92FF920F931F93CF93DF93D82E76
:10F9E000C92E282F392FC9018C01C0E0D0E0E62EA6
:10F9F000FF24F801878161E00E947C85B7010C2E0D
:10FA000002C0759567950A94E2F76170F8018781E5
:10FA10000E94E08521960F5F1F4FC830D10549F73E
:10FA20008D2D9C2D0E94C67CDF91CF911F910F914F
:10FA3000FF90EF90DF90CF900895CF92DF92EF92FA
:10FA4000FF920F931F93CF93DF93D82EC92E282FA9
:10FA5000392FC9018C01C0E0D0E0E62EFF24F80167
:10FA6000878161E00E947C85B7010C2E02C07595EC
:10FA700067950A94E2F76170F80187810E94E0853A
:10FA800021960F5F1F4FC430D10549F78D2D9C2D56
:10FA90000E94C67CDF91CF911F910F91FF90EF9054
:10FAA000DF90CF9008951F93CF93DF93EC01162F33
:10FAB0008C81642F0E94E0858D818F3F19F060E07A
:10FAC0000E94E0858F8584FF05C0CE01612F0E94D2
:10FAD000E77C0EC0612F70E084E0759567958A958C
:10FAE000E1F7CE010E941D7DCE01612F0E941D7D98
:10FAF000DF91CF911F91089541E00E94537D81E0F5
:10FB000090E0089540E00E94537D0895DF93CF93E5
:10FB1000CDB7DEB728970FB6F894DEBF0FBECDBFC6
:10FB20009C01FE013196A4ECB1E088E00D900192B9
:10FB30008150E1F7F9018389481708F040E0E42F8C
:10FB4000F0E0EE0FFF1FEC0FFD1F8181680F606872
:10FB5000C9010E94827D28960FB6F894DEBF0FBEC1
:10FB6000CDBFCF91DF91089562E00E94827D80ED4C
:10FB700097E00E9408850895EF92FF920F931F93DC
:10FB8000CF93DF938C017A0170E06770707023E08F
:10FB9000660F771F2A95E1F760640E94827DC0E0BE
:10FBA000D0E0F701EC0FFD1F4491F801A081B18175
:10FBB0002D913C91C801642FF90109952196C83017
:10FBC000D10579F7C8010E94B47DDF91CF911F91D3
:10FBD0000F91FF90EF900895CF93DF93EC014230A7
:10FBE00018F08F8588608F874B8B1C8A222329F021
:10FBF000413019F48F8584608F8780E593EC0E94F3
:10FC000008858C8160E00E94E0858E8160E00E9422
:10FC1000E0858D818F3F19F060E00E94E085CE0184
:10FC200063E00E941D7D88E893E10E940885CE0173
:10FC300068E00E941D7D88E893E10E940885CE015E
:10FC400062E00E941D7D88E893E10E940885CE0154
:10FC500062E00E941D7D88E893E10E940885CE0144
:10FC600068E00E941D7D88E893E10E940885CE012E
:10FC700068E00E94827D88E893E10E940885CE01B9
:10FC800061E00E94827D88E893E10E940885CE01B0
:10FC900066E00E94827D88E893E10E940885CE019B
:10FCA00062E00E94827D88E893E10E940885CE018F
:10FCB0006CE00E94827D88E893E10E940885DF91D4
:10FCC000CF9108956F927F928F92AF92CF92EF92E1
:10FCD0000F931F93DF93CF93CDB7DEB73C01162F61
:10FCE000842FF301448325830683E782C086A1869F
:10FCF00082869D8593879E8594879F859587988921
:10FD0000968761E00E947C85F30185818F3F19F021
:10FD100061E00E947C85F301868161E00E947C8520
:10FD2000112319F0F301178603C080E1F3018787DF
:10FD3000C30160E141E020E00E94EC7DCF91DF91C2
:10FD40001F910F91EF90CF90AF908F907F906F9019
:10FD500008958F92AF92CF92EF920F931F93CF930C
:10FD6000DF93DC01362F542F722F102FAE2C8C2CEA
:10FD700013961C921E92129780EC91E011969C9320
:10FD80008E9300D000D0EDB7FEB73196CDB7DEB779
:10FD90001982118212821382CD0161E0432F2FEF6D
:10FDA000052FE72EC12E0E94627E0F900F900F90BC
:10FDB0000F90DF91CF911F910F91EF90CF90AF9067
:10FDC0008F90089581E08093A33860931E3810923D
:10FDD000A1381092A238089581E08093A3386093EF
:10FDE0001E381092A1381092A238089520911D3823
:10FDF00030E080911C38281B3109C90108954091D9
:10FE00001C3880911D38481718F02FEF3FEF0AC0BB
:10FE1000E42FF0E0E656F84C8081282F30E04F5F69
:10FE200040931C38C9010895E0911C3880911D3819
:10FE3000E81718F0EFEFFFEF06C0F0E0E656F84CD9
:10FE40008081E82FF0E0CF01089508951092A7383F
:10FE50001092A63888EE93E0A0E0B0E08093A83836
:10FE60009093A938A093AA38B093AB3880ED91E075
:10FE70009093A5388093A4380895CF92DF92EF92A3
:10FE8000FF920F931F93CF93DF937C016B018A0145
:10FE90008091A3388823A1F0C0E0D0E00DC0D70145
:10FEA000ED91FC91D601AC0FBD1F0190F081E02DCA
:10FEB000C7016C9109952196C017D10780F304C042
:10FEC000CB01642F0E947380C801DF91CF911F91F5
:10FED0000F91FF90EF90DF90CF900895DF93CF9335
:10FEE0000F92CDB7DEB7FC0169838091A3388823D8
:10FEF000C9F08091A238823838F081E090E0938395
:10FF0000828320E030E015C08091A138E82FF0E036
:10FF1000E15EF74C998190838F5F8093A138809345
:10FF2000A23805C0CE01019661E00E94738021E0F5
:10FF300030E0C9010F90CF91DF9108950F93062F04
:10FF400080911E386FE178E34091A23821E00E9451
:10FF50001E801092A1381092A2381092A3380F91EF
:10FF6000089561E00E949E7F0895433808F042E8BA
:10FF7000862F6AE977E30E94D57F10921C38809320
:10FF80001D38089521E00E94B57F089521E00E9468
:10FF9000B57F089510921C3810921D381092A13828
:10FFA0001092A2380E9423820895382F433810F00F
:10FFB00040E042C08091B0388823E1F791E090930F
:10FFC000B0382093B2388FEF8093433A10923A3989
:10FFD000415040933B394F5F9093B1388091B13895
:10FFE000330F832B8093B1388091B338813041F443
:10FFF0001092B3388091B1388093BB0085EC01C07A
:020000021000EC
:1000000085EE8093BC008091B0388130E1F380911F
:100010003A39841710F440913A3920E030E00AC0B0
:10002000FB01E20FF31FD901A854B74C8C918083D8
:100030002F5F3F4F2417A0F3842F08950F931F9332
:10004000582F122F433810F081E04AC08091B03809
:100050008823E1F782E08093B0380093B2388FEFC5
:100060008093433A10923A3940933B39A8EBB8E376
:10007000FB0102C081918D938E2F861B8417D0F3D4
:100080001092B1388091B138550F852B8093B138DB
:100090008091B338813041F41092B3388091B138F7
:1000A0008093BB0085EC01C085EE8093BC001123DA
:1000B00021F08091B0388230E1F38091433A8F3F54
:1000C00011F480E00DC08091433A803211F482E057
:1000D00007C08091433A803311F084E001C083E08F
:1000E0001F910F910895482F633810F081E0089513
:1000F0008091B038843011F082E008956093BF3968
:10010000ACE3B9E3842F9C01F90102C081918D9386
:100110008E2F841B8617D0F380E008951F920F92D4
:100120000FB60F920BB60F9211242F933F934F935C
:100130005F936F937F938F939F93AF93BF93EF934F
:10014000FF938091B90090E0887F90708036910590
:1001500009F4F2C081369105CCF58832910509F495
:100160007BC089329105B4F48031910509F46FC0E8
:10017000813191053CF4009709F447C1089709F0D3
:100180004FC165C08831910509F466C0809709F0B8
:1001900047C182C08034910509F4A4C0813491051F
:1001A00044F48033910509F482C0C89709F038C13E
:1001B00089C08035910509F489C08835910509F415
:1001C00096C08834910509F02BC1AEC088399105DD
:1001D00009F413C189399105ECF48837910509F4C4
:1001E000ABC0893791054CF48836910509F4A4C059
:1001F0008037910509F014C19FC08838910509F432
:10020000FCC08039910509F49DC08038910509F042
:1002100007C198C0803B910509F4C6C0813B910598
:100220004CF4803A910509F49FC0883A910509F091
:10023000F7C0BAC0803C910509F4E3C0883C910541
:1002400009F4DFC0883B910509F0EAC0C2C0809183
:10025000B1388093BB00CFC090913A3980913B393F
:10026000981768F490913A39E92FF0E0E854F74C88
:1002700080818093BB009F5F90933A39BCC080918E
:10028000B238882309F44BC085ED8093BC0080917F
:10029000BC0084FDFCCFC2C080E28093433A85ED70
:1002A0008093BC008091BC0084FDFCCFB7C080E38C
:1002B0008093433A85ED8093BC008091BC0084FD1F
:1002C000FCCFACC088E38093433A9BC080913A391D
:1002D0009091BB00E82FF0E0E854F74C90838F5FDB
:1002E00080933A3990913A3980913B3982C080911C
:1002F0003A399091BB00E82FF0E0E854F74C908336
:100300008F5F80933A398091B238882341F085ED30
:100310008093BC008091BC0084FDFCCF7FC081E055
:100320008093B33884EA6EC085ED8093BC008091E1
:10033000BC0084FDFCCF72C083E08093B038109283
:10034000423A59C08091423A823808F056C08091B2
:10035000423A9091BB00E82FF0E0E054F64C9083D5
:100360008F5F8093423A47C08091423A823830F49E
:10037000E091423AF0E0E054F64C108285ED809333
:10038000BC008091BC0084FDFCCF1092B03860911D
:10039000423AE091B638F091B73880EC99E370E0DA
:1003A00009951092423A2DC084E08093B0381092A3
:1003B000BE391092BF39E091B438F091B538099543
:1003C0008091BF39882329F481E08093BF3910924E
:1003D0003C399091BE39E92FF0E0E45CF64C808125
:1003E0008093BB009F5F9093BE399091BE398091FE
:1003F000BF39981710F485EC01C085E88093BC00E4
:100400000FC085EC8093BC0009C01092433A85ED83
:100410008093BC008091BC0084FDFCCF1092B0386A
:10042000FF91EF91BF91AF919F918F917F916F91CC
:100430005F914F913F912F910F900BBE0F900FBE88
:100440000F901F9018951092B03881E08093B238C9
:100450001092B33881E161E00E94E08580E161E0C3
:100460000E94E085E9EBF0E080818E7F80838081CF
:100470008D7F808388E48093B80085E48093BC00FE
:100480000895F999FECF72BD61BDF89A80B50895BF
:10049000F999FECF1FBA72BD61BD40BD0FB6F89489
:1004A000FA9AF99A0FBE089508951F920F920FB607
:1004B0000F920BB60F9211242F933F934F938F936C
:1004C0009F93EF93FF934091C6002091853A30911E
:1004D000863A2F5F3F4F2F7330708091873A90910B
:1004E000883A2817390759F0E091853AF091863A11
:1004F000EB5BF54C40833093863A2093853AFF912D
:10050000EF919F918F914F913F912F910F900BBE43
:100510000F900FBE0F901F901895E091613BF091E6
:10052000623BE05CFF4F8191919120813181821B80
:10053000930B8F739070892B11F00E945482089551
:100540001F920F920FB60F920BB60F9211242F939A
:100550003F938F939F93EF93FF932091C93A3091EC
:10056000CA3A8091CB3A9091CC3A2817390731F4A6
:100570008091C1008F7D8093C10014C0E091CB3A7F
:10058000F091CC3AE757F54C20818091CB3A90918D
:10059000CC3A01968F7390709093CC3A8093CB3A7B
:1005A0002093C600FF91EF919F918F913F912F91E2
:1005B0000F900BBE0F900FBE0F901F9018951F92BB
:1005C0000F920FB60F920BB60F9211242F933F93F9
:1005D0008F939F93EF93FF932091513B3091523B28
:1005E0008091533B9091543B2817390731F4809107
:1005F000C9008F7D8093C90014C0E091533BF091F6
:10060000543BEF5EF44C20818091533B9091543BDE
:1006100001968F7390709093543B8093533B20933B
:10062000CE00FF91EF919F918F913F912F910F906D
:100630000BBE0F900FBE0F901F901895DC011C96FB
:10064000ED91FC911D97E05CFF4F219131918081EC
:100650009181281B390B2F733070C9010895DC017B
:100660001C96ED91FC911D97E05CFF4F208131813C
:10067000E054F040DF01AE5BBF4F8D919C9111972C
:100680002817390719F42FEF3FEF07C08D919C9180
:10069000E80FF91F8081282F30E0C9010895DC019F
:1006A0001C96ED91FC911D97E05CFF4F20813181FC
:1006B000E054F040DF01AE5BBF4F8D919C911197EC
:1006C0002817390719F42FEF3FEF10C08D919C9137
:1006D0001197E80FF91F20818D919C911197019638
:1006E0008F73907011969C938E9330E0C90108959A
:1006F000FC0186859785DC01A05CBF4FFC01EE5BA9
:10070000FF4F2D913C9111978081918128173907D6
:10071000C1F70895CF93DF93EC01EE85FF85E05C90
:10072000FF4F20813181E054F0402F5F3F4F2F7306
:100730003070DF01AE5BBF4F8D919C9111972817F0
:100740003907D1F3E05CFF4F80819181E054F040A4
:10075000E80FF91F6083EE85FF85E05CFF4F318372
:100760002083EE89FF89208181E090E00D8C02C01A
:10077000880F991F0A94E2F7282B208381E090E0EC
:10078000DF91CF9108951F931092583B1092573BE1
:1007900028EE33E040E050E02093593B30935A3B41
:1007A00040935B3B50935C3B60EE71E07093563B33
:1007B0006093553B85E49AE39093623B8093613B61
:1007C00089E89AE39093643B8093633B85EC90E0E7
:1007D0009093663B8093653B84EC90E09093683BFC
:1007E0008093673B80EC90E090936A3B8093693BF9
:1007F00081EC90E090936C3B80936B3B86EC90E0B7
:1008000090936E3B80936D3B14E010936F3BB3E08D
:10081000B093703BA7E0A093713BF5E0F093723B7F
:10082000E1E0E093733B1092773B1092763B20938C
:10083000783B3093793B40937A3B50937B3B70936A
:10084000753B6093743B8DEC9AE39093813B80936E
:10085000803B81E19BE39093833B8093823B8DECD3
:1008600090E09093853B8093843B8CEC90E0909358
:10087000873B8093863B88EC90E09093893B809304
:10088000883B89EC90E090938B3B80938A3B8EEC85
:1008900090E090938D3B80938C3B10938E3BB09374
:1008A0008F3BA093903BF093913BE093923B1F9141
:1008B00008951F920F920FB60F9211242F933F931A
:1008C0008F939F93AF93BF938091973B9091983B69
:1008D000A091993BB0919A3B30919B3B0196A11D11
:1008E000B11D232F2D5F2D3720F02D570196A11D0F
:1008F000B11D20939B3B8093973B9093983BA09393
:10090000993BB0939A3B8091933B9091943BA091FB
:10091000953BB091963B0196A11DB11D8093933BF1
:100920009093943BA093953BB093963BBF91AF912E
:100930009F918F913F912F910F900FBE0F901F901D
:1009400018958FB7F8942091973B3091983B409140
:10095000993B50919A3B8FBFB901CA0108959B0101
:10096000AC017FB7F8948091933B9091943BA09118
:10097000953BB091963B66B5A89B05C06F3F19F0BB
:100980000196A11DB11D7FBFBA2FA92F982F8827CF
:10099000860F911DA11DB11D62E0880F991FAA1F2E
:1009A000BB1F6A95D1F7BC012DC0FFB7F8948091A9
:1009B000933B9091943BA091953BB091963BE6B5CB
:1009C000A89B05C0EF3F19F00196A11DB11DFFBF07
:1009D000BA2FA92F982F88278E0F911DA11DB11D09
:1009E000E2E0880F991FAA1FBB1FEA95D1F7861B6B
:1009F000970B885E9340C8F22150304040405040F1
:100A000068517C4F211531054105510571F6089556
:100A1000019739F0880F991F880F991F0297019746
:100A2000F1F70895789484B5826084BD84B58160BF
:100A300084BD85B5826085BD85B5816085BDEEE6E6
:100A4000F0E0808181608083E1E8F0E010828081C5
:100A500082608083808181608083E0E8F0E0808133
:100A600081608083E1EBF0E0808184608083E0EB53
:100A7000F0E0808181608083E1E9F0E08081826044
:100A80008083808181608083E0E9F0E08081816003
:100A90008083EAE7F0E080818460808380818260E7
:100AA00080838081816080838081806880831092D0
:100AB000C1000895982F883108F09851977080915F
:100AC000AB018295880F880F807C892B80937C00F6
:100AD00080917A00806480937A0080917A0086FD0C
:100AE000FCCF2091780040917900942F80E030E095
:100AF000282B392BC9010895482F50E0CA01805E88
:100B0000944FFC0124914050554FFA018491882361
:100B1000C1F0E82FF0E0EE0FFF1FEE51F54FA59169
:100B2000B491662341F49FB7F8948C912095822369
:100B30008C939FBF08959FB7F8948C91822B8C93D0
:100B40009FBF08958430C9F0853038F48230F1F0C9
:100B5000833078F4813099F516C08730F9F0883009
:100B600018F4863061F516C08830F1F0893039F517
:100B700021C0809180008F7703C0809180008F7D9D
:100B800080938000089584B58F7702C084B58F7DEF
:100B900084BD08958091B0008F7703C08091B0002C
:100BA0008F7D8093B0000895809190008F7780931F
:100BB00090000895809190008F7D8093900008951B
:100BC000FF920F931F93F62E482F50E0CA01805CCE
:100BD000944FFC012491CA01805E944FFC01149152
:100BE0004050554FFA0104910023C9F0222319F017
:100BF000822F0E94A285E02FF0E0EE0FFF1FE4514C
:100C0000F54FA591B4919FB7F894FF2021F48C91F2
:100C10001095812302C08C91812B8C939FBF1F91D3
:100C20000F91FF900895CF93DF930E9412850E9449
:100C3000F47ACDE8D2E80E94DF7A2097E1F30E94AF
:100C40008D82F9CFFC0120E030E08081882311F40F
:100C500021E030E0C9010895FC0181E0808308951E
:100C6000CF92DF92EF92FF920F931F93CF93DF9378
:100C70007C016B018A01C0E0D0E00FC0D6016D910C
:100C80006D01D701ED91FC910190F081E02DC7013C
:100C90000995C80FD91F015010400115110571F7B2
:100CA000CE01DF91CF911F910F91FF90EF90DF90D8
:100CB000CF900895EF92FF920F931F93CF93DF93FE
:100CC0007C018B01C0E0D0E0F8010F5F1F4F649101
:100CD000662359F0D701ED91FC910190F081E02D50
:100CE000C7010995C80FD91FEFCFCE01DF91CF9172
:100CF0001F910F91FF90EF900895DC01ED91FC9111
:100D00000190F081E02D09950895CF93DF93DB01E9
:100D10000D900020E9F71197A61BB70BEC01E881B5
:100D2000F9810280F381E02DAD010995DF91CF912A
:100D300008954F925F927F928F929F92AF92BF924F
:100D4000CF92DF92EF92FF920F931F93DF93CF9397
:100D5000CDB7DEB7A1970FB6F894DEBF0FBECDBFFB
:100D60002C01742ECB01223008F42AE019A231E2C2
:100D7000C32ED12CCC0EDD1E822E9924AA24BB2496
:100D8000672D752FA50194010E94818D79018A013B
:100D9000C801B701A50194010E942F8D472D461B64
:100DA0000894C108D1084A3014F4405D01C0495C80
:100DB000F6014083E114F1040105110521F07E2CB8
:100DC0005F2DC801DDCFC201B6010E948586A196C4
:100DD0000FB6F894DEBF0FBECDBFCF91DF911F914C
:100DE0000F91FF90EF90DF90CF90BF90AF909F90CA
:100DF0008F907F905F904F900895DC012115310511
:100E000041F4ED91FC910190F081E02D642F099562
:100E100008950E9499860895EF92FF920F931F9371
:100E20009A017B0100E010E0B801A7010E94FD8655
:100E30001F910F91FF90EF900895EF92FF920F9303
:100E40001F939A01E62EFF2400E010E0B801A701ED
:100E50000E94FD861F910F91FF90EF900895CF9211
:100E6000DF92EF92FF920F931F93CF93DF93EC01EA
:100E70006A017B012115310541F4E881F981019076
:100E8000F081E02D642F09951FC02A303105D1F47F
:100E900077FF17C0E881F9810190F081E02D6DE2C4
:100EA00009958C0144275527BA014C195D096E0933
:100EB0007F09CE012AE00E9499869801280F391FE8
:100EC00004C02AE00E9499869C01C901DF91CF915C
:100ED0001F910F91FF90EF90DF90CF900895EF92C8
:100EE000FF920F931F937B019A010027F7FC009557
:100EF000102FB801A7010E942F871F910F91FF901B
:100F0000EF9008950E94858608957F928F929F9218
:100F1000AF92BF92CF92DF92EF92FF920F931F9307
:100F2000CF93DF934C017A018B01722ECB01BA0172
:100F300020E030E040E050E00E94798B87FD03C064
:100F4000C0E0D0E00EC0D401ED91FC910190F081A1
:100F5000E02DC4016DE20995EC0117FB109517F91E
:100F6000109520E030E040E05FE3AA240BC0CA0106
:100F7000B90120E030E040E251E40E947D8B9B010A
:100F8000AC01A394A71498F3C801B7010E94158B74
:100F90005B016C010E94EA8B7B018C01C401B801EA
:100FA000A7012AE030E00E94FD86C80FD91F7720F4
:100FB00039F0C40160E271E00E948586C80FD91F34
:100FC000C801B7010E94168C9B01AC01C601B50196
:100FD0000E94148B24C020E030E040E251E40E94E3
:100FE000CC8C7B018C010E94E58B5B016C01CC24D5
:100FF000B7FCC094DC2CC401B601A5012AE030E0A6
:101000000E942F87C80FD91FC601B5010E94188CF6
:101010009B01AC01C801B7010E94148B7A94772020
:10102000D1F6CE01DF91CF911F910F91FF90EF90FC
:10103000DF90CF90BF90AF909F908F907F9008955A
:101040000E9485870895AF92BF92CF92DF92EF9270
:10105000FF920F931F93CF93DF935C016B01EE24FC
:10106000FF24C0E0D0E010C0D501ED91FC910081DB
:101070001181C601BE010E949E88682FC501F8013A
:101080000995E80EF91E2196F60184819581C8170D
:10109000D90750F3C701DF91CF911F910F91FF90B6
:1010A000EF90DF90CF90BF90AF900895EF92FF92B6
:1010B0000F931F937B018C016115710581059105CB
:1010C00029F420E030E040E050E00BC00E943607F9
:1010D000A80197010E94A38DAC01CB01DA019C010C
:1010E000AD01B901CA011F910F91FF90EF900895D2
:1010F000EF92FF920F931F937B018C01621773078E
:101100008407950764F4261B370B480B590BCA015B
:10111000B9010E945688E60EF71E081F191FB70175
:10112000C8011F910F91FF90EF900895009729F04B
:10113000BC0180E090E00E943B070895FC0184819F
:1011400095816817790748F40190F081E02D309778
:1011500021F0E60FF71F8081089580E00895CF9376
:10116000DF939C01FB01EC01A881B981109729F064
:101170006081718161157105D1F4C081D1812097A1
:1011800059F084819581892B39F0888190E022275C
:101190003327281B390B12C0109771F0F901848195
:1011A0009581892B49F08C91282F30E007C0CD0123
:1011B0000E9429089C0102C020E030E0C901DF91B3
:1011C000CF910895FC01DB012481358114968D9126
:1011D0009C9115972817390711F020E007C0CF011F
:1011E0000E94AF8820E0892B09F421E0822F089526
:1011F0000F931F93CF93DF93EC018B016F5F7F4FB2
:10120000888199810E944407009711F480E005C00D
:10121000998388831B830A8381E0DF91CF911F919B
:101220000F910895CF93DF93EC0188819981892BE9
:1012300029F08A819B818617970760F4CE010E946E
:10124000F888882341F08C819D81892B19F4E881ED
:10125000F981108281E0DF91CF910895EF92FF92A2
:101260000F931F93CF93DF93EC017B016C817D8102
:10127000E114F104C1F04115510599F08A01060FFE
:10128000171FB8010E941289882369F0888199810B
:101290002C813D81820F931FB7010E9432081D836C
:1012A0000C8381E001C080E0DF91CF911F910F910D
:1012B000FF90EF900895DF93CF9300D0CDB7DEB7C6
:1012C00069831A82BE016F5F7F4F41E050E00E9448
:1012D0002E890F900F90CF91DF910895CF93DF93D8
:1012E000EC0188819981009711F00E948B06198288
:1012F00018821D821C821B821A82DF91CF91089571
:101300000F931F93182F092F0E945B89882321F4C4
:10131000812F902F0E946E89812F902F1F910F9106
:1013200008950F931F93182F092FFB01608171817E
:10133000448155810E942E89882321F4812F902F8A
:101340000E946E89812F902F1F910F910895EF9227
:10135000FF920F931F93CF93DF93EC017B018A01E0
:10136000BA010E941289882321F4CE010E946E895D
:1013700007C01D830C8388819981B7010E943208C0
:10138000CE01DF91CF911F910F91FF90EF900895C3
:10139000CF93DF93EC01198218821B821A821D827F
:1013A0001C821E826115710551F0DB010D90002039
:1013B000E9F71197A61BB70BAD010E94A789DF9132
:1013C000CF910895CF93DF93EC01198218821B828D
:1013D0001A821D821C821E826115710551F0DB018B
:1013E0000D900020E9F71197A61BB70BAD010E94E5
:1013F000A789DF91CF9108950F931F93182F092F7D
:101400006115710559F0DB010D900020E9F7119786
:10141000A61BB70BAD010E94A78902C00E946E896E
:10142000812F902F1F910F910895EF92FF920F93AC
:101430001F93DF93CF93CDB7DEB761970FB6F894C4
:10144000DEBF0FBECDBF8C01CB01F801118210822F
:10145000138212821582148216827E010894E11C86
:10146000F11CB70150E00E945A08C801B7010E9460
:10147000FC8961960FB6F894DEBF0FBECDBFCF9149
:10148000DF911F910F91FF90EF900895EF92FF92DF
:101490000F931F93DF93CF93CDB7DEB762970FB64D
:1014A000F894DEBF0FBECDBF8C01CB01F8011182D5
:1014B0001082138212821582148216827E01089491
:1014C000E11CF11CB70150E00E943908C801B701C6
:1014D0000E94FC8962960FB6F894DEBF0FBECDBFA6
:1014E000CF91DF911F910F91FF90EF900895EF92B0
:1014F000FF920F931F93DF93CF93CDB7DEB729975A
:101500000FB6F894DEBF0FBECDBF8C01862FF80159
:10151000118210821382128215821482168290E048
:101520007E010894E11CF11CB70150E00E945A08AA
:10153000C801B7010E94FC8929960FB6F894DEBF56
:101540000FBECDBFCF91DF911F910F91FF90EF9014
:101550000895DF93CF9300D0CDB7DEB7FC011182A1
:1015600010821382128215821482168269831A8273
:10157000BE016F5F7F4F0E94FC890F900F90CF914B
:10158000DF910895DF93CF9300D0CDB7DEB7FC0194
:10159000118210821382128215821482168269834C
:1015A0001A82BE016F5F7F4F0E94FC890F900F90DF
:1015B000CF91DF910895CF93DF93EC01FB01861764
:1015C000970761F0608171816115710529F044818F
:1015D00055810E94A78902C00E946E89CE01DF91C9
:1015E000CF910895FC01118210821382128215821C
:1015F000148216820E94DB8A0895FC0111821082F7
:10160000138212821582148216820E94DB8A089548
:10161000FC01808191810E948B060895FC018081EC
:1016200091810E948B0608955058BB27AA270ED09F
:1016300075C166D130F06BD120F031F49F3F11F4C9
:101640001EF45BC10EF4E095E7FB51C1E92F77D1A1
:1016500080F3BA17620773078407950718F071F4CF
:101660009EF58FC10EF4E0950B2EBA2FA02D0B0125
:10167000B90190010C01CA01A0011124FF27591BD7
:1016800099F0593F50F4503E68F11A16F040A22FDD
:10169000232F342F4427585FF3CF4695379527954E
:1016A000A795F0405395C9F77EF41F16BA0B620B4D
:1016B000730B840BBAF09150A1F0FF0FBB1F661F94
:1016C000771F881FC2F70EC0BA0F621F731F841FD7
:1016D00048F4879577956795B795F7959E3F08F0FD
:1016E000B3CF9395880F08F09927EE0F97958795BC
:1016F0000895D9D008F481E008950CD00FC107D126
:1017000040F0FED030F021F45F3F19F0F0C05111ED
:1017100039C1F3C014D198F39923C9F35523B1F318
:10172000951B550BBB27AA2762177307840738F050
:101730009F5F5F4F220F331F441FAA1FA9F333D0AF
:101740000E2E3AF0E0E830D091505040E695001C63
:10175000CAF729D0FE2F27D0660F771F881FBB1F1F
:10176000261737074807AB07B0E809F0BB0B802DF9
:10177000BF01FF2793585F4F2AF09E3F510568F045
:10178000B6C000C15F3FECF3983EDCF386957795D9
:101790006795B795F7959F5FC9F7880F911D969547
:1017A000879597F90895E1E0660F771F881FBB1FA3
:1017B000621773078407BA0720F0621B730B840B50
:1017C000BA0BEE1F88F7E095089504D06894B11124
:1017D000D9C00895BCD088F09F5790F0B92F9927B1
:1017E000B751A0F0D1F0660F771F881F991F1AF02C
:1017F000BA95C9F712C0B13081F0C3D0B1E00895F5
:10180000C0C0672F782F8827B85F39F0B93FCCF375
:10181000869577956795B395D9F73EF49095809521
:10182000709561957F4F8F4F9F4F0895E89409C041
:1018300097FB3EF490958095709561957F4F8F4F03
:101840009F4F9923A9F0F92F96E9BB279395F69519
:10185000879577956795B795F111F8CFFAF4BB0F97
:1018600011F460FF1BC06F5F7F4F8F4F9F4F16C0FB
:10187000882311F096E911C0772321F09EE8872F85
:10188000762F05C0662371F096E8862F70E060E041
:101890002AF09A95660F771F881FDAF7880F9695BA
:1018A000879597F90895990F0008550FAA0BE0E85E
:1018B000FEEF16161706E807F907C0F01216130612
:1018C000E407F50798F0621B730B840B950B39F452
:1018D0000A2661F0232B242B252B21F408950A26B8
:1018E00009F4A140A6958FEF811D811D089597F9F8
:1018F0009F6780E870E060E008959FEF80EC0895B6
:1019000000240A94161617061806090608950024DE
:101910000A9412161306140605060895092E039458
:10192000000C11F4882352F0BB0F40F4BF2B11F4CC
:1019300060FF04C06F5F7F4F8F4F9F4F089557FD2B
:101940009058440F551F59F05F3F71F04795880F2D
:1019500097FB991F61F09F3F79F0879508951216C4
:1019600013061406551FF2CF4695F1DF08C0161670
:1019700017061806991FF1CF869571056105089421
:101980000895E894BB2766277727CB0197F9089538
:101990008ADF08F48FEF08950BD0C0CFB1DF28F0B5
:1019A000B6DF18F0952309F0A2CFA7CF1124EACF14
:1019B000C6DFA0F3959FD1F3950F50E0551F629FAE
:1019C000F001729FBB27F00DB11D639FAA27F00D98
:1019D000B11DAA1F649F6627B00DA11D661F829FBF
:1019E0002227B00DA11D621F739FB00DA11D621FA4
:1019F000839FA00D611D221F749F3327A00D611DC1
:101A0000231F849F600D211D822F762F6A2F1124A2
:101A10009F5750408AF0E1F088234AF0EE0FFF1FF5
:101A2000BB1F661F771F881F91505040A9F79E3F2C
:101A3000510570F05CCFA6CF5F3FECF3983EDCF32E
:101A4000869577956795B795F795E7959F5FC1F769
:101A5000FE2B880F911D9695879597F90895629FA3
:101A6000D001739FF001829FE00DF11D649FE00D96
:101A7000F11D929FF00D839FF00D749FF00D659FF7
:101A8000F00D9927729FB00DE11DF91F639FB00DF6
:101A9000E11DF91FBD01CF0111240895991B79E0C3
:101AA00004C0991F961708F0961B881F7A95C9F7EE
:101AB00080950895AA1BBB1B51E107C0AA1FBB1F3D
:101AC000A617B70710F0A61BB70B881F991F5A95CA
:101AD000A9F780959095BC01CD01089597FB092E3B
:101AE00007260AD077FD04D0E5DF06D000201AF4DF
:101AF000709561957F4F0895F6F7909581959F4F6A
:101B00000895A1E21A2EAA1BBB1BFD010DC0AA1F3E
:101B1000BB1FEE1FFF1FA217B307E407F50720F056
:101B2000A21BB30BE40BF50B661F771F881F991FD1
:101B30001A9469F760957095809590959B01AC011A
:101B4000BD01CF01089597FB092E05260ED057FD44
:101B500004D0D7DF0AD0001C38F45095409530955A
:101B600021953F4F4F4F5F4F0895F6F79095809521
:101B7000709561957F4F8F4F9F4F0895EE0FFF1F18
:101B80000590F491E02D09942F923F924F925F922D
:101B90006F927F928F929F92AF92BF92CF92DF927D
:101BA000EF92FF920F931F93CF93DF93CDB7DEB7E2
:101BB000CA1BDB0B0FB6F894DEBF0FBECDBF099476
:101BC0002A88398848885F846E847D848C849B84CD
:101BD000AA84B984C884DF80EE80FD800C811B81DB
:101BE000AA81B981CE0FD11D0FB6F894DEBF0FBE0A
:101BF000CDBFED0108951BE0C6E6DBE004C0FE01A9
:101C00000E94C08D2296C836D107C9F7F894FFCF3D
